:020000022000DC
:1060000000F0002035620200656202006762020053
:10601000696202006B6202006D6202000000000013
:106020000000000000000000000000006F6202009D
:1060300071620200000000007362020075620200DB
:10604000796202007B6202007D6202007F620200D0
:106050008162020083620200ED6D0200876202002D
:10606000896202008B620200155B03008F620200EE
:106070009162020093620200956202009762020040
:10608000996202006D93030015B802009F6202003E
:1060900095930300A36202001D890300A76202001A
:1060A000A9620200AB620200AD620200AF620200B0
:1060B000B1620200B36202007762020077620200FE
:1060C000B5620200B7620200B9620200BB62020060
:0C60D000BD620200BF620200C16202005B
:1060DC00354936480A1A02D0072291438D46344975
:1060EC0034480A1A06D00722914381F30988022208
:1060FC0082F3148830483149314A00F043F8314872
:10610C003149324A00F03EF831483249324A00F007
:10611C0039F832483249334A00F034F832483349BE
:10612C00334A00F02FF833483349344A00F02AF848
:10613C0033483449344A00F025F8344834490022B5
:10614C0000F02BF833483449002200F026F833488D
:10615C003349091A082903DB00220260043001606C
:10616C001F482049884205D00268043003B4904788
:10617C0003BCF7E700208646EC4600200021294AA4
:10618C009047FEE7884207D0521A05D003780130B9
:10619C000B700131013AF9D17047884202D002707C
:1061AC000130FAE77047000000F0002000E8002002
:1061BC0000F0002000F00020BC060400C8320020D3
:1061CC0028340020C4620200C462020064F203009E
:1061DC00BC060400C8320020C832002094F2030030
:1061EC0094F2030094F2030094F2030094F203007F
:1061FC0094F2030094F2030094F20300BC06040032
:10620C001C080400283400202834002028340020E6
:10621C00146B0020146B0020146B0020146B0020F6
:10622C00146F0020CD68020008484FF00701884326
:10623C008546074880470748016841F470010160B2
:10624C00BFF34F8FBFF36F8FFFF742BF00F00020FB
:10625C007597030088ED00E0FEE7FEE7FEE7FEE73A
:10626C00FEE7FEE7FEE7FEE7FEE7FEE7FEE7FEE7FA
:10627C00FEE7FEE7FEE7FEE7FEE7FEE7FEE7FEE7EA
:10628C00FEE7FEE7FEE7FEE7FEE7FEE7FEE7FEE7DA
:10629C00FEE7FEE7FEE7FEE7FEE7FEE7FEE7FEE7CA
:1062AC00FEE7FEE7FEE7FEE7FEE7FEE7FEE7FEE7BA
:0862BC00FEE7FEE7FEE700BF6C
:1062C40041DF704776DF70477ADF70477CDF7047C5
:1062D40008B504F01DF908BD2DE9F04188B004AFFC
:1062E40064212D4800F084FC08F02CFEA0B92B4B4F
:1062F4001B78BBB100F04AFF294B1B6813F4804F95
:1063040046D0284B1B68032B42DDE8468AB00DF1CA
:10631400100C6646002326E0234A4FF4957113F0CF
:1063240051FBE4E7214A3B1D07CA83E807001846EE
:1063340000F0F8FB0028DDD01B4A40F2351113F0C1
:1063440041FBD7E7C25C4FEA121E5900184C25687E
:1063540015F80EE006F813E002F00F02013124688C
:10636400A25C725401330F2BECD900238CF820303B
:10637400104BD3F80435CDF808C00F4A01920F4AE8
:10638400009240F239120E49042006F087FAC546FD
:106394001037BD46BDE8F081D166020028340020E4
:1063A4003833002034330020E0F3030094F2030078
:1063B4003C33002000B0004028F4030038F403000C
:1063C40020F4030000B583B09DF80430012262F389
:1063D400030362F3071302A800F8043D10220549E1
:1063E400FFF774FF10B903B05DF804FB13F0DCFA97
:1063F400F9E700BFC8F2030008B513F0D5FA08BDE9
:1064040000B583B0037823B1012B0BD003B05DF842
:1064140004FB3B214088FFF755FF0028F6D013F01A
:10642400C3FAF3E7094B1B6813F4804FEED0084B13
:106434001B68032BEADD074BD3F80435064A0092A8
:10644400BC220649042006F029FADFE7383300208D
:106454003433002000B0004068F3030020F403004C
:1064640000B58BB00023ADF808307823ADF80430C4
:10647400C823ADF806304FF4C873ADF80A3001A84C
:10648400FFF722FFC0B900230693079301AB0393E0
:1064940040F6CD4304934FF48033059303238DF8E2
:1064A4001830084B0893084B099303A812F04AFCD0
:1064B40028B90BB05DF804FB13F076FAE3E713F0A8
:1064C40073FAF6E705640200FD63020000B585B0C7
:1064D4001F4B1B6813F4804F03D01E4B1B68032B08
:1064E4001DDCFFF76FFFFFF7BBFF03A80DF012FDE4
:1064F400174B1B6813F4804F03D0164B1B68032BF8
:1065040018DC00214FF4F01000F0E7FB0422C8214E
:106514004FF4003000F0ECFB05B05DF804FB0E4BCB
:10652400D3F804350D4A00925E220D49042006F08A
:10653400B5F9D6E7084BD3F80435BDF80C20019221
:10654400084A009266220649042006F0A7F9D8E713
:10655400383300203433002000B00040ACF3030093
:1065640020F40300C8F3030008B5112000F098FBE1
:1065740008BD000010B582B00C460E4B1B6813F426
:10658400804F03D00C4B1B68032B06DC21461120E3
:1065940000F092FB204602B010BD084BD3F804353E
:1065A4000191074A009273220649042006F076F905
:1065B400ECE700BF383300203433002000B0004043
:1065C40094F3030020F4030000B583B00F4B1B6861
:1065D40013F4804F03D00E4B1B68032B0ADC0322F9
:1065E400C8214FF4003000F083FB08F0B5FC03B081
:1065F4005DF804FB074BD3F80435074A00927A226E
:106604000649042006F04AF9E9E700BF38330020C0
:106614003433002000B000404CF3030020F40300A6
:1066240010B582B00446224B1B6813F4804F03D08C
:10663400204B1B68032B04DC7CB1032C30D002B04C
:1066440010BD1D4BD3F8043501901C4A00928A22D8
:106654001B49042006F022F9EEE7112000F020FB8C
:1066640080F00100C4B2124B1B6813F4804F03D0B6
:10667400104B1B68032B08DC2146112000F01CFB87
:106684002146104818F0C2FBD9E70B4BD3F8043568
:106694000D4A009293220A49042006F0FFF8EBE722
:1066A40009F0B6FF08F0FEFBFFF78EFFC7E700BF57
:1066B400383300203433002000B00040A4F203003B
:1066C40020F403002C340020B8F2030030380428EE
:1066D40000D9704708B5FFF7A3FF08BD08B50378D4
:1066E4001C2B00D008BDFFF76FFFFBE700B58FB090
:1066F400174BDB680EA941F8143D04220AA800F0E8
:10670400A9FBD0B920220021684618F044FD0123DA
:106714008DF8003007238DF803308DF808300AAB6C
:1067240003930C4B04930C4B08930C49684608F0F4
:10673400CFFB38B90FB05DF804FB094AD52113F03B
:1067440041F9DFE7064ADE2113F03CF9F2E700BF26
:1067540094F20300E166020031680200283400204C
:10676400E0F3030000B585B0284A042146F2010095
:1067740006F078F8264B1B6813F4804F03D0254BA2
:106784001B68032B20DC12F007FE48BB00F0E0FA84
:10679400214800F0FDFA48BB12F030F860BB04A9B0
:1067A400002341F8043D012012F016F938BB03A878
:1067B40012F064F930BBFFF705FEFFF751FEFFF757
:1067C40095FF05B05DF804FB144BD3F80435144A67
:1067D40000924FF487721349042006F05FF8D2E761
:1067E400114A4FF4887113F0EDF8CFE70E4A4FF4D5
:1067F4008A7113F0E7F8CFE713F0D6F8CFE713F078
:10680400D3F8D4E713F0D0F8D5E700BF3DC80200B1
:1068140038330020343300202566020000B00040E5
:10682400DCF2030020F40300E0F3030000B583B0BE
:106834001C4B1B6813F4804F03D01B4B1B68032BAA
:106844001BDC1A481A4B43601A4B8360002118F072
:10685400B9FAE8B9154B18880BF014FBE8B9002114
:106864004FF4F01000F039FA0222C8214FF4F0106E
:1068740000F03EFA03B05DF804FB0F4BD3F8043587
:106884000E4A0092C7220E49042006F007F8D8E702
:106894000C4ACA2113F096F8DCE70A4ACB2113F01C
:1068A40091F8DCE738330020343300202C34002006
:1068B4006D6502007965020000B000402CF303000E
:1068C40020F40300E0F3030030B583B0FFF74AFF80
:1068D400EFF3108572B6354B9B689BB9334A01239D
:1068E4009360334BD3F88010324801401160C3F8F1
:1068F4008000D3F8841051604FF0FF32C3F8842035
:10690400002400E0012405B962B6FFF7E5FC274B3B
:106914009B686BB164B9EFF3108372B6234A1068B5
:1069240023490860506848600021916003B962B649
:10693400002401E000BF2C46FFF7C2FC09F096FEDC
:106944000546C0B1002CF5D11B4B1B6813F4804FD6
:10695400F0D01A4B1B68032BECDD194BD3F804352C
:1069640001220192174A009240F24912164904206A
:1069740005F094FFDEE744B10F4B1B6813F4804F1E
:1069840003D00E4B1B68032B01DC00BFD3E70C4B79
:10699400D3F80435002201920A4A00924FF4A972F6
:1069A4000949042005F07AFFEFE700BF34690020AD
:1069B40000E100E0FC06FFBD383300203433002042
:1069C40000B0004014F3030020F403002A4B1B78AA
:1069D400002B4FD000B585B0012804D0032842D045
:1069E40005B05DF804FB04A9002341F8083D01202B
:1069F40011F0F2FF40BB02A812F040F838BB04A922
:106A0400012341F8043D0DF106000DF0BBFF08BB66
:106A1400BDF806000DF054FC0DF105010DF0A2FDCA
:106A2400D8B909F0DFFC9DF80510002009F09CFDA1
:106A340003F004FDA0B9104B00221A700F4B1B6821
:106A4400002BCDD09847CBE712F0AEFFD3E712F07E
:106A5400ABFFD4E712F0A8FFDAE712F0A5FFE0E7F6
:106A640012F0A2FFE7E711F0C9FE0028B8D012F037
:106A74009BFFB5E7704700BF393400203C34002049
:106A840008B5084B01221A7003F0FAFC18B911F08A
:106A9400FBFE18B908BD12F087FFF8E712F084FF77
:106AA400F8E700BF3934002008B503230022034966
:106AB4004968034813F060FD08BD00BF3C34002062
:106AC4008036002008B50378052B0DD0082B16D08E
:106AD400022B00D008BD104B1B7813B9FFF7E4FF5D
:106AE400F8E7FFF7CDFFF5E710220C4B99680C4847
:106AF40013F0CCFD0028EDD012F056FFEAE78168D0
:106B0400C06808F094F918B9034B01221A70E1E740
:106B140012F04AFFF8E700BF383400203C3400206C
:106B24008036002010B586B00446214A03AB07CA5C
:106B340003C323F8022B120C1A701E4B94E80700AF
:106B440083E80700002A31D01B491C4813F0F8FCE5
:106B5400034610B1184606B010BD194B009303ABA1
:106B6400154A1649174813F0A7FC03460028F1D12B
:106B7400154815F05FF80146124813F0C9FC0346A6
:106B84000028E7D1114813F081F803460028E1D129
:106B94000E4813F0B1F801460A4813F0B9FC034655
:106BA4000028D7D1FFF780FF0346D3E70723D1E7B7
:106BB40050F403003C34002048340020B437002053
:106BC400C96A020080360020683400203036002074
:106BD40008B5064B1B683BB110F098F8002803DB9E
:106BE400024B1B689847F7E708BD00BFF437002045
:106BF40010B50C46144B1860144A0121144812F0C5
:106C0400FBFBA0B9610CE00341F26F7200238B42DD
:106C140008BF824210D24FF47A72002318F047F969
:106C2400014600220B4812F0FDFB38B910BD0A4A98
:106C3400462112F0C7FEE5E70521F2E7064A47219F
:106C440012F0C0FEF2E700BFF4370020D56B02005B
:106C54005CF40300F837002060F4030008B50D4B22
:106C64001B6873B14FF0A042D2F804350A49096891
:106C74004B40C2F80435074A1368013B136023B143
:106C840008BD002012F090FEECE7044812F0E8FB87
:106C9400F6E700BF183800201C38002020380020F8
:106CA4004FF0A043D3F80425012303FA00F0024275
:106CB4000CBF18460020704739B9012303FA00F0CD
:106CC4004FF0A043C3F808057047012303FA00F00E
:106CD4004FF0A043C3F80C05704721B94FF0A0430F
:106CE400C3F8080570474FF0A043C3F80C0570477C
:106CF40012B11346132900D8704770B5114A1060B9
:106D04005B00013B104A136000264D0CCC034FF48A
:106D14007A72002314F5FA7045F1000118F0C7F8EF
:106D240032460146094812F07DFB48B94FF0A042B3
:106D3400D2F804350349096823EA0103C2F804358B
:106D440070BD00BF1C3800201838002020380020F7
:106D540008B511230BE04FF0A04103F5E0720320C6
:106D640041F8220001229A40C1F808250133142B6E
:106D7400F1D9054A0121054812F03EFB00B908BDCE
:106D840012F012FEFBE700BF616C02009CF40300EA
:106D9400F0B1104A1060002309E00F4AD25C02F5FA
:106DA400E0724FF0A0410D4841F822000133032B5B
:106DB400F3D90B4B4FF00042C3F804230020C3F86F
:106DC4007C01084BE02283F8062340221A607047B6
:106DD4000E20704740380020A0F403000C0003008C
:106DE4000060004000E100E010B50024144BC3F83B
:106DF4007C410EE043F23333994208D9114BD3F866
:106E04000425114B1A60114B1B6820469847013426
:106E1400E4B2032C12D84FF0A043D3F810250C4B46
:106E2400195D01238B409343F1D0074B1B68054A3E
:106E3400D2F80425991ADDD5D11ADBE710BD00BFBD
:106E44000060004000B0004044380020403800207A
:106E5400A0F40300082A10D838B51446054618F0E3
:106E640071F9C4F108020021281918F094F9044BAF
:106E740003CBA860E960002038BD0920704700BF3B
:106E84006000001072DF704773DF704774DF704773
:106E94002DE9F047A2B0074688469146314C0026BA
:106EA400C4F80660E68130490B78C3EB43102F4DDC
:106EB400054425602E4A0244A2601F22A280A281BA
:106EC400013303F001030B704FF03C0A5246314684
:106ED40013A818F060F906238DF84F30ADF8487008
:106EE40001238DF84A30ADF85C3012AA1892ADF83F
:106EF4003C70ADF84090CDF844800DEB0A021D9231
:106F04008DF8783052463146684618F044F9022329
:106F14008DF80030221D294613A811F04FFB90B9BB
:106F2400104B03F10C029968684611F047FB68B9ED
:106F3400104A0C491048FFF7A5FF082809D070B97A
:106F440022B0BDE8F08712F02FFDE9E712F02CFD26
:106F5400EEE7002203490848FFF794FFEFE712F039
:106F640023FDEDE78C380020483800204C38002001
:106F74009C380020CC320020C8320020034B00EBA8
:106F8400800042009A819960704700BFCC32002093
:106F940008B50121054B1878FFF776FF10B904F006
:106FA40071FA08BD12F000FDF9E700BFC8320020F5
:106FB40008B5044B1878FFF769FF00B908BD12F053
:106FC400F3FCFBE7C83200200620704700B587B009
:106FD40041F20103984245D020D944F2010398427A
:106FE40056D044F2020398426DD1454B1B6813F40A
:106FF400804F1ED0434B1B68002B1ADD424BD3F845
:107004000435108803905268029201913F4A00921D
:107014005F223F49012005F041FC0AE0012852D1DA
:10702400374B1B6813F4804F03D0364B1B68002B7F
:107034000BDC4FF0A0434FF4F012C3F81825C3F84B
:107044000C25EFF3108372B653E02F4BD3F80435BD
:10705400029201912F4A009254222D49012005F0F9
:107064001DFCE6E7264B1B6813F4804FE1D0254B4B
:107074001B68002BDDDD244BD3F80435029201910B
:10708400254A009257222249012005F007FCD0E747
:107094001B4B1B6813F4804FCBD01A4B1B68002B7F
:1070A400C7DD194BD3F80435106804905068039079
:1070B400029192680192194A0092692214490120AE
:1070C40005F0ECFBB5E70E4B1B6813F4804FB0D012
:1070D4000C4B1B68002BACDD0B4BD3F80435019132
:1070E4000F4A00926D220A49012005F0D7FBA0E760
:1070F40030BF0C4B1B78002BFAD107B05DF804FBB2
:10710400383300203433002000B0004024F503005D
:10711400D1F40300E4F4030000F5030044F5030094
:1071240068F50300E432002000B583B00023ADF815
:107134000030054B01936A46014644F20200FFF712
:1071440045FF03B05DF804FB64F5030010B4034687
:10715400044C006859689A68DB680FC45DF8044BF6
:10716400704700BFDC380020064B074A92E8030052
:1071740083E803000833443292E8030083E8030001
:10718400704700BFDC3800206000001000487047E2
:10719400DC380020002308E0074901EBC30000228B
:1071A4004280426001F8332001331F2BF4D9034B92
:1071B40000221A60704700BFEC380020EC39002030
:1071C40030B405460F4B1B6800240AE01F230E4A07
:1071D40012F83300A0B102EBC3025288AA4207D0CE
:1071E40001341F2C0BD85A1E002BEFD01346EEE7A8
:1071F400054A02EBC30252688A42F1D100E0002042
:1072040030BC7047EC390020EC38002030B40A4A16
:1072140013680A4C04EBC30568806960012104F813
:1072240033100B441360202B01D030BC704713463D
:1072340000221A60F9E700BFEC390020EC38002086
:10724400C0F30C038B4202D3C91A08447047C91A0D
:107254000844A0F500507047C37D002B42D08378CA
:107264000A7802F0800203F07F0313430B70027864
:107274000B7803F07F0343EAC2130B700378002BEF
:1072840041D030B44378082B14BF002201224B783C
:1072940003F07F0343EAC2134B70858803F0800335
:1072A400C5F3861423434B708A7802F0030242EA42
:1072B4008502D2B28A70857902F0FC02C5F3C1045A
:1072C40022438A70CB7803F01F0343EA4513DBB2F1
:1072D400CB70C27903F0E00302F01F021343CB70BA
:1072E40030BC704783780A7802F0BF029B0103F038
:1072F400400313430B70C27803F0C00302F03F0253
:1073040013430B70B3E770470023032B22DC10B444
:1073140002E00133032B19DC0F4C6C2202FB034205
:1073240092F84420012AF4D16C2202FB0342948A8D
:10733400C2899442EDD1084C6C2202FB034292882C
:107344008A42E6D16C2202FB034000E000205DF893
:10735400044B704700207047643A0020002300E08B
:107364000133032B13DC0B496C2202FB031292F84A
:107374004420022AF4D16C2202FB0312918A828AED
:107384009142EDD103486C2202FB030070470020B8
:10739400704700BF643A002008B1082070470420F9
:1073A4007047000038B505460C46CB695B78C3705E
:1073B400CB691B7883F001038370CB694362087B3C
:1073C400022814D0FFF7E8FF6870E27A32B9A18A84
:1073D400C0F10F03994201DC082831D0A18A034689
:1073E400C0F10F00814207DC42B3012205E0154BD6
:1073F400987DFFF7D1FFE7E701222A7062B1A28AE4
:1074040013440B33104A82FB0312DB17C3EB6203F2
:10741400013BEB710023AB710023EB7505F10C020A
:1074240094E8030082E80300A2692A622289AA82FE
:10743400A27AAA75226AAA62184638BD0022DCE73D
:107444000720FAE74C3A0020ABAAAA2A30B4034634
:107454000C460978817000214162A1680B2903D888
:10746400217BF1B1012100E0012119700020587045
:1074740029B1A1680731C9080139D971987101216D
:10748400D97503F10C0504F1100103C985E8030063
:10749400E1899982A1691962217F99759A6230BC48
:1074A40070470021E1E700000021164B1B688B4266
:1074B40026D90023144A02EBC10252689A421DD90C
:1074C40010B4114A52F8312002EBC30412F83320ED
:1074D40082420DD001330C4A02EBC10252689A4237
:1074E400EFD80131074B1B688B4205D90023F2E723
:1074F40060685DF8044B70470020FAE70131D4E777
:1075040000207047F0390020F439002070B58CB0A9
:1075140006460D4614462C22002101A817F03BFE16
:107524000E238DF80430ADF808604FF0000365F3C6
:1075340000038DF80A308DF80B4001A801F0B0F972
:107544000CB070BD30B58DB005460C462C22002120
:1075540001A817F020FE0F238DF8043002958DF852
:107564000C4001A801F09CF90DB030BD00B58DB000
:1075740048B913F1020F06D001228DF804200293BA
:1075840001A801F08DF9034B186804F071F80DB0EF
:107594005DF804FB003A00202DE9F04105468846D9
:1075A4000378BBB10D4B1C68621C1A6004F007041D
:1075B400AB8A0B4F07EBC4067380A988A869FFF751
:1075C4003FFE7060EB6903F00103737007F83480C9
:1075D400BDE8F0817846FFF7A7FDE3E7483A0020CD
:1075E400083A002070B5064603784BB1B58A347F5B
:1075F40004F00104B188B069FFF722FE002304E01F
:107604007846FFF791FDF1E70133072B15D80C4AB3
:1076140002EBC30252688242F6D1094A02EBC3026A
:107624005288AA42F0D1064A02EBC3025278A2421F
:10763400EAD1034800EBC30000E0002070BD00BFA6
:10764400083A0020F0B40D684C688F68CE68D560A5
:107654001461576196610D694C69D56114620378B0
:10766400DB091370D17DF9B1037803F07F039370C4
:107674000023537013789BB143789B0103F4FE53AA
:10768400817843EA910393808378DB0003F0180345
:10769400C17843EA51139371C37803F01F03D37184
:1076A40000235362F0BC70470178C1F380119170DC
:1076B400017801F03F01D17043B190F90130002B02
:1076C40002DB04235370D5E70823FBE7042353703C
:1076D400D0E770B50C461E4603788BB104252A44C6
:1076E400A26000F10C032360836A6360204604F007
:1076F40065FB024610B923691D443560104670BD10
:107704000125ECE72DE9F0418EB00D4616461C46E6
:10771400804600282DD0002D2FD0002C31D0636A54
:107724000233059304F10C00A378002B2DD0012122
:10773400627801AF3B46082A14BF0022012204F0FC
:1077440094F80697CDF81C80B2B2ADF820200B95C2
:1077540015440C9563788DF83430237B022B16D0B6
:107764000023ADF8283005A804F077F80EB0BDE882
:10777400F0817846FFF7D8FCCDE77846FFF7D4FCD4
:10778400CBE77846FFF7D0FCC9E70221D0E72369AD
:107794002BB1236909931023ADF82830E3E7784629
:1077A400FFF7C2FCF5E72DE9F04186B004460D462B
:1077B400C37D002B3ED0082605FB06F8E379AB42D7
:1077C4003AD0A5716B46324601A92046FFF781FFE6
:1077D400074648BB4DB994F84F3033B9A369C3F396
:1077E4000C03A380012384F84F30E37D7BB994F824
:1077F4004E3063B92DBBB4F84610627823468A1A1A
:10780400A16E0846FFF77EFF012384F84E300599E8
:107814002046FFF721FDA16E32464144009817F03F
:1078240091FC01A804F0E4FAB7FA87F0400906B025
:10783400BDE8F0810C26BFE7B4F84660A6EB080665
:10784400BFE77846FFF770FCD5E770B5054690F8BA
:107854004C40002605E00136631C85F84C300134A9
:10786400E4B2EB79A3420AD3AA6C0123A3401A42DF
:10787400F5D121462846FFF796FF0028EBD1304684
:1078840070BDF0B587B045781544C37DDBB10B23DB
:107894009D4221D816460F4604466B462A4601A946
:1078A400FFF717FF0546C0B905992046FFF7D4FC3A
:1078B400E37D53B132463946009817F043FC01A8E2
:1078C40004F096FA09E00F23E2E7234632460099D2
:1078D4003846FFF717FFF2E70925284607B0F0BD41
:1078E40010B5044690F84430012B0ED1237B012BB4
:1078F4000FD00C4BDB68A36303F0B6F9A16B014412
:1079040004F12C0003F014F910BD7846FFF70CFCC9
:10791400ECE7A37D034AD168126902FB0313A36356
:10792400EAE700BF4C3A002038B5002400E00134F7
:10793400032C13D80A4A6C2303FB042393F8443022
:10794400012BF4D16C2505FB04252846FFF77DFFA8
:107954000028ECD02846FFF7C3FFE8E738BD00BF96
:10796400643A002038B5044690F84430022B02D023
:107974007846FFF7D9FB054B1D6803F075F94119EB
:1079840004F12C0003F0D4F838BD00BF4C3A0020B9
:1079940038B5044690F84430022B02D07846FFF7FD
:1079A400C3FB084B5D7D5A689B6803FB052503F008
:1079B4005BF9411904F14C0003F0BAF8012384F88F
:1079C400643038BD4C3A002010B504460C4B1B689B
:1079D400806E98470023A36604F12C0003F078F826
:1079E40094F84430022B05D0002084F8440002F0BF
:1079F4000BF910BD04F14C0003F06AF8F4E700BF82
:107A0400043A002010B504460121FFF7C5FD2046C5
:107A1400FFF7DAFF10BD10B58CB0044690F844307F
:107A2400012B02D07846FFF77FFB01238DF8043049
:107A3400236D029301A800F033FF2046FFF7C4FF33
:107A44000CB010BD2DE9F04104460E4615461F4604
:107A5400531EDBB2012B46D8A36E13B17846FFF751
:107A640063FB2E4B1B6838469847A066002852D00B
:107A74003346224606F12001D3F80080D3F804E00F
:107A8400D3F808C0D868C2F80080C2F804E0C2F88D
:107A940008C0D060103310328B42EDD11868596899
:107AA4009B681060516093600023A364A4F846703F
:107AB400B188B069FFF7C4FBA061012D17D06FF046
:107AC4000103A362002384F86430154B6365E46505
:107AD400144B6363E463012002F096F884F8445085
:107AE4000120BDE8F0817846FFF71EFBB4E70E4B9A
:107AF4001B7D84F84D30002384F84E3084F84F30D9
:107B040084F84C30B36A23656FF00103A362074B1A
:107B14006363E463DFE70020E3E700BFFC39002090
:107B240073860200597C02004C3A0020657C0200F6
:107B340030B583B0C3790133C27D92B1082505FB0A
:107B440003F582B14FF48073AB422AD21E4B1B68FB
:107B540013F0040F36D01D4B1B68002B06DC0024E9
:107B64002DE00C25EBE74FF4C073EDE7184BD3F889
:107B740004350195174A00924FF4177216490120F3
:107B840004F08CFE00241AE0144C6C2303FB024422
:107B94002B46022201462046FFF754FF78B9002401
:107BA4000DE00022032A09DC0C4B6C2404FB023494
:107BB40094F84430002BE7D00132F3E70024204648
:107BC40003B030BD0024FAE73833002034330020FA
:107BD40000B00040DCF50300CFF50300643A002058
:107BE40030B585B00D460446A8B100212046FFF704
:107BF400D3FC2946206DFFF7A5FC2046FFF7E4FEE1
:107C04000F4B1B6813F0040F03D00E4B1B68032BA0
:107C140005DC05B030BD7846FFF786FAE5E70A4B88
:107C2400D3F8043594F8442002950192074A00924F
:107C34004FF4D2720649042004F030FEE9E700BF95
:107C4400383300203433002000B0004084F50300B2
:107C5400CFF5030008B508460021FFF7C1FF08BDB2
:107C640010B50C4691F84430012B09D194F84D30ED
:107C74007BB9237B012B07D02046FFF7CCFE10BD38
:107C84007846FFF751FAF1E700212046FFF7A8FFF5
:107C9400F5E7013B84F84D30002384F84C3020464E
:107CA400FFF7D3FDEBE70000062900D0704770B55D
:107CB40082B003460178890101F4FE5140789D7831
:107CC400DC78240444EA05641D7944EA05245B79DC
:107CD4001C4341EA90011046FFF716FB0546B8B174
:107CE400866C2643866444B3037853B3EB795A1CF9
:107CF40001239340013B9E4227D0002385F84C305A
:107D04002846FFF7A2FD2846FFF7EAFD02B070BD42
:107D1400104B1B6813F0040FF8D00F4B1B68012B9A
:107D2400F4DD0E4BD3F804350D4A009240F2B24212
:107D34000C49022004F0B2FDE8E70321FFF750FFED
:107D4400E4E77846FFF7F0F9D0E72846FFF763FE4B
:107D5400DCE700BF383300203433002000B000409B
:107D6400F0F50300CFF503002DE9F04389B0804618
:107D74000F4614461E4695780DB32846FFF794FB2C
:107D84008146C8B18DF80050236A0693A38AADF8E2
:107D94000E3004AB04F10C0292E8030083E8030004
:107DA400A37D8DF81C30CDF80480029723788DF8DC
:107DB4000C3031466846C84709B0BDE8F083FFF788
:107DC40073FFF9E700B585B000238DF80F3098B143
:107DD4000346084602330B600DF10F0103F041FD29
:107DE4009DF80F3043B10D4B1B6813F0040F03D003
:107DF4000B4B1B68032B04DC9DF80F0005B05DF8EA
:107E040004FB084BD3F80435074A00924FF4397247
:107E14000649042004F042FDEEE700BF3833002099
:107E24003433002000B0004030F60300CFF50300E7
:107E34002DE9F0438FB004460E4615461F46D0F890
:107E44001890037823B181884846FFF7F9F9A061B7
:107E540004F10C00A378002B3AD0012162780DF1D3
:107E640028084346082A14BF0022012203F0FDFC1F
:107E7400C4F81890CDF8088003966378EA1A92B291
:107E8400ADF810203244089207978DF8243000236F
:107E9400ADF81830237B022B1CD0A3786BB3237B63
:107EA400022B1BD02546002345F8243F2A46E178BF
:107EB400206A0DF0A7F8606A98B101A9FFF782FF64
:107EC40000283AD12A46E178206A0DF09BF8F2E7BF
:107ED4000221C3E71023ADF81830DEE723690593C8
:107EE400E0E7237B022B2CD104F10C01E0890DF097
:107EF40037F90028D3D1052020E000236362237BD7
:107F0400012B0DD02146002341F8243FA08A0DF017
:107F140096F801A9606AFFF755FFA0B100200DE0B3
:107F240004F12401E0890DF08AF801A9606AFFF7E1
:107F340049FF0028E6D0002000E000200FB0BDE893
:107F4400F0830520FAE70520F8E7000070B5F0B0EB
:107F54000D4614461E4610AB0A4601462046FFF75E
:107F640067FFA0B11F4B1B6813F0040F37D01E4BE3
:107F74001B68052B33DD1D4BD3F804351C4A0092D6
:107F840040F221521B49062004F088FC27E003AB91
:107F940001228DF80C20A28AADF80E200022049252
:107FA4008DF8142010AA06926278AD1AADF81C5010
:107FB40008AA93E8030082E803000AAB04F10C0268
:107FC40092E8030083E80300A37D8DF83830236A28
:107FD4000C93636A0D930F9605A800F061FC70B0D2
:107FE40070BD00BF383300203433002000B000409F
:107FF40054F60300CFF5030010B5D47D14B9FFF790
:10800400A5FF10BDFFF7B0FEFBE700002DE9F0432C
:1080140085B004AF43781344C47D94B14FF48074A5
:108024009C4273D3EFF3108C72B60024032C10DC43
:108034003B4E6C2505FB046595F8445025B101348D
:10804400F4E74FF4C074EBE735466C2606FB0454A2
:1080540000E00024BCF1000F00D162B6002C5AD01D
:1080640015460E46014601222046FFF7EBFC002888
:1080740053D02A463146A06E17F064F8294B1B688A
:1080840013F0040F3AD0284B1B68032B36DD6D46E2
:10809400B4F846E04FEA4E030833DB08A5EBC3030C
:1080A4009D460DF11008C446002312E0A26ED25C76
:1080B4004FEA121959001D48066816F809600CF8B1
:1080C400136002F00F0201310068825C0CF8012099
:1080D40001337345EAD3002308F81E30144BD3F858
:1080E4000435CDF80880134A0192134A00924FF4E4
:1080F4007C721249042004F0D1FBAD462046FFF700
:10810400A4FB2046FFF7ECFB002000E00920043725
:10811400BD46BDE8F0830420F9E70420F7E700BF7B
:10812400643A002038330020343300203C330020EC
:1081340000B0004020F6030038F40300CFF503003C
:1081440070B504460D461646808A02F023F80128CD
:108154001AD1237BD3B1022B0BD094F91630002B08
:1081640016DB237853B9324629462046FFF789FBAC
:108174000BE02369002BF0D1102006E0324629469B
:108184002046FFF743FF00E0102070BD1020FCE7FD
:108194000720FAE708B50549054800F04FF800B98B
:1081A40008BD7846FEF7C0FFFAE700BF15F00300EC
:1081B40081EF030010B5FFF7EDFF4FF4D8720021F3
:1081C400134816F0E8FF05F0F9FC0024114B1C607D
:1081D40040222146104816F0DEFF104B104A1A6068
:1081E400104A5A604CF250329A600F49D9601A61B1
:1081F40004221A759C7508225A750C4803F018FA63
:108204000B4B18600B4B1C600B4805F0DDFD10BDDB
:10821400643A0020483A0020083A00204C3A0020F2
:1082240080969800F049020020A1070029840200EA
:10823400003A0020F03900207175020008B50346A9
:10824400B0FA80F040090A46B1FA81F1490988423E
:1082540010D14BB1EFF3108072B608490B60084B94
:108264001A6048B962B606E0002AF3D1FFF792FF1C
:10827400002000E00E2008BD0020FCE7FC390020AF
:10828400043A0020C0B110B58CB004460369B3B100
:10829400C369B3B18369B3B1014601A8FFF782F89A
:1082A400034610B118460CB010BDA28A216901A87A
:1082B400FFF746FF0346F5E70E23184670470E23E3
:1082C400F0E70E23EEE70E23ECE7D0B110B58CB047
:1082D40004464068B8B1A269BAB1207C022816D01D
:1082E400B8B194F90020002A15DB0A46214601A8FA
:1082F400FFF7ACF8A268616801A8FFF721FF0CB092
:1083040010BD0E2070470E20F9E70E20F7E710206D
:10831400F5E71020F3E70720F1E70000037B012BCA
:1083240001D00020704710B58AB000228388C3F3BF
:1083340086148DF800409B008DF801300B0E8DF8EB
:1083440002300B0C8DF803300B0A8DF804308DF8D5
:1083540005100623049301238DF81830838AADF8A1
:108364001A3007928DF80820CDF80CD0036A0893D0
:108374008DF81420C389ADF81630837D43B98DF888
:1083840024206FF0010102A8FFF79FFF0AB010BD7F
:10839400024B5B7D8DF82430F3E700BF4C3A00209C
:1083A40038B500240BE01E4A6C2303FB0423DB795D
:1083B4005A1C01239340013B9D4228D00134032CD5
:1083C4002CD8174A6C2303FB042393F84430022B64
:1083D400F4D16C2303FB042393F86430022BEDD116
:1083E4006C2000FB0420816CFFF798FF0028E5D186
:1083F4000B4A6C2303FB04F3D11881F864008D6CE1
:10840400D35C002BCFD17846FEF78EFECBE7044B2E
:108414006C2000FB0430FFF7F5FACFE738BD00BF4E
:10842400643A002008B5FFF77FFAFFF7B9FF01208F
:1084340008BD00002DE9F04182B007460E461446FF
:1084440098461046FEF78AFF054620B1A288838825
:108454009A4210D312D82046FFF7C4F8B8B1037873
:108464004BB123787BB1E1794B1C0121994001394F
:108474002046FFF753FF02B0BDE8F0810521FFF766
:10848400AFFB0025E7E77846FEF74EFEEBE7002D4D
:108494004FD0464B1B6813F0040F03D0444B1B68AA
:1084A400032B55DC2846FFF75DFA2B7B012B5DD0AF
:1084B400AA6CA17901238B401A42DCD11343AB642B
:1084C400A279EB799A4259D0E37D002B61D008233D
:1084D400B34260D1AB6EA079E27D002A60D008245B
:1084E4003246394604FB003016F02CFEAC6C2B7877
:1084F400002B57D0EB795A1C01239340013B9C423B
:10850400B9D1022385F86430A96C2846FFF706FF29
:10851400044643462A46B5F84610A86EFFF76CFD9C
:10852400002CA8D1002385F864302846FFF76AFAA6
:10853400A1E72046FFF7FCFA05460028A9D100214F
:108544002046FFF7EBFE02210020FEF7FBFF92E737
:10855400184BD3F80435A2790192174A00924FF4CC
:1085640028721649042004F099F99BE795F86430C1
:10857400002B9DD12846FFF70BFA99E79BB2E27DC9
:108584002AB1082203FB0263A5F84630A2E70C22B5
:10859400F8E70C239CE704212846FFF721FB6AE750
:1085A4000C249DE77846FEF7BFFDA3E7383300208F
:1085B4003433002000B0004044F60300CFF503003C
:1085C4002DE9F0418EB000284DD00546002A4CD04C
:1085D400984614460F4600220C920D920CA960880E
:1085E4000CF0BEFD20B9002630460EB0BDE8F08187
:1085F400226902F00102E168208905F0ADFA08B1B0
:108604000026F1E7226902F00102E168208905F001
:1086140073FA0646C0B901AA21462846FFF712F8A4
:1086240004AB0EAA12E9030083E8030002F0BEFFC4
:108634009DF8043083B1434601AA391F281DFFF772
:10864400F9FE02F0D3FFCFE72169002201F0010116
:108654002089FEF75BFFC7E7434601AA791E681C21
:10866400FFF7CAFCEDE70E26BEE70E26BCE710B501
:108674000C4691F84430022B0BD1022384F8643069
:10868400A16C2046FFF74AFE10B9002384F8643039
:1086940010BD7846FEF748FDEFE70000002959D0E9
:1086A400A0F59670072857D8DFE800F0040E1A25C5
:1086B400313D454D4A68314B134431498B424DD8C5
:1086C400304B1A60002070474A68A2F51233A3F5B4
:1086D400F8732D498B4243D82A4B5A6000207047C7
:1086E4004A68A2F54343503B28498B423AD8254B6C
:1086F4009A60002070474A68A2F54333A3F5A0733B
:1087040023498B4230D81F4BDA60002070474A68F7
:10871400A2F54333A3F5A0731D498B4226D8194B08
:108724001A61002070474B689A1EFD2A20D8154A0A
:108734001375002070474B685A1E7E2A1AD8114AB6
:108744005375002070474B68012B15D80D4A93755B
:10875400002070470E20704705207047072070479F
:10876400072070470720704707207047072070478D
:10877400072070470720704707207047806967FF0C
:1087840080778E064C3A0020904C960030D39700A8
:1087940040899500002934D000220A604A60A0F57F
:1087A400967007282FD8DFE800F004090E13181D6F
:1087B4002227164A12684A6000207047134A5268FA
:1087C4004A6000207047114A92684A60002070474E
:1087D4000E4AD2684A60002070470C4A12694A6007
:1087E40000207047094A127D4A6000207047074AFA
:1087F400527D4A6000207047044A927D4A600020FE
:1088040070470E2070470520704700BF4C3A002087
:10881400F8B500B30546164B1F68F7B90E463C463B
:10882400B4420ED205EBC4035B68CBB115F8340037
:1088340010F0800F16D1B8B1FEF736FEB0B901348E
:10884400EEE70C4B43F8375003EBC7035E607B1C29
:10885400074A136002E00E2700E004273846F8BDFB
:108864000E27FBE70B27F9E70F27F7E70F27F5E7B5
:10887400F0390020F4390020084B196861B110B5B3
:1088840001E021463CB10C680B79002BF9D0034878
:1088940003F06DFFF5E710BD704700BF183C0020E2
:1088A40038B5054630B1104B1C68ACB10F4B0122F2
:1088B4001A7004E07846FEF737FCF4E724683CB10C
:1088C4002379002BFAD154F8043C28469847F5E75D
:1088D400064B1B78022B00D038BDFFF7CDFF034BAE
:1088E40000221A70F8E700BF183C0020143C002056
:1088F40010B5044630B100232372211D034803F050
:108904000BFF10BD7846FEF70FFCF4E7183C00207F
:1089140010B5044650B10A4B1B78013BDBB2012B66
:1089240008D9211D074803F022FF10BD7846FEF741
:10893400FBFBF0E7024B02221A7001232372F4E7D7
:10894400143C0020183C00200A8883689B5A073393
:108954009BB223F0030313449BB20288043A93426C
:1089640000D900230B80704710B582B00446836899
:10897400CB1A02A921F8023DFFF7E6FFBDF8063045
:10898400A068184402B010BD0088043880B2704753
:1089940043888268D018D15201238370704782685B
:1089A40000239370438083807047073189B221F09C
:1089B400030189B2428883889A4204D29B1A99425D
:1089C4001CDC0020704710B59A420FD90488A41A01
:1089D400A14215D98B4215D3032C03D983681344C0
:1089E40004229A7000234380184606E082681344E8
:1089F4009B784BB9FFF7D3FF002010BD04207047CC
:108A04000020FAE70420F8E70420F6E738B5044626
:108A14000D468368828813448B4202D07846FEF761
:108A240083FB0023AB70211D2046FFF78DFFA28836
:108A3400A36813449B78042B00D038BD0023A38083
:108A4400FBE710B50C468368428813448B4202D07E
:108A54007846FEF769FB0023A37010BD70B5064687
:108A640015460C46002944D0002E46D0B4F1005FD0
:108A740008D94FF08053D3F80C3103F50023B4EB3D
:108A8400832F0ED3B4F5000F08D94FF08053D3F8D9
:108A94000C3103F50053B4EB832F02D37846FEF771
:108AA40043FB6B1E2344B3F1005F08D94FF080529F
:108AB400D2F80C2102F50022B3EB822F0ED3B3F5CA
:108AC400000F08D94FF08052D2F80C2102F5005261
:108AD400B3EB822F02D37846FEF726FB042D10D980
:108AE400358000237380B380B460043D2580A37077
:108AF40070BD7846FEF718FBB6E77846FEF714FB20
:108B0400B4E77846FEF710FBEAE738B50446A0B1AF
:108B14006288A36813449B78012B12D0A388A168B0
:108B24001944EFF3108572B68B78032B0DD02046D1
:108B3400FFF735FF05B962B638BD7846FEF7F4FA9B
:108B4400E6E77846FEF7F0FAE8E72046FFF70CFF81
:108B5400A368C31A638000238370EBE7F8B50E465D
:108B640015460446C0B1DEB16288A36813449B78FD
:108B7400012B19D0E5B12046FFF706FFA84219D30F
:108B840029462046FFF711FF0746A0B9294620468B
:108B9400FFF7FEFE30600EE07846FEF7C5FAE2E726
:108BA4007846FEF7C1FADFE77846FEF7BDFAE1E75B
:108BB400092700E009273846F8BD70B50C4616466B
:108BC4000546B8B1D4B1A378012B1BD12388B34295
:108BD4001CD3FEB126800223A370E9182846FFF7B0
:108BE400B3FE6A88AB889A4203D0AB681344002270
:108BF4009A7070BD7846FEF797FAE3E77846FEF779
:108C040093FAE0E77846FEF78FFADFE77846FEF757
:108C14008BFADEE77846FEF787FADBE738B50D46D0
:108C2400044650B16DB1A288A36813449A78022A0D
:108C34000BD0032A0ED005200BE07846FEF774FA19
:108C4400F0E77846FEF770FAEDE703229A702B609E
:108C5400002038BD7846FEF767FA0020F9E710B522
:108C6400044640B1A288A36813449878022814BF2C
:108C74000020012010BD7846FEF756FAF2E710B541
:108C8400044618B1A088A168014407E07846FEF7BD
:108C94004BFAF7E72046FFF767FE0146887803287A
:108CA400F8D0022814BF0020012010BD38B50C46AE
:108CB400054650B16CB1A378012B0ED0032B11D112
:108CC40021462846FFF7A2FE38BD7846FEF72CFA67
:108CD400F0E77846FEF728FAEDE721462846FFF745
:108CE400B0FEF1E77846FEF71FFAEDE708B5064B4C
:108CF400986800221A605A609A60DA601A615A61B0
:108D04009A6104F04FFD08BD1C3C002000B585B0FD
:108D14000A4BDB6802228DF8002001934FF4805344
:108D24000293074A6946012001F098F918B100201E
:108D340005B05DF804FB0120FAE700BF1C3C0020ED
:108D4400383C002000B585B00A4B1B6802228DF820
:108D5400002001934FF480530293074A694601208F
:108D640001F07CF918B1002005B05DF804FB012086
:108D7400FAE700BF3C3C0020383C0020164BDA6880
:108D8400137951795B1A03F57F2303F6FF7302EB22
:108D940003339A4205D002F580520F4BDA60032068
:108DA400704700B585B00D4B1B6801208DF800009D
:108DB40001930B4B0393042302930A4A694601F07F
:108DC4004DF918B1002005B05DF804FB024B0122F7
:108DD4001A760220F7E700BF1C3C00203C3C002030
:108DE400403C0020383C002000B585B00C4BDA68CC
:108DF4000C4B1B68043301208DF80000019203938F
:108E040040F6FC730293084A694601F027F928B931
:108E14000120034B187605B05DF804FB0020FAE747
:108E24001C3C00203C3C0020383C002000B585B0B0
:108E34000A4B1B6801208DF800000193084B039333
:108E440004230293074A694601F008F918B1002087
:108E540005B05DF804FB0120FAE700BF3C3C0020AC
:108E6400283C0020383C002010B584B0114BDA684F
:108E74001478114B1B68043301208DF80000019312
:108E8400039202940D4A694601F0E8F880B90A4B4E
:108E94001B6804F0FC041C440434064B5C61D96870
:108EA4000A780A441A6100225A76012004B010BDDF
:108EB4000020FBE71C3C00203C3C0020383C002008
:108EC40008B50023092B09D8064A52F82320824208
:108ED40001D00133F6E7044A536002E07846FEF716
:108EE40023F908BD80F603001C3C002010B5214B7B
:108EF400DB6853B11F4B1B7E5BB91E4B5B68092BB0
:108F040015D97846FEF710F911E07846FEF70CF90A
:108F1400F0E77846FEF708F9EFE7164B00225A60AF
:108F2400012C01D0032C23D1124B1B7E03BB114B0C
:108F34005A68114B53F822309847044602280DD042
:108F44000328EAD00128EBD10A4A5368013353605D
:108F5400092BE5D97846FEF7E7F8E1E7054B1B7ED8
:108F64001BB1044B02221A70DAE7FFF7BFFED7E702
:108F740010BD00BF1C3C002080F60300104B1B6892
:108F84001B685A1E12F1030F18D8C3F30B020AB15F
:108F94000020704710B50B4AD36000231376537634
:108FA4000124147093600848FFF78AFF074920469C
:108FB40001F042F8FFF79AFF204610BD00207047E9
:108FC4003C3C00201C3C0020118D0200D58F020087
:108FD40008B50B78032B06D00B4B1B78012B06D05E
:108FE400022B0BD008BD084B00221A76F4E7064B7F
:108FF4001B7E002BF6D1FFF779FFF3E70B78032BE9
:10900400F0D1FFF773FEEDE71C3C002000B585B0FE
:10901400174BDB6818784FF6FF7203F5805118443C
:1090240004F088FEF0B10246114BD9680B780B446A
:10903400984219D00E4B5B7E93B10E4B01208DF8F4
:10904400000001920393042302930B4A694601F042
:1090540005F858B90120064B187605B05DF804FBF5
:10906400064BEBE70120F8E70120F6E70020F4E7E0
:109074001C3C002060F80300383C00205CF803002E
:1090840008B5104BDB681878002203F580511844AA
:1090940004F050FE08B1012008BD0A4BDA681379C8
:1090A40051795B1A03F57F2303F6FF7302EB033355
:1090B4009A4205D002F58052024BDA600320EBE7B6
:1090C4000220E9E71C3C0020F0B585B0524BDE6875
:1090D40072793379591E8A4200F0968006F58051E0
:1090E4000D780D444D490968081D0F7907449B1AF2
:1090F40003F57F2303F6FF731B0303F580531E441C
:109104006B88013B9BB247F6FE6293425CD92C46C6
:1091140016E07846FEF708F815E024F47F6424F09E
:109124000F0404F5805423781C44A64247D9A54271
:1091340047D26388013B9BB247F6FE62934211D942
:109144002388002BE5D0238804EB830323F47F6278
:1091540022F00F029342E0D06288B2F5FE4FDCD0D9
:109164001C46E2E725462FE07846FDF7DDFF15E0D3
:1091740024F47F6424F00F0404F5805423781C4401
:10918400A64220D9A5423BD26388013B9BB247F655
:10919400FE62934211D92388002BE5D0238804EB87
:1091A400830323F47F6222F00F029342E0D06288AB
:1091B400B2F5FE4FDCD01C46E2E7254604E000256C
:1091C40002E0002500E00025E5B1144B19686A8827
:1091D40001F58051384604F0ADFD0746B8B10120D1
:1091E4000D4B18768DF8000001950D4B0393042365
:1091F40002930C4A694600F031FF50B92C46CAE785
:109204000025E1E7012000E0012005B0F0BD0120C8
:10921400FBE70020F9E700BF1C3C00203C3C002099
:1092240058F80300383C00202DE9F04186B06A4B21
:109234001B692BB1684B5B6933B14FF0000848E000
:109244007846FDF771FFF5E77846FDF76DFFF4E723
:109254007846FDF769FF15E025F47F6525F00F05D5
:1092640005F580552B781D44AE421CD9AC421ED264
:109274006B88013B9BB247F6FE62934211D92B885F
:10928400002BE5D02B8805EB830323F47F6222F0C7
:109294000F029342E0D06A88B2F5FE4FDCD01D463F
:1092A400E2E72C4600E000241CB1009445E00024D1
:1092B400FAE700230093019B002B68D14FF00108CB
:1092C40024B1628847F6FF739A4202D1424B0122CD
:1092D4005A76414B5B7E002B7AD1B8F1000F75D1E1
:1092E4003D4B5A6922F47F6727F00F07BF1A07F531
:1092F40080571C69DE68337972799B1A03F57F23E2
:1093040003F6FF731B0303F580531E4400230193EC
:109314006388013B9BB247F6FE629342C5D925465A
:10932400ADE77846FDF700FF22E024F47F6424F0E3
:109334000F0404F5805423781C44A642BBD9238827
:10934400019A02EB83029742B5D9009B634023F450
:109354007F6323F00F03002BADD16388013B9BB2E5
:1093640047F6FE618B42A6D801922388002BD8D001
:10937400238804EB830323F47F6222F00F029342D9
:10938400D3D06288B2F5FE4FCFD01C46D5E7124A3F
:10939400526901208DF808000392009A0592049303
:1093A4000E4A02A900F05AFE70B90B49019B23F042
:1093B40003024B6913444B6114B1074B1C617FE7F3
:1093C4007846FDF7B1FEF8E7002002E0012000E056
:1093D400012006B0BDE8F0811C3C0020383C002090
:1093E40008B54FF010235B69B3F1FF3F03D04FF092
:1093F40010235B6963B94FF080525169136903FB11
:1094040001F3A3F58053054A1360FFF7B7FD08BDC8
:109414004FF010235B69A3F58053F2E73C3C002036
:10942400024B1878003018BF012070471C3C002004
:1094340010B504460E4B1B78ABB92378032B02D02E
:109444007846FDF771FE0A4B9C60E268DA60002200
:109454005A601A76012018705A76064900F0ECFD1D
:10946400FFF744FD10BD7846FDF75EFEE5E700BF5B
:109474001C3C0020D58F0200014B1868704700BFC8
:109484003C3C002010B5044680B163681BB12368DE
:109494000BB1A36813B97846FDF746FEA3685A1EBC
:1094A400134207D10023E360236110BD7846FDF722
:1094B4003BFEEAE77846FDF737FEF3E7F8B5F8B187
:1094C4000446F9B18268FAB1EFF3108572B6026905
:1094D40080680244E668B24203D1C5B962B6042585
:1094E40013E027686368013830401A4600FB0370B4
:1094F40015F028FEE3680133E36055B962B604E071
:109504000E2502E00E2500E009252846F8BD0425B5
:10951400FBE70025F9E770B5F0B104468268EAB1CB
:10952400EFF3108572B60669C268964210D00846F9
:1095340021686268A368013B1E4006FB021108B162
:1095440015F000FE23690133236165B962B606E0B4
:109554003DB962B6052502E00E2500E0092528463E
:1095640070BD0525FBE70025F9E70000C0F30B03F8
:1095740033BB39B301F6FF71090B134B0222C3F855
:109584000425114BD3F80034002BFAD000220AE052
:109594000D4BC3F808050C4BD3F80034002BFAD05C
:1095A40000F5805001328A42F2D3074B0022C3F8FF
:1095B4000425054BD3F80034002BFAD00020704763
:1095C400102070470920704700E0014010F0030F9D
:1095D4002FD111F0030F2FD182B312F0030F2FD12B
:1095E40010B49208174B0124C3F80445154BD3F863
:1095F4000034002BFAD002E0043004312246541E19
:1096040052B10B68B3F1FF3FF6D003600D4BD3F8B2
:109614000034002BFAD0EFE70A4B0021C3F80415FD
:10962400084BD3F80034002BFAD010465DF8044BF5
:1096340070471022104670471022FBE70922F9E711
:109644000922F7E700E001400180002343804260E3
:109654007047000038B5124C4FF480552A4600215B
:10966400204615F098FD0F4B1C600AE000222821CB
:109674002046FFF7E9FF2388083323446360303D25
:109684001C46502DF2D8083D05D00022A9B2204630
:10969400FFF7DAFF38BD7846FDF746FDF5E700BF72
:1096A400443C0020444C002008B50822022108480C
:1096B40003F0F9FE38B1074A91684160127B0272E7
:1096C40003F02AFF08BD044804F044F8FAE700BF99
:1096D400504C0020984C0020F83200200E4B1B7890
:1096E400CBB910B50D4B5C6804F50054B4F1807F20
:1096F40000D910BD04220121094803F0D4FE30B181
:109704004460054A0121117003F006FFF1E70548A2
:1097140004F020F8EDE77047AC4C0020984C002092
:10972400504C0020E832002010B5044608B1A04790
:1097340010BD7846FDF7F8FCF9E7000008B50121F3
:109744000B4803F011FF20B90221094803F00CFF74
:1097540028B1084803F0FEFFFFF7C0FF08BD064B21
:1097640000221A605A609A60DA601A61F4E700BF56
:10977400504C002018330020984C002000B58DB0C8
:1097840004918DF8082003900CA8022300F82C3DC6
:10979400FFF786F80DB05DF804FB000010B58CB03F
:1097A4000C4682B94B88012B20D1134B1B7833B163
:1097B4006268124B5A60104B00221A7016E0784609
:1097C400FDF7B2FCF4E7032A12D12C22002101A8F0
:1097D40015F0E1FC10238DF804300394084BDA688B
:1097E40005921B69069301A8FFF75AF80CB010BD47
:1097F4007846FDF799FCE8E7AC4C0020984C002033
:10980400504C002038B503F0BDFF28B901F098FF93
:109814000028F8D020BFF6E701F0C8FE0022114668
:109824001A4803F09AFD00252C4605E0051D024662
:109834000021164803F091FD30B14388012BF5D087
:10984400022BF4D1041DF2E7A4B19DB12268104BA0
:109854009A6022791A73AC4201D9237993B12A68A8
:109864000B4B1A600A4B1A685A60FFF737FF01F076
:10987400BDFE38BD064B00221A609A601A73FFF7CA
:1098840013FFEFE7024B00221A60EBE7504C002075
:10989400984C002008B503F0B7FFA0F5805008BD30
:1098A40000B587B0002300930193029303930493BC
:1098B4000593FFF7EFFF009001230193064B0393F9
:1098C4006946064803F000FF10B907B05DF804FBD1
:1098D400034803F03FFFF8E7A1970200504C002033
:1098E4000833002038B50F4B00241C605C609C607A
:1098F400DC601C6101F0B8F90B4D68600B4BAB6088
:109904000B4BEB602C616C610A4B1C700A480B4BCF
:10991400036000F0F9FD284601F0A8F8FFF7C0FF46
:1099240038BD00BF984C0020744C00200D9B0200F1
:1099340000879303AD4C00208C4C0020E19A020078
:1099440038B501F033FE174B1B7B13BB154B9B7BC8
:1099540023BB144B1A8A41F282639A4204D8124BF5
:109964001B78A3B1012300E00123CBB10D4D0123EA
:109974002B7300242C82AB680133AB60FFF794FE99
:10998400A9682A7B01392046FFF7F8FE02E000238C
:10999400EBE7082401F02AFE204638BD0824F9E745
:1099A4000824F7E7984C0020AD4C002010B501F0D6
:1099B400FDFD214B5B7B9BB11F4B9B7BF3B91E4B86
:1099C4001A8A41F282639A4204D81C4B1B782BB149
:1099D400012300E001239BB1012302E00023FAE705
:1099E40000231C461BB3144B00225A731B7B4BB140
:1099F400012B0ED07846FDF797FB18E00023F0E723
:109A04000023EEE7FFF79CFF88B17846FDF78CFB57
:109A14000DE0094B00201860586018731882024644
:109A24009968FFF7ABFEFFF73FFEFFF757FE01F023
:109A3400DDFD204610BD00BF984C0020AD4C002039
:109A440038B5254B1B7B002B36D10446224B5B8A51
:109A540033BB1AB9204B9B688B4205D302B31E4B10
:109A64009B6801338B421BD21B4B9B682A338B426E
:109A740024D3194B9B7B0BBB174DA9602B606B60E8
:109A84002B8242F606526A826B732B73FFF70CFE2D
:109A9400FFF724FE2A7BA9682046FFF76FFE0DE03E
:109AA40062B10D4B9B6801338B4207D10A4B0122F3
:109AB4005A73FFF77BFF01E0012B00D038BD002A69
:109AC400FCD1054B9B688B42F8D1034B01225A739E
:109AD400FFF76CFFF2E700BF984C00200378042BDB
:109AE40000D0704743681B78002BFAD010B5846807
:109AF400027E437E012A14BF00220122416904F13F
:109B04001000FFF79DFF10BD08B5214B1B7B7BB1F7
:109B1400012B20D07846FDF707FB1D4A138A013339
:109B240013821B4B5B8A13B1013B194A538208BD54
:109B3400174B1A8A41F282639A4204D8154B1B7858
:109B44003BB1012300E00123002BE6D0FFF72EFFF9
:109B5400E7E70023F8E70E4B1B8A41F28262934247
:109B640004D80C4A127872B1012200E00122002AC2
:109B7400D3D042F2B012934207D9054B01225A7353
:109B8400FFF714FFCDE70022F1E7FFF70FFFC4E76B
:109B9400984C0020AD4C002010B5184B1A685B6837
:109BA4009A4225D20446154B1B7B012B13D0144B30
:109BB4009A4212D2114B1A685B68403B9A4214D203
:109BC400EFF3108072B60D4A1368591C11602360BC
:109BD40090B962B610BD0B4BEAE7084B01225A73E9
:109BE400FFF7E4FE0028EBD1E4E7FFF777FDE7E7B2
:109BF400FFF774FD0F20EDE70020EBE7984C002001
:109C0400FFFF7F0000E0FF0008B568B90C4B1B683C
:109C140093B10B4A1368013B136063B9094B0022EB
:109C24009A73FFF7C3FE06E0064B01229A73044AB7
:109C340013680133136008BD7846FDF775FAE8E749
:109C44004C4C0020984C002000B58DB0ADF80800B5
:109C54008DF8102003910CA8032300F82C3DFEF787
:109C64001FFE0DB05DF804FB014B9868704700BF00
:109C7400984C0020054B1B7B012B02D0034B9868AA
:109C84007047024B98680138704700BF984C002019
:109C9400044B9B68584010F0010F00D0013B18465C
:109CA400704700BF984C0020014B187B704700BFE1
:109CB400984C002038B50A4B1B7873B9084B012225
:109CC4001A70084DA8602973FFF7EEFC00242C607D
:109CD4006C60FFF703FD204638BD0820FCE700BF99
:109CE400484C0020984C00202DE9F041002724E046
:109CF4002449BC2303FB04F3CA5A0132CA52022189
:109D0400284602F07BFB01360221284602F046FB7E
:109D140080B11C4ABC2303FB0423D3F80880B8F1A8
:109D2400000FE5D0BC2303FB04F3D25A01463846A6
:109D3400C047DDE78EB90137FFB2022F1FD83C467A
:109D4400BC2303FB07F308330E4D1D4404350221E5
:109D5400284602F023FB0026DAE70021284602F019
:109D6400B5FB0828E7D1074BBC2202FB0434A368E7
:109D7400002BE0D00022044938469847DBE7012055
:109D8400BDE8F081B84C0020A8F6030008B508230C
:109D940083731023437300F11C0343610323037390
:109DA40000F1180303610C3002F062FB08BD0000EF
:109DB40008B50378012B06D0022B07D07846FDF7AF
:109DC400B3F9002001E04FF4A97008BD0048FCE796
:109DD400645E010008B50278012A07D0022A13D074
:109DE4007846FDF7A1F94FF4FA7308E083685B1A2B
:109DF40098084FF4A97303FB00F303F5FA730748BB
:109E0400984228BF184608BD83685B1A180B044B98
:109E140003FB00F303F5FA73F1E700BFA08601002A
:109E2400645E010010B5044601210C3002F0B6FA5C
:109E3400A0B10D4AC4F89C200022C4F8A020616897
:109E4400FFF7C8FFC4F8A800C4F8AC40012384F8A5
:109E5400B83004F19C000BF0CBFE00B910BD78467D
:109E6400FDF762F9FAE700BF6D9F0200F8B50646F8
:109E74000C46174615680378012B18D11249A1FB2B
:109E84000431C9098900B468641B8C4200D30C46B0
:109E94008CB1706825F00305F168224629442844F2
:109EA400FFF794FB58B93B681C443C60F8BD784606
:109EB400FDF73AF9E2E77846FDF736F9E9E778463F
:109EC400FDF732F9EFE700BFEB5DF260F8B5074646
:109ED4000C46164615680378022B16D1114BA3FBCA
:109EE40004231B0C1B03BC68641B9C4200D31C464C
:109EF4007CB1786825F0030521462844FFF736FB3A
:109F040058B933681C443460F8BD7846FDF70CF941
:109F1400E4E77846FDF708F9EBE77846FDF704F93E
:109F2400EFE700BFB77609BB38B505460C461146C6
:109F34002378012B06D0022B0FD07846FDF7F4F8D6
:109F4400002304E0021D2046FFF790FFA368686821
:109F5400984214BF0020012038BD021D2046FFF79F
:109F6400B5FFA368F3E700002DE9F8430F46D1F8E5
:109F7400A850234B1B7863B90646A5F5FA7501F181
:109F84000C090121484602F009FA804640B1002438
:109F940022E00BF069FE002387F8B830BDE8F883AF
:109FA4007846FDF7C1F8F2E70BF05EFE0121484662
:109FB40002F024FA00237B6087F8B830114B18684C
:109FC40001F056FB3846FFF72DFFE7E74046FFF761
:109FD400EFFE2044A8420CD82A1B41463846FFF71E
:109FE400A3FF0028E0D100F03FFE841BEED5341A15
:109FF400ECE70BF039FE3846FFF714FFCEE700BF5D
:10A00400B44C0020B04C002010B5084801F010FBFF
:10A01400074B1860002406E0064BBC2000FB04300C
:10A02400FFF7B4FE0134022CF6D910BDED9C0200FA
:10A03400B04C0020B84C002038B504460D46022828
:10A0440005D8054BBC2202FB0434A56038BD784614
:10A05400FDF76AF8F5E700BFB84C00202DE9F84396
:10A0640006460C461746022816D8CCB12378012B95
:10A074001AD0022B3ED16368C3F30B03002B31D1FA
:10A08400A368C3F30B03002B30D1A368002B34D196
:10A094007846FDF749F830E07846FDF745F8E4E7FF
:10A0A4007846FDF741F8E1E7636813F0030F0DD13B
:10A0B400E36813F0030F0DD1A36813F0030F0DD160
:10A0C400A368D3B97846FDF72FF816E07846FDF774
:10A0D4002BF8EDE77846FDF727F8EDE77846FDF72E
:10A0E40023F8EDE77846FDF71FF8C9E77846FDF752
:10A0F4001BF8CAE77846FDF717F8EFF3108872B635
:10A10400BC2505FB06F505F10803204D1D44043567
:10A114000021284602F042F9814668B3002128460E
:10A1240002F06CF920686168A268E368C9F800006D
:10A13400C9F80410C9F80820C9F80C302FB1134A23
:10A14400BC2303FB06235B883B80104ABC2303FB30
:10A1540006235A8801325A8093F8B83073B90C4BED
:10A164001B780BB100200AE0084BBC2000FB063032
:10A17400FFF758FE002002E0042000E00020B8F1C0
:10A18400000F00D162B6BDE8F88300BFB84C0020D0
:10A19400B44C002018B1830B024AD05C70470020F5
:10A1A400704700BFB8F6030012DF704700B583B0F4
:10A1B4001378A3B1042B14D1072110F8013C163BEA
:10A1C400152B31D8DFE803F05930303030303030DF
:10A1D40030303030303030303030302E0F3A517D26
:10A1E400EBE70021E9E7022901D007291CD110F887
:10A1F400021C013901F062FEB0B1264B1B6813F05A
:10A20400400F11D0244B1B68012B0DDD234BD3F8D9
:10A2140004350190224A00928A222249022002F047
:10A224003DFB01E0022902D003B05DF804FB10F805
:10A23400021C0139C9B211F01FFDF5E70229F3D15F
:10A2440010F8021C0139C9B203F0E6FC0028EBD077
:10A25400104B1B6813F0400FE6D00F4B1B68012B0B
:10A26400E2DD0E4BD3F8043501900F4A00929D2293
:10A274000C49022002F012FBD6E701884FF6E46392
:10A284009942D1D110F8021C03390230FCF79CFE2C
:10A29400CAE700BF383300203433002000B0004048
:10A2A40008F70300FBF6030034F7030000B58DB094
:10A2B4002C22002101A814F06EFF0D238DF8043028
:10A2C40001A8FEF7EDFA0DB05DF804FB70B58AB095
:10A2D4000CF00EFA58B3064600238DF8103005AC86
:10A2E40005460FCD0FC42B682360727D052A04D95F
:10A2F400337D03F00F03072B20D1184B1B689BB150
:10A3040004AB0393337DC3F303038DF80430737DEF
:10A31400062B1DD9063B8DF8053006F11D0302936B
:10A324000E4B1B6801A8984730460CF0C1F90CF09D
:10A33400F9F980F00100C0B20AB070BD307D04AB01
:10A34400063A06F11D0100F00F000AF0ADFFD4E754
:10A3540000238DF805300293E2E700BFF04E0020A1
:10A3640070B582B0304B1B78002B55D1002857D0E4
:10A37400067A0F2E01D0072E54D10446C06870B15E
:10A38400FCF7E4FE0DF10700FFF70EFF0546002879
:10A3940043D19DF80730012B04D002253DE0FCF7A2
:10A3A400E3FEEFE7FCF7F6FE00F04CFB304601F06D
:10A3B400C5F8E07800F02CF900F0CAFF0BF0D6FBEA
:10A3C4001A480CF04BFA0BF00DF9FFF71DFE02F0E2
:10A3D4003DFF174803F01CFA04F08AFC204601F004
:10A3E40049FC2046FDF7E6FE03F096FF2046FFF702
:10A3F40031F9FCF7E9FD18B1062801D005460CE057
:10A4040000F050FD0B480AF031FF0B4B00221A609C
:10A41400054B01221A7000E00825284602B070BDE1
:10A424000E25FAE70725F8E7ED4E0020D1A2020039
:10A43400B1A2020028330020F04E002010B50E4BCC
:10A444001B789BB10D4B1B7893B900F0A7FF48B95B
:10A454000BF0AEFB044660B90CF0EAF8074B01229E
:10A464001A7006E07846FCF75FFEF1E7082400E086
:10A474000824204610BD00BFED4E0020EC4E002005
:10A4840010B5094B1B785BB10BF0A2FB044640B935
:10A494000CF0E4F800F0ECFF034B00221A7000E02B
:10A4A4000824204610BD00BFEC4E002030B583B018
:10A4B40004460D460E4B1B6813F4804F03D00D4B1E
:10A4C4001B68062B05DC29462046FDF7DBFE03B09E
:10A4D40030BD094BD3F80435084A0192084A00926A
:10A4E40040F2B1120749072002F0D8F9EBE700BFA8
:10A4F400383300203433002000B00040BCF60300A1
:10A504003CF40300FBF6030008B5FEF7F1F908BDBF
:10A5140008B500F0F3FE002008BD08B505F0B2FF51
:10A5240008BD0000064A136801331360B3F1704F8D
:10A5340002D0034B18687047134601221A60F8E7EB
:10A54400F44E002010B5044618B100232360636064
:10A5540010BD7846FCF7E8FDF7E738B50C4605462C
:10A5640068B184B100236360EFF3108372B62A6884
:10A574006AB16A6854606C6003B962B638BD7846E3
:10A58400FCF7D2FDEDE77846FCF7CEFDEAE72C6058
:10A59400F1E710B5044658B1EFF3108372B62068A2
:10A5A40008B142682260226832B103B962B610BDB4
:10A5B4007846FCF7B9FDEFE76260F6E710B50446AC
:10A5C40008B1206810BD7846FCF7AEFDF9E735DF29
:10A5D40070473CDF7047000010B504464FF0FF3071
:10A5E400FFF7F5FF4FF0FF312046FFF7F2FFBFF30F
:10A5F4004F8F0549CA6802F4E062044B1343CB60F1
:10A60400BFF34F8F00BFFDE700ED00E00400FA0543
:10A61400072814D8DFE800F0080C1504110F0A0607
:10A624006420704714207047FA2070471E2070473A
:10A634004FF4FA707047322070474B207047FA206D
:10A6440070479620704746DF7047F8B504460D46BC
:10A654004B1EDBB2012B09D8002222616261A26188
:10A66400E2612046FFF7EFFF012616E07846FCF78B
:10A674005BFDF1E7CA5CC8185200D2B2407842EAE6
:10A68400D012CA5401339BB20E2BF3DDCB7B5B009B
:10A69400CB73002F08DB0136F6B2AE420BD821464D
:10A6A40011F9207F0023EFE794F82F3083F087031C
:10A6B40084F82F30EFE7F8BD2DE9F04190B08446DF
:10A6C4000C4696461F4602F10F0636111FFA86F80D
:10A6D40004AD0068DCF80410DCF80820DCF80C3069
:10A6E4000FC50EF00F05B8F1000F02D085B100239D
:10A6F40000E0002398466BB1012104A8FFF7A5FFF1
:10A70400B8F1000F1BD0B0B20138000110230EE0E5
:10A714000123EFE70221F0E7013B9BB22218D25C50
:10A7240010A9194411F8101C4A400DF80320002BFD
:10A73400F2D100250C950D950E950F9534E0B1B22C
:10A744000139ADB22A4604EB0111684614F0FAFC53
:10A7540080230DF805306B1C03E000220DF8032064
:10A7640001330F2BF9DD10230AE0013B9BB21DF8E6
:10A77400032010A9194411F8101C4A400DF80320B5
:10A78400002BF2D1D5E7013B9BB210AA1A4412F870
:10A79400102C2118C95C4A4008A9CA54002BF2D1D4
:10A7A40004A8FFF750FF0135B3B2013BAB4202DD11
:10A7B40028011023F2E710230AE0013B9BB210AA00
:10A7C400D11811F8402C11F8101C4A4008A9CA5499
:10A7D400002BF2D104A8FFF736FF0CAC0FCC386085
:10A7E4007960BA60FB6010B0BDE8F08170B51E4EB0
:10A7F40010E063693360002363611B4AD368591E08
:10A80400D160ABB1184A9368013B93600023237075
:10A81400032D11D034682CB3134B9B6813B32578E4
:10A82400EDB2EB1EDBB2012BE3D904F11406F1E720
:10A834007846FCF779FCE5E723781BB12378DBB293
:10A84400062B0BD1636913B17846FCF76DFC012329
:10A854002370054B5A6862615C60DBE77846FCF75D
:10A8640063FCEFE770BD00BFFC4E002010B504464A
:10A87400436913B17846FCF757FC164B1B684BB180
:10A884006068144B1B685B68C31A002B02DB114B16
:10A8940019680DE00F4A136863611460D3680133CB
:10A8A400D36003B110BD7846FCF73EFCFAE71946C5
:10A8B4004B691BB15A68121A002AF8DB63614C61B8
:10A8C400044AD3680133D360002BEBD17846FCF7FC
:10A8D4002BFCE7E7FC4E0020114B5B68FBB110B585
:10A8E4000AE00023237004E0022323702046FFF7CC
:10A8F400BDFF0B4B5B688BB1094B5C6862695A60A6
:10A90400002363612378DBB2052BEAD02378DBB222
:10A91400012BE9D07846FCF707FCE5E710BD70474A
:10A92400FC4E002038B505461BE06269234B1A60D3
:10A9340000226261DA68511ED9602AB3A3683BB36E
:10A9440006232370A36821692846984700F08CF9F0
:10A954000546FFF74BFFFFF7BFFF2378DBB2062B5B
:10A964001AD0164B1B6843B3144B1B685B685B1B04
:10A97400642B22D5114B1C682378DBB2022BD4D074
:10A984007846FCF7D1FBD0E77846FCF7CDFBD5E75A
:10A994007846FCF7C9FBD3E7E26812B900232370B9
:10A9A400DFE76368134463605B1B642BF9D4022301
:10A9B40023702046FFF75AFFD3E738BDFC4E002032
:10A9C40008B5124B1B6873B1104B1B685B68C31A44
:10A9D40013F1640F08D402230D4A00F1640101202D
:10A9E40000F006F970B908BD084B19680223084A3B
:10A9F4004968012000F0FCF80028F4D07846FCF700
:10AA040093FBF0E77846FCF78FFBECE7FC4E002065
:10AA140039AA020008B5FFF7E9FEFFF75DFF00F071
:10AA240023F9FFF77FFF00F01FF9FFF7C9FF0120AB
:10AA340008BD000008B5024B186800F019FE08BDF7
:10AA4400F84E002008B5064B00221A605A609A603E
:10AA5400DA60044800F0ECFD034B186008BD00BF49
:10AA6400FC4E002019AA0200F84E002038B5044616
:10AA7400F0B1A36803B3EFF3108572B600236361EA
:10AA840023781BB12378DBB2062B19D1636913B188
:10AA94007846FCF749FB012323700B4B5A6862612B
:10AAA4005C6005B962B6094B186800F0E1FD38BD79
:10AAB4007846FCF739FBDCE77846FCF735FBDAE748
:10AAC4007846FCF731FBE1E7FC4E0020F84E00200D
:10AAD40038B50446E0B1EFF3108572B62378DBB2E3
:10AAE400062B19D02378DBB2012B1AD02378ABB113
:10AAF4002378033BDBB2012B03D90B4A9368013360
:10AB0400936004232370094B186800F0B1FD05E03D
:10AB14007846FCF709FBDEE70023237005B962B62B
:10AB240038BD05232370F9E7FC4E0020F84E0020C1
:10AB340070B50E460446E0B1EFF3108572B6237883
:10AB4400DBB12378DBB2062B17D02378DBB2012BE1
:10AB540030D02378DBB2052B2CD02378033BDBB237
:10AB6400012B03D9154A936801339360032323709F
:10AB740014E07846FCF7D8FADEE723781BB1237893
:10AB8400DBB2062B12D1636913B17846FCF7CCFA19
:10AB940001232370094B5A6862615C606660084B4C
:10ABA400186800F065FD05B962B670BD7846FCF71B
:10ABB400BBFAE8E701232370F0E700BFFC4E002056
:10ABC400F84E002010B4094B00F15002002443F861
:10ABD400224000F110040122A240C3F8042300F52E
:10ABE400A87043F820105DF8044B704700800040C3
:10ABF400022825D838B533F0030423D1EFF31084A9
:10AC0400124D2C6072B6124C44F82020114A42F8BE
:10AC14002010114A1354114B002243F82020104BEA
:10AC24001B7833B10F4B1B68CA1A07D41146FFF7C0
:10AC3400C9FF064B186838B962B604E05A1AF5E73A
:10AC4400072070470A2038BD0020FCE7304F002061
:10AC5400104F0020244F00200C4F0020384F0020BC
:10AC64001C4F0020204F0020EFF310830C4A136088
:10AC740072B60C4B1B787BB10B4B0022C3F84C21F2
:10AC84000122DA64D3F84C05084B1B681844044BC2
:10AC94001B6803B962B67047054B1868F7E700BF35
:10ACA400304F00201C4F002000800040204F002027
:10ACB400344F002070B5002418E01F4B002243F8E5
:10ACC4002420012303FA05F51C4BC3F80853FFF7AE
:10ACD400CBFF1B4B1B5D13F0020F21D0B04704F1D7
:10ACE4005003164A002142F823100134022C21D8C3
:10ACF40004F15003114A52F82330002BF5D0D2F856
:10AD0400043304F11005EB4013F0010FEDD00A4BAE
:10AD140053F82460002ED0D17846FCF705FACCE72E
:10AD24000146304600F02EFC0028D8D07846FCF7C7
:10AD3400FBF9D4E770BD00BF104F00200080004035
:10AD44000C4F002070B50546002414E0981A27E043
:10AD54005E1A29E02946184600F014FC002836D172
:10AD64002A4B53F824302BB101221A60274B0022BE
:10AD740043F824200134022C3AD8254B04F5A87258
:10AD8400002143F8221004F1500243F8221053F832
:10AD94002230204B53F824201F4B1B68D01AD5D4E3
:10ADA40005F17801CE1AD3D4864214D91B4B53F83B
:10ADB4002430002BD4D0194A002142F82410184A18
:10ADC400125D12F0020FC5D028469847C8E77846AE
:10ADD400FCF7AAF9C4E7114B53F82430002BC9D06F
:10ADE400E0B2511B02D4FFF7EDFEC3E7A91AFAE75C
:10ADF4000C4B1B681BB90C4B4FF480721A60064B4A
:10AE04001D600A4B01221A7070BD00BF384F00202C
:10AE140000800040244F0020204F0020104F0020CD
:10AE24000C4F0020304F002000E100E01C4F0020B8
:10AE3400002300E00133022B0ED80F4AD25C12F03B
:10AE4400010FF7D000220C49CA540C4941F82320C1
:10AE54000B4941F82320EDE70A4B18600A4B002206
:10AE64001A700A4B4FF0FF32C3F80823084B4FF413
:10AE74008072C3F8802170470C4F0020104F0020CF
:10AE8400384F0020344F00201C4F00200080004029
:10AE940000E100E0024A136801331360704700BF09
:10AEA400444F002010B50023084A1360084C094A97
:10AEB400A260094AE2602361FFF7D6FE00F5C330C1
:10AEC400A03060602046FFF7D1FD10BD444F002044
:10AED400484F002099AE0200A086010030DF704781
:10AEE40031DF704710B402684368A2EB73128468C0
:10AEF40083EAF4330360C1680C4444601144816004
:10AF04001344C36018465DF8044B704770B582B0B3
:10AF14000D46064608B100240BE07846FCF704F918
:10AF2400F9E79DF807103019FFF7DAFF9DF80730AD
:10AF34001C44A5420DD90DF10700FFF7CFFF9DF882
:10AF44000730002BF7D02A1B9342EAD98DF807204B
:10AF5400E7E702B070BD000030B583B005460024B9
:10AF640002A840F8044D0421FFF7D0FF074B2B60E3
:10AF7400019B6B60AB60EB6003E02846FFF7B2FF18
:10AF84000134132CF9D903B030BD00BFED5EEAF1F2
:10AF940008B5A0F1C8039BB2632B0AD9A0F5967338
:10AFA4009BB2632B08D9B0F5C87F08D300F07AFEB2
:10AFB40001E00FF043FD08BDFDF770FBFBE7062041
:10AFC400F9E708B5A0F1C8039BB2632B0AD9A0F531
:10AFD40096739BB2632B08D9B0F5C87F08D300F0F1
:10AFE400B3FE01E00FF03CFD08BDFDF7D3FBFBE72A
:10AFF4000620F9E748DF704749DF70474ADF7047AA
:10B004002DE9F00F1F4BD3F804650027837AA3BB07
:10B014001D4BD3E90023B41A24F07F4A4FF0000BF0
:10B024004FEA4A124FEA4B13B2EB0A0263EB0B03EB
:10B03400590241EAD2514FEA422C0D461CEB0A0157
:10B0440045EB0B024FEA821949EA91694FEA8118EC
:10B054001346B8EB010269EB03031AEB02044BEB52
:10B064000305E30B43EA4542436813444360064B3C
:10B07400C3E90067BDE8F00F7047002383720268DC
:10B08400F2E700BF00B00040984F002010B504461E
:10B094000023C3600361FFF7B3FF2368084A926883
:10B0A40022600121217503B9064B991AA161B1F5FA
:10B0B4007A7F01D39A4202D94FF47A73A36110BD07
:10B0C400804F002080969800094B03221A75094A84
:10B0D4009A611A6840F6D8639A4204D8054B40F640
:10B0E400D8629A607047034B43F2B0629A6070472B
:10B0F400604F0020804F002008B50B4B1B78012BBC
:10B1040005D0022B0BD07846FCF70EF803E002239F
:10B11400037501238372044B00221A7008BD0323B4
:10B124000375024B8361F6E7914F0020804F0020A6
:10B1340038B5054600240475012343724068FFF7BF
:10B1440001FE0AF0FDFD6B682A6813440A49096888
:10B15400283101FB02F1094AA2FB0121A3EB914131
:10B164000323074A78392046FFF742FD00B938BD6A
:10B174007846FBF7D9FFFAE77C4F002083DE1B43B8
:10B18400CDB0020010B50C4631B10369013303613F
:10B194008269036813440360C3680133C3600122F6
:10B1A4000275826952088261012B0DD0022B19D0DD
:10B1B40082690368134417498B4222D840F6D76347
:10B1C4009A4221D800231DE0B2F5FA7F05D040F65B
:10B1D400D8639A42ECD88361EAE7002CF7D10023C4
:10B1E4008361E5E70369022B06D0012BE0D1002C33
:10B1F400DED100238361DBE70268064B9B1A83617F
:10B20400D6E7002313B110BD0123FBE7FFF790FF3E
:10B21400F9E700BF80969800437A1BB90E4B0022D1
:10B224001A70704710B504460AF0A6FD60682268DB
:10B2340010440A4B1B68283303FB02F3084AA2FBA1
:10B244000323A0EB93407838FFF7F2FD00236372E9
:10B25400014B00221A7010BD904F00207C4F00203B
:10B2640083DE1B4308B5224B01221A72214B1B7843
:10B2740013B1214B1B781BB31D4B00221A750428F4
:10B284001AD8DFE800F00314110C07001848FFF780
:10B29400FDFE1EE001211648FFF774FF19E00021AE
:10B2A4001348FFF76FFF14E00AF004FD11E0FFF705
:10B2B40001FD0AF033FD0CE07846FBF735FF08E0AA
:10B2C400FFF7D2FC0A4B5A68801A18601846FFF739
:10B2D40013FF074B1B7D023BDBB2012B04D904484F
:10B2E40000230372143008BD0148FFF795FFF6E709
:10B2F400604F0020914F0020904F002008B5043883
:10B3040003280DD8DFE800F00D190902FFF774FED9
:10B3140030B17846FBF708FF02E07846FBF704FFFC
:10B3240008BD0A4840F6D8638360FFF767FE00282B
:10B33400F6D07846FBF7F8FEF2E70448FFF75EFE26
:10B344000028EDD07846FBF7EFFEE9E7804F0020B8
:10B3540010B40D4A0023137013710121517143F28B
:10B36400B064946043F69824D460084A1060084A94
:10B374001370084A1370084A13725372136091725F
:10B3840053605DF8044B7047804F00207C4F0020D1
:10B39400904F0020914F0020604F002008B50648D0
:10B3A400FFF728FE034608B1184608BD0348FFF717
:10B3B40025FE0346F8E700BF69B20200804F002073
:10B3C400084B1B7D032B09D0074B1B78012B07D09F
:10B3D400022B01D0002070470120704701207047E4
:10B3E40001207047604F0020914F0020014B5868A6
:10B3F400704700BF604F00200E4B5B7A0BB90020F2
:10B40400704710B50B4B5C681A6814440A4B1B68F0
:10B41400283303FB02F3094AA2FB0323A4EB93445E
:10B42400783CFFF721FC0346201A00D410BD181BFA
:10B43400FCE700BF604F00207C4F002083DE1B43ED
:10B44400014B187A704700BF604F0020EFF3108360
:10B4540072B6054A527A22B1044A4FF48071C2F896
:10B46400001103B962B67047604F002000E100E0AC
:10B4740008B5034B01221A70FFF7E8FF08BD00BFAF
:10B48400914F002008B5034B02221A70FFF7DEFF2C
:10B4940008BD00BF914F002008B5094B1B782BB1A4
:10B4A40048B9084B1B7813B1012300E00023044A78
:10B4B400107013B908BD0023F9E7FFF7C7FFF9E7D8
:10B4C400904F0020914F002008B50378012B10D035
:10B4D40013B1022B06D008BD4368002BFBD0806853
:10B4E4009847F8E74368002BF5D0C168806898470F
:10B4F400F1E74368002BEED080689847EBE7000043
:10B50400044B1B780F2B04D0034B4FF48022C3F859
:10B5140000217047E450002000E100E010B501462E
:10B524000548FDF7CBFF20B90446FFF7E9FF2046A5
:10B5340010BD0424FBE700BFA04F002010B50C4C45
:10B5440020700C480C4B0360102343608360FDF7AC
:10B5540099FF0A48FEF7F6FF23780F2B07D05B010B
:10B56400DBB2074A82F812334FF48023136010BD14
:10B57400E4500020A04F0020B44F0020E8500020E9
:10B5840000E100E030B585B00C46054648B1002323
:10B594008DF80030019502946846FFF7BFFF05B0AF
:10B5A40030BD7846FBF7C0FDF1E7000010B5EFF3BE
:10B5B400108472B60A490A68531C0B6042B9094ADE
:10B5C40012780F2A04D0084A4FF48021C2F8801060
:10B5D40013B104B962B610BD7846FBF7A5FDF8E7D0
:10B5E400B4500020E450002000E100E010B5EFF377
:10B5F400108472B60B4B1B687BB10A4A1368013B7B
:10B6040013603BB9084B1B780F2B03D0074B4FF447
:10B6140080221A6004B962B610BD7846FBF784FD37
:10B62400EBE700BFB4500020E450002000E100E04C
:10B6340010B5044680B10C4B1B68082B10D8EFF3EF
:10B64400108372B6084A1068411C1160074A42F818
:10B65400204003B962B610BD7846FBF765FDEAE702
:10B664007846FBF761FDEAE7B8500020BC500020A3
:10B6740038B504460D4B1B68834213D9EFF310858C
:10B6840072B661090A4A04F01F04012303FA04F4A0
:10B6940052F82130234342F82130FFF731FF05B936
:10B6A40062B638BD7846FBF73FFDE7E7B8500020A7
:10B6B400E050002070B50D461646044658B175B1E9
:10B6C400EFF3108372B6A560E66000222274246052
:10B6D40003B962B670BD7846FBF726FDEFE77846FE
:10B6E400FBF722FDECE7000038B5044690B1A368EF
:10B6F400A3B1EFF3108572B6237C9BB901232374A5
:10B7040021460948FEF729FFFFF7FAFE002005B994
:10B7140062B638BD7846FBF707FDE8E77846FBF7E5
:10B7240003FDE6E71120F2E7E850002010B50446D7
:10B7340008B1207C10BD7846FBF7F6FCF9E7000061
:10B7440070B584B02C4B1B7823B901252A4B1D708E
:10B7540000240AE07846FBF7E7FCF6E7274B53F8AA
:10B76400243098470646F0B10134254B1B68A342A8
:10B774001ED96109234A52F8213004F01F00C34046
:10B7840013F0010FF0D0EFF3108372B6012606FA1E
:10B7940000F052F8216026EA000642F82160002BEE
:10B7A400DCD162B6DAE72046FFF762FF3546DBE715
:10B7B4001548FEF7EEFE07E0A368E068984700230B
:10B7C40023741148FEF7E5FE50B10468237C002B76
:10B7D400F2D17846FBF7A8FCEEE76846FFF774FE63
:10B7E40069460A48FDF797FE0028F6D0024B00226E
:10B7F4001A70284604B070BDF0500020BC500020E0
:10B80400B8500020E0500020E8500020A04F002055
:10B8140008B5FFF795FF08BD46DF704770B58CB0DB
:10B8240003460E4615466C46006859689A68DB68FC
:10B834000FC430687168B268F3680FC46846FFF7D4
:10B84400EBFF08AC0FCC28606960AA60EB600CB019
:10B8540070BD08B5FEF730FF08BD08B502F0ABF8BF
:10B8640008BD08B502F0E1F808BD38B5032900F2B7
:10B874009380DFE801F0023535671970817A5A78D0
:10B8840061F306025A70C17AD2B261F3C7125A70D8
:10B89400C168C1F3074201F47F442243090401F45F
:10B8A4007F010A4300219A70C2F30724DC70120C52
:10B8B4001A710489220A42EA0422A3F80520D971E4
:10B8C400197201690A0202F47F0242EA0162080A5B
:10B8D40000F47F40024342EA1162C3F8092038BDF4
:10B8E4001970597801F0800162F3C7115970C16869
:10B8F400C1F3074201F47F442243090401F47F01A8
:10B904000A439A70C2F30721D970120C1A71018983
:10B914000A0A42EA0122A3F8052041880A0A42EAF7
:10B924000122A3F8072001690A0202F47F0242EA15
:10B934000162080A00F47F40024342EA1162C3F83C
:10B944000920CCE7197000245C70C168C1F3074278
:10B9540001F47F452A43090401F47F010A439A70E4
:10B96400C2F30721D970120C1A7101890A0A42EA3A
:10B974000122A3F80520DC711C7201690A0202F499
:10B984007F0242EA0162080A00F47F40024342EA6D
:10B994001162C3F80920A2E77846FBF7C5FB9EE7CE
:10B9A40070B584B00E461446054668B162B10023F2
:10B9B4000093019302930393234632462946684633
:10B9C400FFF747FF04B070BD7846FBF7ADFBEEE729
:10B9D400F0B585B00F4614461D46064618B112B19F
:10B9E4000BB10B9B13B97846FBF79EFB6B463A46AB
:10B9F40031462046FFF72DFF0B9B9DF82820294652
:10BA04006846FFF726FF05B0F0BD00002DE9F047BA
:10BA140086B000AF884615469946044608B101B180
:10BA240013B97846FBF780FB05F1110605F1100AFE
:10BA340005F11803DB086A46A2EBC3039D46254BB8
:10BA44001B6807F1180040F8043D6A460421FFF71B
:10BA5400A7FF3B1D102221466846FFF7FAFE2A463F
:10BA64004146684613F06EFB01230DF80530EA18D1
:10BA74006B4692B26946381DFFF7EBFE9DF80F3016
:10BA840003F07F034C4604F8013B2A46414604A8D0
:10BA940013F058FB02230DF80A30B6B2234632469F
:10BAA4006946381DFFF7D5FE20686168A268E3681F
:10BAB400009001910292039303230DF80A3009F1D7
:10BAC400110332466946381DFFF7C3FE1837BD46D9
:10BAD400BDE8F08760F7030070B588B00D460646F0
:10BAE40000B3F9B1114C6368039304AA042103A8B9
:10BAF400FFF756FF04AB102231461846FFF7A9FEA4
:10BB0400083494E8030001908DF8081004AB052272
:10BB140001A91846FFF79DFE06AB03CB28606960B8
:10BB240008B070BD7846FBF7FFFADBE760F7030067
:10BB340070B586B00D460646F8B1F1B1114C2369D3
:10BB4400019302AA04210DEB0100FFF729FF02ABC8
:10BB5400102231461846FFF77CFE636906A941F8B6
:10BB6400183D02AB04221846FFF773FE9DF8173008
:10BB740003F03F032B7006B070BD7846FBF7D4FA90
:10BB8400DCE700BF60F7030010B5044658B1237822
:10BB94007BB1E368B3F1807F0DD294F90A30002BB6
:10BBA40005DB012006E07846FBF7BEFAEFE700204C
:10BBB40000E0002010BD0020FCE730B587B004464B
:10BBC400037B8DF8043002688368D27A22B308229A
:10BBD400134409330293236803936368049305A908
:10BBE40001A802F0F7F8E0B1237B012B09D0256806
:10BBF400FEF740F8286120680C30FDF7CDFF0546BC
:10BC040060B92168059800F0B8F9059B09332361F0
:10BC14000025284607B030BD0422D9E702F056F9C2
:10BC2400F7E70425F5E7000030B583B00F4B1D7826
:10BC340075B1837A012B16D904460378012B0AD0F7
:10BC44000B4B1B6823B1A27A61882089984705466B
:10BC5400284603B030BD6946408809F081FA0028BF
:10BC6400EED00025F4E70025F2E700BFF8500020ED
:10BC7400F450002008B560B14268084B1A60084BC4
:10BC840001221A70FDF72EFEFDF7BCFD02F014FD33
:10BC940008BD024B00221A60F1E700BFF4500020F7
:10BCA400F8500020002945D008B5A0F5C870062832
:10BCB40042D8DFE800F00A1B0424302A390049681E
:10BCC400012003F069F8002008BD1E4A12784B6871
:10BCD4009A4201D10020F7E7003318BF0123194A23
:10BCE4001370012002F0F4FA0020EDE749680729F7
:10BCF40024D8C9B2012003F029F80020E4E7097927
:10BD0400012003F073F80020DEE74968002003F007
:10BD140043F80020D8E74968072911D8C9B20020A0
:10BD240003F014F80020CFE70979002003F05EF84F
:10BD34000020C9E70E2070470520C5E70720C3E7A8
:10BD44000720C1E7F8500020002931D010B50C4677
:10BD5400A0F5C87005282DD8DFE800F00B12032CDD
:10BD6400221A012003F02CF86060042323600020D1
:10BD740010BD114B1B784B6004230B600020F7E7C8
:10BD8400012002F0F9FF6060042323600020EFE744
:10BD9400002003F015F86060042323600020E7E727
:10BDA400002002F0E9FF6060042323600020DFE745
:10BDB4000E2070470520DBE7F850002010B504463C
:10BDC40050B1236863B123685B696BB100232373AB
:10BDD4002046FFF7F2FE10BD7846FBF7A5F9F0E721
:10BDE4007846FBF7A1F9EEE77846FBF79DF9EDE716
:10BDF40010B5044690B12369A3B12368B3B1236895
:10BE04005B69BBB1206900F01EF900230246A168FA
:10BE1400206800F078FA02F031F810BD7846FBF79C
:10BE240083F9E8E77846FBF77FF9E6E77846FBF71E
:10BE34007BF9E4E77846FBF777F9E3E770B588B078
:10BE440004460E461546837A013B8372039005929D
:10BE54004FF0FF33049301238DF8183003A8FFF744
:10BE6400ACFE98B1104B1B6813F0020F16D00F4BA9
:10BE74001B68012B12DD0E4BD3F804350D4A0092DA
:10BE840091220D49022000F009FD07E02A463146BF
:10BE9400079813F057F903A8FFF7AAFFA37A013311
:10BEA400A37208B070BD00BF3833002034330020C3
:10BEB40000B00040ACF703009FF7030070B590B0EA
:10BEC400002843D0044616460D4600F0C2F8021B73
:10BED400214608A813F036F90023009308AB224644
:10BEE400294602A800F0CEF9044610B1204610B04D
:10BEF40070BD02A8FFF748FE0028F7D0079BD3B116
:10BF0400314602A804F0F0FA294602A800F093F89A
:10BF1400C5B2334602AA29460DF12900FCF750FBAD
:10BF2400044602A8FFF780FE48B90599BDF8100041
:10BF3400FBF76CF9DAE77846FBF7F6F8E0E72A4610
:10BF44000DF1290102A8FFF779FFEEE70E24CDE7F2
:10BF54004B78DB09C3724B7803F07F0383728A78D2
:10BF6400CB781B0243EA02430A791343C3604A793C
:10BF74008B7943EA02230381704738B50D460446A2
:10BF8400002840D0002D42D02889FEF703F901286B
:10BF940041D195F90A30002B41DBEB68B3F1807F86
:10BFA40041D26B69002B42D02B6903F00102237844
:10BFB40003F07F0343EAC21323706A69127803F023
:10BFC400800302F07F0213432370EA7A637803F05C
:10BFD4007F0343EAC213DBB26370AA7A03F08003DF
:10BFE40002F07F0213436370EB681A0CA2701A0A02
:10BFF400E27023712B891A0A6271A3716B881A0A81
:10C00400E271237238BD7846FBF78EF8BAE77846BA
:10C01400FBF78AF8B8E77846FBF786F8B9E778467D
:10C02400FBF782F8B9E77846FBF77EF8B9E778467C
:10C03400FBF77AF8B8E7C37A1BB90420081A093861
:10C0440070470820FAE7093870470730704709300D
:10C0540070470130704770B588B004460D461646E7
:10C06400002300938DF804300269130203F47F0364
:10C0740043EA0263110A01F47F410B4343EA12636A
:10C08400CDF805302846FFF7E0FF0368CDF8093006
:10C0940082888379ADF80D208DF80F30606904AA89
:10C0A40069461130FFF7BAFB3046FFF7D2FF04466A
:10C0B4002846FFF7CEFF062308E0013B9BB2C25C93
:10C0C40008A9194411F8101C4A40E254002BF4D179
:10C0D40008B070BD2DE9F04395B004AF04460D4699
:10C0E40091461E4697F86480002387F83F303B84CE
:10C0F400FB6107F130033B611046FFF7A6FF78614F
:10C104003046FFF7A2FF78623B6E636132464946D0
:10C114002046FFF7A0FF31462046FFF719FF20898C
:10C12400FEF738F801281DD04FF00009B9F1000FCF
:10C134004BD0E37A002B33D00823DBB287F82C30C2
:10C14400ED1A073DADB23D837B691D44BD62B8F174
:10C15400000F27D0B8F1010F3DD07846FAF7E4FF7D
:10C16400002120E0A5F10902E37A2BB108239A42C9
:10C1740004D24FF00009D9E70423F8E7E1682089E5
:10C18400FBF71EF8814610B14FF00009CEE7391DC8
:10C19400208908F0E5FF0028C8D14FF00109C5E760
:10C1A4000423CAE7002107F1300300222046FFF7E9
:10C1B4005CFB63690133FB6007F13F0107F10C008D
:10C1C400FFF74FFB97F83F303BB997F83F004437F0
:10C1D400BD46BDE8F0830321E5E7F379307A40EA10
:10C1E40003206080FDF7D6FF20701F4B1B6813F0FF
:10C1F400020FEAD01D4B1B68032BE6DD6C46B7F833
:10C2040018C04FEA4C030833DB08A4EBC3039D4674
:10C214000DF1100E7546002311E07A6AD25C4FEAE4
:10C22400121859001248066816F8086005F81360D9
:10C2340002F00F0201310068825C6A5401336345E5
:10C24400EBD300230EF81C300A4BD3F80435CDF899
:10C2540008E0094A0192094A0092E62208490420AA
:10C2640000F01CFBA546B0E738330020343300202F
:10C274003C33002000B0004010F8030038F4030001
:10C2840003F803002DE9F04784B088461546994623
:10C294009DF83070064618B112B10BB19A4202D122
:10C2A4007846FAF741FF2878C009FDF7F1FC3061C0
:10C2B4000023736195F800A00AF07F0A02930393A8
:10C2C40001E0029BCBB103AA02A9504608F024FE68
:10C2D4000024012CF5D804AB03EB840353F8083C89
:10C2E400002BEED0019700934B462A464146304638
:10C2F400FFF7F0FE18B90134EBE7052000E0002059
:10C3040004B0BDE8F087F0B58FB00C4615461F4663
:10C31400064650B16DB1012F0FD897B1012F39D016
:10C324007846FAF701FF00210CE07846FAF7FCFEA4
:10C33400F0E77846FAF7F8FEEDE77846FAF7F4FE08
:10C34400EBE700210AAB00223046FFF78EFAF37ABE
:10C3540013BB04238DF824307369013301930AABB2
:10C3640002932846FFF771FE03900790A31C9BB22B
:10C37400ADF810300022ADF818200592184408904A
:10C3840001A8FFF76AFA2A4629463046FFF763FEFA
:10C394000FB0F0BD0321D5E70823DBE738B50D4620
:10C3A4000446C8B12378AB421AD9EDB96268237840
:10C3B400134413F8013CA1780B44DBB212789B1AA6
:10C3C400DBB2CBB16368585DA378013B1840A36826
:10C3D400627802FB003038BD7846FAF7A5FEE1E743
:10C3E4007846FAF7A1FEE0E76268531913F8013CB6
:10C3F400525D9B1ADBB2E4E70020ECE738B50C464B
:10C404000546A0B12B78A34215D9C4B96A682B7824
:10C41400134413F8013CA9780B44DBB212789B1A3D
:10C42400DBB21BB16A68135D0133135538BD78461E
:10C43400FAF77AFEE6E77846FAF776FEE5E76A6801
:10C44400131913F8013C125D9B1ADBB2E9E710B52E
:10C45400044608B1002307E07846FAF765FEF9E7D9
:10C4640062680021D154013322789A42F8D810BD71
:10C4740010B5044643786BB12378012B0ED9A36819
:10C4840083B1636893B1A378A3B15A1E134217D042
:10C49400002310E07846FAF747FEEDE77846FAF70E
:10C4A40043FEECE77846FAF73FFEEAE77846FAF708
:10C4B4003BFEE8E700232BB12046FFF7C8FF10BD81
:10C4C4000123F8E77846FAF72FFEF5E738B50C466E
:10C4D400054658B12B78A3420CD97CB16B681A1964
:10C4E40012F8010C1B5DC01AC0B238BD7846FAF7C9
:10C4F4001BFEEFE77846FAF717FEEEE76A682B783B
:10C50400134413F8010CAB781844C0B21378C01A62
:10C51400C0B2EAE728B108B529B1FFF709FB00204A
:10C5240008BD0E2070470E20FAE768B171B110B54E
:10C5340082B00B46002402A901F8014D0122FFF745
:10C5440065FA204602B010BD0E2070470E207047D9
:10C5540000B330B58BB00546F1B10C461031FFF78E
:10C56400BBFA0E4B09930E4B93E803000790ADF80A
:10C57400201003AA042109A8FFF712FA0194062344
:10C58400009307AB03AA10212846FFF721FA0020E5
:10C594000BB030BD0E2070470E20F9E76E6B626B56
:10C5A40024F80300E8B130B58BB00546D9B10C4688
:10C5B4000E4B09930E4B93E803000790ADF820103F
:10C5C40003AA042109A8FFF7EBF9019406230093B9
:10C5D40007AB03AA10212846FFF7FAF900200BB095
:10C5E40030BD0E2070470E20F9E700BF6E6B696BFB
:10C5F40024F8030010B330B587B0044601B30D46E8
:10C60400104B019302AA04210DEB0100FFF7C8F9B6
:10C6140002AB102221461846FFF71BF99DF816308D
:10C624001B0203F47C536FEA43436FEA53439DF8C0
:10C63400172013432B80002007B030BD0E20704715
:10C644000E20F9E77674616438B50C4683692BB122
:10C654000268406801FB0020984738BD05684068BF
:10C664000246002104FB005012F095FDF5E738B5B1
:10C674000546002404E021462846FFF7E5FF01347F
:10C68400AB68A342F7D8013BEB6038BDF8B504466C
:10C694000F46C56800260CE0216863681A4605FB4E
:10C6A4000311384612F018FD88B9012316E001364B
:10C6B4001D46A368B34210D96369002BECD02268ED
:10C6C400616805FB012138469847034630B96B1E63
:10C6D400002DECD1A368013BE9E700231846F8BD1F
:10C6E40038B5C3680133C3608268934208D00369D4
:10C6F4004BB10268C468406800FB0420984738BD09
:10C704000023C360F3E70468C5684068024600FB81
:10C71400054012F017FDF2E770B50E46044648B125
:10C7240041B12368B34209D0256865B92660002366
:10C73400336017E07846FAF7F7FCF2E77846FAF741
:10C74400F3FCF1E725462C682CB1B442FAD17846C3
:10C75400FAF7EAFCF6E735B12EB1B54202D02B6800
:10C7640033602E6070BD7846FAF7DEFCF5E738B525
:10C7740005460C4649B140B12A68CAB1A24209D162
:10C7840023682B60002020600CE07846FAF7CCFC8C
:10C79400F2E71A4613680BB1A342FAD152B1A3428D
:10C7A40001D0052038BD2368136000202060F9E71C
:10C7B4000520F7E70520F5E72DE9F0410D4617467A
:10C7C400064608B101B112B97846FAF7ADFC3368F0
:10C7D400AB4204D0346834B14FF0000809E0784625
:10C7E400FAF7A2FCF6E73560002028600FE0A046C7
:10C7F400344654B129462046B84730B92668B54274
:10C80400F5D17846FAF790FCF1E714B10F20BDE8B2
:10C81400F081B8F1000F09D045B1A8450AD0D8F885
:10C8240000302B60C8F800500020F0E77846FAF793
:10C834007BFCF2E70020EAE730B583B0184606AC8B
:10C8440054F8045B00920B460246054900200AF0A6
:10C854005BFC2246294600200AF06CFB03B030BD85
:10C864002CF80300034B1860034B1960034B1A6048
:10C87400704700BF38330020343300204033002099
:10C8840030B583B0044C246824B1079D0195069DFE
:10C894000095A04703B030BD4033002030B585B0CB
:10C8A40008AC54F8045B039401940095FFF7E8FF87
:10C8B40005B030BDC268137951795B1A03F57F2343
:10C8C40003F6FF731B0303F58053134442699B1A59
:10C8D4008068181A704770B50579012D01D90020B8
:10C8E40070BD044606683046FFF7E4FF3DB9A389EE
:10C8F4009B00834207DB73681BB90020F0E7002329
:10C90400F7E70120ECE70020EAE738B505460C46D6
:10C9140010F0030F0DD114F0030F0ED10023B3EB6D
:10C92400940F0ED255F82320B2F1FF3F0BD10133FF
:10C93400F5E77846FAF7F8FBEDE77846FAF7F4FB03
:10C94400ECE7012038BD0020FCE770B50546002463
:10C954000EE0002300E0002318463BB35379A342C2
:10C964001BD1EB681E4432792B699A4219D10134E8
:10C974002B69A34219D9EB6826039A199B5D083BDE
:10C98400DBB2F62BE7D85379FF2B04D01379FF2BB6
:10C99400DFD00123E0E70023DEE77846FAF7C4FBA3
:10C9A400DFE77846FAF7C0FBE1E7012070BD00003D
:10C9B400F0B585B004460368DB68187819795A79AC
:10C9C400891A01F57F2101F6FF71090301F58051F0
:10C9D400E2891944184401F0ADF9074623689E68BA
:10C9E40026F47F6525F00F0505F58055A81BA2895F
:10C9F4009200824237D2B51804F10C02A3899B003D
:10CA040001208DF8000001960392029300226946EA
:10CA1400FDF724FB002852D101208DF80000019578
:10CA24002E4B0393042302932D4A6946FDF716FB0C
:10CA3400002848D19FB122683988536803EB8103E9
:10CA4400536001208DF800000197264B03930423C3
:10CA54000293234A6946FDF701FB002837D1A660FB
:10CA6400002005B0F0BDD9680B7991F805C0A3EB9F
:10CA74000C0303F57F2303F6FF731B0303F58053B5
:10CA84000B449D4227D0824202D12A781544B3E751
:10CA940001208DF800000196134B039304230293A5
:10CAA40000226946FDF7DAFA28B92E782E44A589C2
:10CAB40006EB8505A0E77846FAF736FBF5E77846F6
:10CAC400FAF732FBA8E77846FAF72EFBB2E7784686
:10CAD400FAF72AFBC3E70120C3E700BF60F80300AD
:10CAE4002252002058F803005CF8030010B584B00B
:10CAF40004460368DB68187819795A79891A01F5AC
:10CB04007F2101F6FF71090301F58051E28919447F
:10CB1400184401F00FF9E0B10346A06021680088D1
:10CB24004A6802EB80024A6001208DF800000193FC
:10CB3400094B039304230293084A6946FDF78EFACE
:10CB440010B9002004B010BD7846FAF7EDFA0020C1
:10CB5400F8E70220F6E700BF58F80300225200204D
:10CB640070B584B005460368DE68437B06EB033684
:10CB740008213046FFF7C9FE80B9002400E00134E3
:10CB8400072C0BD8335D05F10802125D9342F6D0F1
:10CB9400FF2BF4D07846FAF7C7FAF0E708350120FE
:10CBA4008DF800000196039508230293054A69460F
:10CBB400FDF754FA10B9002004B070BD7846FAF7B6
:10CBC400B3FAF8E72252002000B585B00368DA68AA
:10CBD4001B691B0302218DF8001001920293074A7E
:10CBE40069460120FDF73AFA18B9002005B05DF84E
:10CBF40004FB7846FAF798FAF7E700BF22520020C0
:10CC040082890379012B0FD010B592001BB1022B3E
:10CC140010D0012007E000F10C01806812F05CFAEA
:10CC2400B0FA80F0400910BD83685888B0FA80F0EB
:10CC3400400970470368DB68447B0822811803EBD2
:10CC4400043012F049FAB0FA80F04009EBE7000032
:10CC540038B501460C48FCF729F80C4B5D6845B91A
:10CC640038BD2368002222609A68D8689047A5429C
:10CC7400F6D00648FDF78DFC04460028F1D178462D
:10CC8400FAF752FAEDE700BFFC50002010520020E2
:10CC94002DE9F041044617460D4611B9FFF7B0FFE0
:10CCA40058B10DB104F10C0726682379042B0DD873
:10CCB400DFE803F005464E0C5D000325F2E7A5B15D
:10CCC400B3691BB12A463946304698472E4B9C42DD
:10CCD40003D303F582739C4202D97846FAF724FA07
:10CCE400201FFFF7B5FFBDE8F081D4F80880B8F83D
:10CCF40000300BB3B8F8003008EB830323F47F62F1
:10CD040022F00F02934204D0B8F80220B2F5FE4F8D
:10CD140008D128F47F6828F00F0808F5805898F89F
:10CD240000304344B3605A8847F6FF739A42C7D031
:10CD34007846FAF7F9F9C3E77846FAF7F5F9D9E747
:10CD4400F369002BC2D02A46E18930469847BDE7F3
:10CD54003378012B07D1627B237B013B9A42B5D107
:10CD640002233370B2E77846FAF7DEF9F3E73DB908
:10CD740000233370336A002BA8D030469847A5E7C8
:10CD84007846FAF7D1F9F3E70851002000B583B0EB
:10CD940002A9002341F8043D82B20548FBF7DEFEF8
:10CDA40020B90198043003B05DF804FB0020FAE7D1
:10CDB400FC50002070B50446002536E01020FFF733
:10CDC400E5FF0646002860D002230371082303729E
:10CDD400042343721023C37283724573236903735C
:10CDE4004FF6FF73C3810460294B984203D303F5C4
:10CDF4008273984202D97846FAF796F936F8042CE9
:10CE0400311F2448FBF7D9FE0EE0002300E0002385
:10CE14004BB3E36833445B79AB4228D1E3681E44E7
:10CE2400327923699A4226D101352369AB4226D946
:10CE3400E0682E03304440F6FC710430FFF765FDD2
:10CE44000028BBD1E3689A199B5D083BDBB2F62B43
:10CE5400DDD85379FF2B04D01379FF2BD5D00123D0
:10CE6400D6E70023D4E77846FAF75EF9D1E77846A7
:10CE7400FAF75AF9D2E77846FAF756F9D4E7064BA7
:10CE84001868FEF7F5FB002070BD0420FCE700BF26
:10CE940008510020FC5000201852002038B50546E7
:10CEA400C3681C781C4400200DE07846FAF73CF96E
:10CEB4001FE024F47F6323F00F0303F580531A78F3
:10CEC400134420461C46EA68137951795B1A03F52A
:10CED4007F2303F6FF731B0303F5805313449C4223
:10CEE40015D262884FF6FF739A4210D02388002B24
:10CEF400DBD0238804EB830323F47F6222F00F0248
:10CF04009342D6D06288B2F5FE4FDAD1D1E738BD6C
:10CF140038B50446FFF7C2FFA06010B3428847F655
:10CF2400FF739A4222D00820FFF730FF0546F8B17C
:10CF34000323037104600F4B984203D303F58273F8
:10CF4400984202D97846FAF7EFF835F8042C291FED
:10CF54000948FBF732FE094B1868FEF789FB0020ED
:10CF640005E0E26813781344A36000E0002038BDB4
:10CF74000420FCE708510020FC5000201852002037
:10CF840070B505794379ED1A05F57F2505F6FF752A
:10CF94002D0305F5805505440478044400260DE06E
:10CFA4007846FAF7C1F819E024F47F6424F00F04FA
:10CFB40004F5805420780444A5421ED963884FF6B2
:10CFC400FF7293421DD047F6FF72934219D013B9F2
:10CFD400238806EB83062388002BE1D0238804EB07
:10CFE400830323F47F6222F00F029342DCD0628831
:10CFF400B2F5FE4FD8D01C46DEE77846FAF794F82F
:10D00400DCE7304670BD000070B584B005460068AA
:10D01400FFF744FF044600282FD06388002B30D14B
:10D024002E682388002B3ED0238804EB830323F44B
:10D034007F6222F00F02934203D06288B2F5FE4F62
:10D0440007D124F47F6323F00F0303F580531A7888
:10D054001344B3602B689968DA68137950791B1A02
:10D0640003F57F2303F6FF731B0303F58053134477
:10D0740099421CD3002004B070BD7846FAF754F8E6
:10D08400CBE701208DF8000001941F4B0393042388
:10D0940002931E4A6946FCF7E1FF0028C0D0784697
:10D0A400FAF742F8BCE77846FAF73EF8BCE723887B
:10D0B40033B3238804EB830323F47F6222F00F024B
:10D0C400934203D06288B2F5FE4F07D124F47F6403
:10D0D40024F00F0404F580542378234401208DF8B0
:10D0E400000001930A4B039304230293074A694601
:10D0F400FCF7B4FF0028BDD07846FAF715F8B9E775
:10D104007846FAF711F8D4E758F8030022520020C1
:10D1140060F8030008B50379042B13D8DFE803F0A3
:10D124000306090C0F00FFF743FC08BDFFF7DEFC04
:10D13400FBE7FFF715FDF8E7FFF766FFF5E7FFF7F5
:10D1440043FDF2E77846F9F7EFFF0020EDE7000032
:10D154002E4B1B78022B57D110B582B041E002A9A7
:10D16400002341F8043D2A48FBF758FD90B9019C7F
:10D17400201D284B1860284B01221A70FFF7ABFBC7
:10D1840058B30323214A1370626813706068FCF774
:10D194004FF922E0214B1B6803B19847012002B0EC
:10D1A40010BD1C4B1868FFF7B5FF1D4B187018B95C
:10D1B400194B02221A7010E0174B03221A700CE06C
:10D1C400144B1B68E3B1134B18688268144B19782D
:10D1D400FFF75EFD104B00221A700C4B1B78022BDC
:10D1E400DCD10D4B1B78032BF7D801A252F823F0A6
:10D1F40063D10200A7D10200A1D10200C5D102006F
:10D204007846F9F791FFDEE70120704720520020AD
:10D21400FC500020245200200C5200201C520020FC
:10D224002852002008B5074B1B88934200D008BD44
:10D23400054B1B78022BFAD1034B03221A70FFF71C
:10D2440087FFF4E7225200200C52002008B54FF467
:10D25400827210491048FBF701FC10490120FCF7C9
:10D26400EBFE0F48FEF7E4F90E4B186000230E4A5C
:10D2740013700E4A13800E48FDF764F9FCF7B0F8FA
:10D2840018B90C4B02221A7008BD0A4B03221A70FB
:10D29400FAE700BF08510020FC50002029D2020008
:10D2A40055D10200185200200C52002022520020B6
:10D2B400105200202052002038B505460820FFF700
:10D2C40065FDD0B1044604232B70037105600C4B3B
:10D2D400984203D303F58273984202D97846F9F74A
:10D2E40023FF34F8042C211F0648FBF766FC064B89
:10D2F4001868FEF7BDF9002038BD0420FCE700BF24
:10D3040008510020FC5000201852002038B50C466B
:10D314000546D0B1631E9BB247F6FE62934218D80D
:10D324002B78022B17D1EB68187819795A79891A56
:10D3340001F57F2101F6FF71090301F580512246B1
:10D344001944184400F0F6FC38BD7846F9F7ECFEB1
:10D35400E0E70020F8E70020F6E7F8B50E461546AA
:10D36400074680B33B78022B40F093807DB3FA6884
:10D37400137813449D42C0F08E80137951795B1A5F
:10D3840003F57F2303F6FF731B0303F58053134454
:10D394009D4200F282802B884BB32C8805EB8404D9
:10D3A40024F47F6323F00F039C4203D06B88B3F50E
:10D3B400FE4F0FD125F47F6525F00F0505F5805547
:10D3C4002C782C4406E07846F9F7AEFECAE7FC68F0
:10D3D40023781C44FD682B796A799B1A03F57F2313
:10D3E40003F6FF731B0303F580531D440FE07846D7
:10D3F400F9F79AFED1E77846F9F796FE1DE024F492
:10D404007F6424F00F0404F5805423781C44AC4258
:10D4140026D26288531E9BB247F6FE618B4207D820
:10D42400D6B1718833884A40134217D0002300E0F4
:10D434000023ABB92388002BDDD0238804EB8303BE
:10D4440023F47F6222F00F029342D8D06288B2F5AF
:10D45400FE4FD4D01C46DAE70123EAE70123E8E7CC
:10D46400AC421CD26288531E9BB247F6FE618B42CB
:10D4740007D856B1718833884A40134207D0002335
:10D4840000E000236BB12046F8BD0123FAE7012335
:10D49400F8E70024F7E70024F5E70024F3E7002485
:10D4A400F1E70024EFE770B50E461446054658B17F
:10D4B400731E9BB247F6FE6293420BD947F6FF7385
:10D4C4009E4205D0002306E07846F9F72DFEEFE7EB
:10D4D400012300E0012393B1802C14D82B78B3B13D
:10D4E40004F11000FFF752FC98B100220271C681CA
:10D4F4000334A4080134848140F80C5B70BD784681
:10D50400F9F712FEE8E77846F9F70EFEE6E70020A1
:10D51400F4E70020F2E7000010B504460F4B9842F0
:10D5240003D303F58273984202D97846F9F7FCFDD8
:10D534000C3C0A4B9C4203D303F582739C4202D9F0
:10D544007846F9F7F1FD34F8042C211F0448FBF761
:10D5540034FB044B1868FEF78BF810BD085100200B
:10D56400FC5000201852002070B50D46064658B1F4
:10D574006B1E9BB247F6FE6293420BD947F6FF73CC
:10D584009D4205D0002306E07846F9F7CDFDEFE78C
:10D59400012300E001230BB31020FFF7F7FB04463F
:10D5A40000B301230371C5814FF6FF7383810660C5
:10D5B4000D4B984203D303F58273984202D97846FF
:10D5C400F9F7B2FD34F8042C211F0848FBF7F5FAEB
:10D5D400074B1868FEF74CF8002070BD7846F9F741
:10D5E400A3FDD9E70420F8E708510020FC500020EF
:10D5F400185200202DE9F041C46894F8008004EB2F
:10D6040008068368B34202D80020BDE8F08137469B
:10D61400054634F80830B3B134F8084006EB840406
:10D6240024F47F6323F00F039C4203D07388B3F583
:10D63400FE4F1AD126F47F6626F00F0606F58056B3
:10D644003478344411E07846F9F76EFDE4E778461F
:10D65400F9F76AFD0FE024F47F6323F00F0303F569
:10D6640080531A78134427461C46AB68A34210D053
:10D674002388002BEBD0238804EB830323F47F62FD
:10D6840022F00F029342E6D06288B2F5FE4FEAD14F
:10D69400E1E77A88531E9BB247F6FE618B4201D9BB
:10D6A4000020B2E7EB6818783946184400F042FBD2
:10D6B40030B1874206D041882846FFF755FFA4E7DA
:10D6C4000020A2E70020A0E770B504460D46002321
:10D6D40003700B68C3F30B030BBB6B68FE2B22D8E0
:10D6E40029686A68AE68E868E16022616661A061E1
:10D6F40029696A69E16122620023A36063602046AC
:10D70400FFF723F9D0B12169E068FFF739FC6060C5
:10D714002046FFF7FDFB034648B1184670BD784626
:10D72400F9F702FDD9E77846F9F7FEFCD8E70223BA
:10D7340023702046FFF75EFF0346EEE701232370C4
:10D744002046FFF737FB03460028E6D1E26808329B
:10D75400A260E2E710B5044620B1A36833B12368A0
:10D7640043B110BD7846F9F7DFFCF6E77846F9F7E0
:10D77400DBFCF4E7246021460148FCF7EEFEF0E709
:10D784001052002008B50648FBF769FA08B10020DA
:10D7940008BDFBF745FE08B10020F9E70120F7E7D3
:10D7A400FC50002010B5C0B10446C368187819793C
:10D7B4005A79891A01F57F2101F6FF71090301F5F0
:10D7C400805147F6FF721944184400F0B3FAA06080
:10D7D40078B10223237000236360084B02221A707D
:10D7E40007490120FCF728FC064B1868FDF740FFA9
:10D7F40010BD7846F9F798FCEBE700BF20520020F3
:10D8040029D202001852002008B5FBF735FE08BDE6
:10D8140050B110B50446064B1B6813B17846F9F7AE
:10D8240083FC034B1C6010BD014B00221A6070473F
:10D834001C52002046DF70472DE9F04707460E468C
:10D844008589012411E0013B9BB2C11818F801201D
:10D854001EF803A082EA0A0209F80120002BF2D183
:10D86400A5EB0C05ADB20134A4B2BDB1230A43EA61
:10D874000423F3833046FFF7DDFFAC46102D28BFA9
:10D884004FF0100CD7F81890601E0001D7F80880EC
:10D8940006F1200E5FFA8CFC6346DFE7BDE8F087F3
:10D8A4002DE9F04780460F461646994600F11004CC
:10D8B40000F1200518E05246394604EB090011F046
:10D8C40041FC4E44B6B2103EB6B2574420E0013B90
:10D8D4009BB2EA5CE15C4A40E254002BF7D140463B
:10D8E400FFF7A8FF4FF00009A6B1C9F1100A564589
:10D8F400E1DA3246394604EB090011F023FC06EB69
:10D904000900C0F110020021204411F044FC00265B
:10D914001023E2E7BDE8F087F8B504460D46164645
:10D92400838A002B3BD0402294F82030023B03EB47
:10D93400D3735B10DB0003F03803134343F001039C
:10D944002B746268176850689168C5F81170C5F83F
:10D954001500C5F81910127B6A77A289130A43EAE5
:10D964000223EB832846FFF765FFA38A6BB1B3F567
:10D974007F4F16D2A28A130A43EA02232B82022380
:10D98400A28A21692846FFF78BFFA2896AB994F815
:10D99400202005F12001304611F0D4FBF8BD00220F
:10D9A400C2E77846F9F7C0FBE4E70023A1682846FC
:10D9B400FFF776FFEBE730B58DB0054603686C469C
:10D9C400186859689A68DB680FC4EA69694628468A
:10D9D400FFF7A2FFEC696B6801228DF8102018682C
:10D9E40059689A68CDF81100CDF81510CDF81920B2
:10D9F4001B7B8DF81D300023ADF81E306846FFF701
:10DA040019FF95F8203008E0013B9BB2E25C0CA9B9
:10DA1400194411F8101C4A40E254002BF4D1694611
:10DA24002846FFF709FF0DB030BD2DE9F0418CB059
:10DA340000AF04460E4603683D46186859689A6864
:10DA4400DB680FC5A38933BBD4F80880A369A3603E
:10DA540094F82030073303F4FC73ADEB030D6D46EB
:10DA64006A4639462046FFF757FF636801223A7435
:10DA7400186859689A68C7F81100C7F81510C7F8EC
:10DA840019201B7B7B770023FB833846FFF7D2FEEC
:10DA940094F820301EE0636801223A7418685968CB
:10DAA4009A68C7F81100C7F81510C7F819201B7B2E
:10DAB4007B770023FB8339462046FFF7BDFEC3E78F
:10DAC400013B9BB2EA5C07F13001194411F8101CC8
:10DAD4004A40EA54002BF3D1C4F8088094F820207B
:10DAE400E169284611F0F8FAB0FA80F04009307084
:10DAF4003037BD46BDE8F08100231F2B28D870B411
:10DB0400164603EB4214134D05EBC404A48834B148
:10DB1400844212D001331F2BF2D904200BE003EB13
:10DB2400461355F8334061F3170445F8334005EBC9
:10DB3400C3039880002070BC7047064A03EB461369
:10DB440052F8330061F3170042F833000020F2E783
:10DB5400042070472C52002000231F2B1AD870B4C5
:10DB640003EB42140C4D05EBC404A488844204D096
:10DB740001331F2BF4D9002008E003EB421355F8BE
:10DB84003330C3F317038B4202D2002070BC7047BA
:10DB94000120FBE7002070472C52002008B54FF409
:10DBA40000720021034811F0F6FA034B00221A70A8
:10DBB40008BD00BF2C5200202952002008B5FFF7F1
:10DBC400EDFF08BD2DE9F041D8B1E2B1EBB1FF2979
:10DBD4001DD01C2B1DD81E4690460C469F1CFFB220
:10DBE400791C07F029FD054640B147742B23837443
:10DBF400C47432464146143011F0A4FA2846BDE8F4
:10DC0400F0810025FAE70025F8E70025F6E700256E
:10DC1400F4E70025F2E700002DE9F04F85B004AFEA
:10DC24000C461646054630B3002C69D0611EC9B2B5
:10DC34002A7822B3012A28D0364B1B6813F4807F3C
:10DC440003D0354B1B68012B25DC324B1B6813F4C6
:10DC5400807F5AD0304B1B68032B58DDEB46A0461F
:10DC64006300083303F47E73ADEB030D0DF110096B
:10DC7400CE4600232EE07846F9F756FAD4E732462A
:10DC8400681C0CF0E1FD00203BE03246681C00F00B
:10DC9400B5FD002035E0214BD3F804350192204A2C
:10DCA40000926D221F490220FEF7F8FDCDE76A1CA1
:10DCB400D25C4FEA121A59001B4E306810F80A0061
:10DCC4000EF8130002F00F0201313068825C0EF886
:10DCD400012001334345EAD3002309F814300F4BE4
:10DCE400D3F80435CDF80890104A0192104A0092F6
:10DCF4006E220C490420FEF7D1FDDD460B2000E026
:10DD040009200437BD46BDE8F08F0B20F9E70B204E
:10DD1400F7E700BF383300203433002000B0004060
:10DD240094F803008BF803003C330020BCF8030094
:10DD340038F40300F8B506460D461746884201D864
:10DD4400344613E07846F9F7EFF9F9E77846F9F73E
:10DD5400EBF921E024F47F6424F00F0404F58054EB
:10DD640023781C44A5422AD9A6422BD26288BA42FF
:10DD740026D024F47F6323F00F0303F58053AB42D2
:10DD840007D3B2F5FE4F16D0238804EB8303AB42CE
:10DD940013D22388002BD9D0238804EB830323F4E4
:10DDA4007F6222F00F029342D4D06288B2F5FE4F14
:10DDB400D0D01C46D6E7002402E0002400E0002472
:10DDC4002046F8BD0024FBE7014B1860704700BFF4
:10DDD4005454002070B50E46054678B196B12B78A0
:10DDE400012B13D8234B1B6AA3B96B681D2B15D8C1
:10DDF4002B78012B16D0204B1C681CE07846F9F7D1
:10DE040093F9EBE77846F9F78FF9E8E77846F9F7FD
:10DE14008BF9E7E77846F9F787F9E6E77846F9F703
:10DE240083F9E5E7EB68B3F1FF3FE4D07846F9F70F
:10DE34007BF9E0E7246894B154F8083C1B68294650
:10DE4400A4F1080098470028F4D114F8042C012305
:10DE540003FA02F207490B6A13430B62EAE7054B24
:10DE64001B6A23B16A68034B03F8012B3360014B2F
:10DE7400186A70BD305400205854002010B5114B5E
:10DE84001B6A13B1104B1C6804E07846F9F74CF98F
:10DE9400F8E724688CB1A4F108000A4B1A6A14F854
:10DEA400041C01238B401A42F3D054F8083C5B68ED
:10DEB400044911F8012B9847EBE7024B00221A6240
:10DEC40010BD00BF305400205854002010B50F4B33
:10DED4001B6A13B10E4B1C6804E07846F9F724F969
:10DEE400F8E7246874B1A4F10800084B1A6A14F81E
:10DEF400041C01238B401A42F3D054F8083C9B685D
:10DF04009847EEE7014B00221A6210BD30540020FE
:10DF1400585400202DE9F0410D4617469846064610
:10DF240048B1074B1C6824B143463A463179284628
:10DF3400A047BDE8F0817846F9F7F6F8F1E700BFAD
:10DF44005454002070B50C4616460546C0B1DCB1E9
:10DF5400F6B1236803B3636813B3A36823B3164B02
:10DF64001B781F2B24D82C60134A1378591C11706A
:10DF74002B716E7105F108011048FEF7CDFB70BDE1
:10DF84007846F9F7D1F8E2E77846F9F7CDF8DFE714
:10DF94007846F9F7C9F8DCE77846F9F7C5F8DAE71F
:10DFA4007846F9F7C1F8D8E77846F9F7BDF8D6E727
:10DFB4007846F9F7B9F8D6E72C54002058540020D5
:10DFC400F8B504460F4616461D469B68ABB10A23B6
:10DFD400237000232373AB88E3812B681B8863823F
:10DFE4002B681888FCF7D6F82074AB68A3616760C7
:10DFF400A6602B681B7B2377F8BD7846F9F794F865
:10E00400E5E710B58CB0044603685A680AB9DB89A1
:10E01400EBB12368DB8913F0010F1CD100222368C4
:10E024001B7B03F07F038DF8083000238DF8093043
:10E034008DF80A202346032202A904A8FFF7C0FF93
:10E044006FF0020104A8FAF740F90CB010BD78464D
:10E05400F9F76AF8DDE769464FF4C870FCF7B1FFD9
:10E0640018B9019A02F00102D9E77846F9F75CF889
:10E07400F7E700000378012B00D0704700B585B0A6
:10E084001E4B1B6873B11D4B1B6801A89847A8B9A8
:10E094001B4B1B7863B1019B1A883AB15B6833B19F
:10E0A400012304E07846F9F73FF8ECE7002383B94D
:10E0B400144B1B7813B1019B1B88D3B91248FAF790
:10E0C40027FC00230E4A13700E4A137005B05DF846
:10E0D40004FB01A8FFF795FF0028E9D10B4B1B684F
:10E0E4001BB10A4B1B689847E2E77846F9F71CF81E
:10E0F400F7E701A8FFF785FFE0E700BF80540020A1
:10E1040069540020685400205C5400207C54002092
:10E114000B6813B1013B0B60704710B50C46034804
:10E12400FCF7D6FC0023236010BD00BFA0540020E0
:10E1340010B584B004462C4B1B68EBB12A4B1B680A
:10E1440001A8984700284BD1284B1B68C3B1274925
:10E154000A6801988368934228BF1346B3F5E16FB8
:10E1640094BFD31AA2F5E1630B607BB903885BB15A
:10E17400436853B1012308E07846F8F7D5FFDDE79B
:10E184007846F8F7D1FFE2E7002383B9019B5B6887
:10E1940013B3164B1B68B3F5E16F1BD2144901FB93
:10E1A40003F121441348FCF7C3FC04B010BD01A8DB
:10E1B400FFF727FF28B9104B1B683BB10E4B1B68B8
:10E1C4009847019B9A68094B1A60DFE77846F8F78D
:10E1D400ABFFF3E70949E4E70648FCF779FCE4E719
:10E1E4000448FCF775FCE0E78054002084540020C8
:10E1F40040420F00885400207C54002000D2496B18
:10E2040003780A2B00D07047C389234A12889342AB
:10E21400F9D1418A204A52889142F4D18268032A72
:10E22400F1D11D4A9268002AEDD000B58DB01A4A8A
:10E234005268B2F5803F02D2013217494A60052282
:10E244008DF8042041680A7802F07F028DF80820D6
:10E254000A7802F07F02007F121AD2B20132D2B2DF
:10E264008DF80920897801F00F01ADF80A10ADF896
:10E274000C3093B2084A9289934201D2064A9381A0
:10E28400054AD289934201D9034AD38101A8FAF7F6
:10E2940007FB0DB05DF804FB6C54002038B503682F
:10E2A4009B68094C44F8043B03689D68B5F5E16F2D
:10E2B40028BF4FF4E165FCF7D7FC044901FB0501D5
:10E2C4002046FCF735FC38BD8454002040420F0042
:10E2D40010B584B004460D4B1B6863B10B4B1B682F
:10E2E40001A8984728B9019BDA89224201D01B88EA
:10E2F4002BB904B010BD7846F8F716FFEEE70448D2
:10E30400FAF7F6FA034B01221A70F2E78054002060
:10E314005C5400206854002008B5134B1B78DBB90B
:10E3240001211248FAF774FAD0B90022104B1A707E
:10E33400104B1149D960114B1A605A605A61104A46
:10E344009A60104A1A61104ADA60104B104A1A6037
:10E35400054B01221A7008BD7846F8F7E5FEDFE7A1
:10E364007846F8F7E1FEE0E76A540020D0F80300AD
:10E37400695400208454002035E10200A054002098
:10E3840015E102007454002040420F005C54002048
:10E3940079E0020070B582B0044630B301A90DF1F2
:10E3A400060006F023FFA368B3F5803F3FD820881A
:10E3B400FBF7F0FE012804D02088FBF7EBFE0028D1
:10E3C40038D16088FBF7E6FE98B9A3681BB12288B0
:10E3D4000AB16188C9B9184B00241C805C809C6018
:10E3E4001648FCF775FB204622E07846F8F79CFEB9
:10E3F400D4E76088FBF7CEFE0328E6D06288BDF838
:10E4040006309A42E1D0072012E00B4C2280618052
:10E41400A3600A4DEE68FCF727FC31182846FCF788
:10E4240087FB7F23A3810020E081606000E0072058
:10E4340002B070BD0720FBE76C540020A0540020FC
:10E44400004870476C54002038B50C46054628B186
:10E4540044B1064B1D60064B1C6038BD7846F8F786
:10E4640063FEF5E77846F8F75FFEF2E78054002094
:10E474007C54002000B585B0114B1B688BB1104B48
:10E484001B6801A8984748B9019B1A881AB15A68B1
:10E494000AB19B684BB90B48FCF71AFB05B05DF851
:10E4A40004FB7846F8F740FEE9E701A8FFF7F6FE1B
:10E4B4000548FAF71DFA054B01221A70EEE700BF72
:10E4C40080540020885400205C54002069540020AB
:10E4D40030B585B00D4614466B460D2201462846DC
:10E4E400FDF7B7F96B4603CB2060616005B030BD22
:10E4F40030B58DB004460DF12F025449002006F0CA
:10E50400ABFD1BE0131B21E030F813100A44013368
:10E51400012BF9D9013202EB820252000123012BB3
:10E524001BD94A4B1B685B680021198095421ED297
:10E534000DF12F024549002006F08EFD434B1B6868
:10E54400002B66D058684268A31ADBD4404DA5FB63
:10E5540003239D0C00231A46DAE73C4909684968FD
:10E56400581E31F8100021F813000133D7E7FBF7E8
:10E574007BFB0546FBF798FB9DF82F30022B4AD016
:10E58400324A11680831022B14BF002201229DF87F
:10E59400183062F30003012814BF0022012262F341
:10E5A40041036FF387038DF818300B4653F8102F8F
:10E5B4005B68CDF81920CDF81D302B0203F47F03DE
:10E5C40043EA05632A0A02F47F42134343EA1563CC
:10E5D400CDF821300DF1250206A8FFF779FF1523A8
:10E5E40006AA01211B48FFF7EDFA014688B1012371
:10E5F4000371184807F05EF8174B1B6813F0020FFD
:10E6040003D0164B1B68042B09DC104B1B685B689A
:10E614005C600DB030BD0D4A11683031B3E7104B6A
:10E62400D3F80435094A1268117E507E957ED27E55
:10E6340004920395029001910A4A00924FF4807269
:10E6440009490520FEF72AF9DFE700BFB455002089
:10E6540083DE1B43B85400203833002034330020B9
:10E6640000B000400CF90300FFF8030008B5FCF704
:10E67400FBFAFFF73DFF08BD08B5FFF739FF08BDFA
:10E6840030B583B005460C4608220131103010F035
:10E6940023FD10B1002003B030BD6A462946204650
:10E6A400FFF716FF082204F10D01684610F014FD6F
:10E6B400B0FA80F04009EEE730B583B0194B01227F
:10E6C4001A700023184A1360184C194AE260194A58
:10E6D400A260236104210DEB0100FCF717FCFCF799
:10E6E400C3FAE2680199B1FBF2F302FB1313184475
:10E6F4006060114D3423114A1149284607F0B8F8D7
:10E704004FF47A71284607F02FF8284606F072FF76
:10E714002046FCF7ABF90B4A04210B48FDF740F9FE
:10E7240003B030BD98550020B45500209C550020FE
:10E73400809698007DE60200B854002054550020CD
:10E7440071E602008855002024F9030010B5044640
:10E754000A4B1B7803B920B903B15CB1074B1C7099
:10E7640010BDFCF781FA064BD96801441846FCF742
:10E77400DFF9F3E70248FCF7ABF9EFE7985500201F
:10E784009C550020014B1878704700BF9855002015
:10E79400F8B5069E70B3074676B30D4630460121A0
:10E7A40000F8011B747863F300048A4214BF00224A
:10E7B400012262F341046FF3870474703B4653F8FB
:10E7C400102F5B68C0F80120C0F805302B0203F459
:10E7D4007F0343EA0563290A01F47F410B4343EABB
:10E7E4001563C0F8093006F10E023946FFF770FED2
:10E7F4000020F8BD0E20FCE70E20FAE7F0B58FB03C
:10E804001746054648B100230C936E1C0DF13702E0
:10E814000CA9304606F020FC30E07846F8F784FC7A
:10E82400F1E77846F8F780FC2DE09DF83730FBB12E
:10E8340029460C983030FFF723FFC8B10C993031CA
:10E8440037E004238DF804302A4612F80D3BC3F355
:10E8540040008DF81C00C3F300038DF81D300694AE
:10E864000C9B029303910497059201A8FAF718F8F8
:10E874000DF137020CA9304606F0EEFB0C9B13B3E6
:10E884005B68002BCDD0D5F80940230203F47F0345
:10E8940043EA0463220A02F47F42134343EA146402
:10E8A40029460C980830FFF7EBFE0028BDD00C99E0
:10E8B40008310C9B5A6813884FF6FF708342C0D00E
:10E8C40001331380BDE70FB0F0BD2DE9F041804660
:10E8D40007683E68FF25002405E016F82430FF2B66
:10E8E4000ED00134E4B23B79A3420BD9FF2DF4D00E
:10E8F40016F92430002BF0DA7846F8F715FCECE72B
:10E904002546EEE7FF2D02D0AB4200D8FF2588F85C
:10E914000450BDE8F0810000F0B585B005460C4612
:10E9240017464B78FF2B27D003689E6806B33946F9
:10E934006078B0470646F8B93D4B1B6813F4803F36
:10E944003FD03C4B1B68032B3BDD3B4BD3F80435DA
:10E954002A689169607851F8201002911269019235
:10E96400364A0092AB2236490420FDF797FF28E08F
:10E974007846F8F7D9FBDAE7A378FF2B0ED02B689B
:10E98400DE680EB32A4B1B6813F4803F03D0294B77
:10E994001B68032B1CDC3946A078B047E378FF2BB7
:10E9A40044D0AB79DBB2012B25D1214B1B6813F486
:10E9B400803F03D01F4B1B68032B20DCE3786B7173
:10E9C4000126304605B0F0BD7846F8F7ADFBD9E72F
:10E9D400194BD3F804352A685169A07851F82010EE
:10E9E400029112690192174A0092BA221449042032
:10E9F400FDF754FFCFE77846F8F796FBD5E70E4BC3
:10EA0400D3F804352A68116A6879E67851F82660E3
:10EA1400039651F820100291126901920A4A009259
:10EA2400C92207490420FDF739FFC7E70126C8E7D3
:10EA3400383300203433002000B0004074F9030060
:10EA44006BF9030080F903008CF903002DE9F04110
:10EA540007460E469046427901680C680D7904EB2E
:10EA64008505194613B9D2B203791BB904EB8104A5
:10EA7400043410E0AC42FBD2237883F08003934249
:10EA8400F6D00434F6E7424621463846FFF744FF01
:10EA9400034658B90434AC4207D22378B342F2D0C7
:10EAA40013F0800FF6D0002300E000231846BDE8E1
:10EAB400F081000030B583B00D46044698B1B5B17D
:10EAC40025606B7963710023A371114B1B6813F4E8
:10EAD400803F03D00F4B1B68032B0CDC2046FFF751
:10EAE400F4FE03B030BD7846F8F71EFBE7E778463E
:10EAF400F8F71AFBE4E7084BD3F804352A690192C6
:10EB0400064A0092DE2206490420FDF7C7FEE5E727
:10EB1400383300203433002000B0004038F90300BB
:10EB24006BF9030070B584B00D461646044608B36D
:10EB34001B4B1B6813F4803F03D01A4B1B68032B39
:10EB44001CDCA3790133DBB2A371002332462946CE
:10EB54002046FFF77BFF38B92379FF2B04D03246D8
:10EB640029462046FFF772FFA379013BDBB2A3716C
:10EB740004B070BD7846F8F7D7FAD9E70A4BD3F852
:10EB840004352268D16951F8251002911269019265
:10EB9400064A0092E92206490420FDF77FFED0E7E9
:10EBA400383300203433002000B000402CF9030037
:10EBB4006BF903008079003018BF01207047000012
:10EBC40010B50D4B834202D07846F8F7ADFA0B4BE3
:10EBD4005B686BB1094C237803EB83035A01084843
:10EBE40010446168043006F0AFFD0023636010BD7B
:10EBF4007846F8F799FAEDE7B85500200457002055
:10EC0400C4550020F8B50F461646134B834202D074
:10EC14007846F8F789FA114B5B68C3B10F4D6C68FD
:10EC24002A23A374731C63743246394604F1130017
:10EC340010F088FA2B7803EB83035A010848104438
:10EC44002146043006F036FD00236B60F8BD78469B
:10EC5400F8F76AFAE2E700BFB8550020045700202D
:10EC6400C455002010B50C46144B834202D078469C
:10EC7400F8F75AFA124B5B6813B17846F8F754FA6E
:10EC84002378616803EB83035A010E481044023170
:10EC9400043006F0D1FC0A4B586068B1E3680360A5
:10ECA400237803EB83035A01064B9B5803712278A4
:10ECB400034B1A70002010BD0220FCE7B855002059
:10ECC40004570020C455002008B5064BC01A801014
:10ECD400054B03FB00F00B46C1B20448FFF71AF9D9
:10ECE40008BD00BFC8550020976FF996B85500209D
:10ECF40070B5104C0126254645F8046B4FF480731B
:10ED04000D4A0E49284606F0B3FD284606F072FC6B
:10ED1400C4F8A060A4348023094A0021204606F0E8
:10ED2400A7FD204606F066FC324606490648FFF772
:10ED340009F970BDC45500200C570020CDEC020029
:10ED44000C580020A0F90300B855002038B504463B
:10ED54000D46012806D84DB104EB84046301054A2D
:10ED6400D55038BD7846F8F7DFF9F4E77846F8F778
:10ED7400DBF9F1E7C455002010B50446012802D997
:10ED84007846F8F7D1F904EB84046301014AD05CB6
:10ED940010BD00BFC455002038B504460D460128F7
:10EDA40002D97846F8F7C0F904EB840463010348F8
:10EDB40018442946043006F0D7FC38BDC455002059
:10EDC40010B50446012802D97846F8F7ADF904EBEA
:10EDD40084046201034B1344586F034BA3FB0030BC
:10EDE400800910BDC4550020D34D621038B50446C7
:10EDF4000D46012802D97846F8F796F904EB840405
:10EE04006301034818442946043006F0F1FC38BD78
:10EE1400C455002008B50020FBF7DEFB08BD08B58B
:10EE240003780D2B00D008BDFFF7F4FFFBE770B5A6
:10EE340082B004460E46C38AADF800300123ADF813
:10EE44000230684605F024F8054610B1284602B0A1
:10EE540070BD0DF106022146208A05F021FB05460E
:10EE64000028F3D101AB3246BDF80610E08A05F064
:10EE740097FD05460028E9D1217E01F00101D4F86F
:10EE84001200FAF717FF48B9BDF804000FF0B0FC00
:10EE940005460028DAD102F019F9D7E77846F8F7E1
:10EEA40043F9F1E708B502F0EFFD04F077FFFAF754
:10EEB40045FC08BD00B583B001A805F02BF8BDF8EA
:10EEC4000400003018BF012003B05DF804FB00000B
:10EED40070B582B0002831D004460D46FBF740FAE5
:10EEE400064610B1304602B070BD04F0B3FF02F024
:10EEF400D3FD20690FF044FC06460028F2D1636973
:10EF0400A269217F01910092592200210C480FF03F
:10EF1400EDFE06460028E5D1236A03B1984704F0C4
:10EF24007BFE02F0DDFBFFF7C5FF044618B9002D98
:10EF3400D8D02C70D6E701F055FAF8E70E26D1E7C1
:10EF44008C58002008B5FFF7B5FF10B9FBF776FA27
:10EF540008BD01F0F3FAF9E708B5FEF713FC18B998
:10EF64000348FBF7D1FA08BDFFF754FFFBE700BFE6
:10EF74004433002076DF70477FDF70478FDF7047B0
:10EF840090DF7047A8DF7047AADF7047AEDF704795
:10EF9400B1DF7047B5DF704710B431B983B2934223
:10EFA40008D808465DF8044B7047401A904203DCC9
:10EFB4000320F7E70120F5E70220F3E7002313B16C
:10EFC4004FF6FF7070470A494FF4A67202FB031212
:10EFD400918B4FF6FF72914201D00133EFE7044960
:10EFE4004FF4A67202FB0312908398B2704700BFDD
:10EFF400E8580020002313B14FF6FF70704706490C
:10F004004FF4A67202FB0312928B824201D00133A9
:10F01400F1E798B2704700BFE858002090F8320139
:10F02400003018BF0120704790F8EC000B79013BC9
:10F03400984214BF002001207047032907D890F894
:10F0440031318B4205D0FF2B05D0002070470020C2
:10F054007047012070470120704708B508881321C4
:10F06400FFF788FF20B1082802D07846F8F75CF84B
:10F0740008BD000070B5044686883046FFF7BAFF25
:10F084004FF6FF73984216D00546E488162C05D92E
:10F09400442C11D8452C28BF452400E017242146D0
:10F0A4003046FFF777FF48B9033C064B4FF4A6728E
:10F0B40002FB0535EC8370BD4524F0E77846F8F78C
:10F0C40033F8F1E7E858002030B585B08088FFF7C1
:10F0D40075FF4FF6FF73984219D004460D4D4FF457
:10F0E400A67000FB04F000F12001294418302844E4
:10F0F400D8220C310830F9F7B1FC03238DF8003025
:10F104008DF80140AB69D5F868116846984705B099
:10F1140030BD00BFE8580020D0F8E81051B110B558
:10F1240004460430F9F7C2FD0023C4F8E83084F83B
:10F13400EC3010BD704710B5044600F59A70FBF72B
:10F14400C7FC002384F83231FF2384F8313110BD29
:10F15400F8B50646B8B90E4C4FF4A67505FB06F58E
:10F1640005F118062644371D3846FFF7E4FF3846F4
:10F17400FFF7D2FF06F10800F9F7C7FC2C444FF65D
:10F18400FF73A383F8BD7846F7F7CEFFE3E700BF2C
:10F19400E858002010B584B08088FFF72BFF4FF6A5
:10F1A400FF7398420DD00446FFF7D2FF04238DF875
:10F1B40000308DF80140044B9A69D3F86811684611
:10F1C400904704B010BD00BFE858002010B50446B5
:10F1D400FBF74AFD0349014404F59A70FBF7A8FCC8
:10F1E40010BD00BF002D31012DE9F0478EB08946D6
:10F1F40016460546002867D0002965D00027002F51
:10F2040066D04F4A28681060AB889380C2F8189083
:10F214002B88ADF8343001208DF8360006320DA964
:10F22400FFF7B0FE00287ED1AB88ADF83430002360
:10F2340006930793089309930A930B930C93042260
:10F244008DF818200122114662F307118DF814106D
:10F25400114662F307118DF81510924042F0010235
:10F264008DF816200293039304930DAB009305AB22
:10F2740001934223ADF80C30314800F110036A4683
:10F2840006A9C088FFF780FE002850D16B88ADF82E
:10F294003430002306930793089309930A930B933E
:10F2A4000C9310238DF81830254800F108036A46A2
:10F2B40006A9C088FFF768FE00283CD1204BC3F89C
:10F2C40068610EB0BDE8F0877846F7F72DFF95E743
:10F2D4001B4B4FF4A67404FB07F41A191421D183B1
:10F2E400FF2182F84D111749C2F8581104F118088A
:10F2F400984408F10401C2F860114FF6FF7191833C
:10F304002034234403F10C044FF0D80A5246002160
:10F3140020460FF040FF5246214608F10800F9F755
:10F324009DFB01376BE77846F7F7FEFE7CE77846EE
:10F33400F7F7FAFEAAE77846F7F7F6FEBEE700BF4E
:10F34400E85800205FF00200F0B583B00D46144683
:10F354001E46074610BB032D24D8422C26D81E4A2D
:10F364004FF4A67303FB07239A8B4FF6FF739A425D
:10F3740030D0A21D02A9002341F8043D4FF4A67029
:10F3840000FB07F01830144B184492B20830F9F718
:10F39400E5FB78B1042818D1002014E07846F7F78B
:10F3A400C3FED8E77846F7F7BFFED6E77846F7F707
:10F3B400BBFED4E70198466001340472437A65F3D6
:10F3C400050343720A3003B0F0BD7846F7F7ACFE8C
:10F3D4000020F8E70020F6E7E858002038B5044696
:10F3E4000D46B1B1CCB9114A4FF4A67303FB042303
:10F3F4009A8B4FF6FF739A4213D04FF4A67000FB1A
:10F4040004F01830094B1844691F0830F9F74EFC12
:10F4140038BD7846F7F788FEE4E77846F7F784FEC8
:10F42400E1E77846F7F780FEE7E700BFE8580020F9
:10F4340070B5064680B90A4C4FF4A67505FB06F56F
:10F4440005F5A47020440830FBF742FB2C4413213B
:10F45400A08BFFF78FFD70BD7846F7F765FEEAE7EE
:10F46400E85800202DE9F04786B00546474A4FF496
:10F47400A67303FB0023D3F8046116B3434A4FF485
:10F48400A67303FB052393F80821337A9A421CD20E
:10F49400347A3E4A4FF4A67303FB052393F808A17C
:10F4A400B3F81E904A4651462046FFF775FD804644
:10F4B400471EFFB2012F59D958B1032809D000249F
:10F4C4000AE07846F7F730FED8E77846F7F72CFEDF
:10F4D400DEE7A4EB0A04A4B2A14549D32B494FF4B7
:10F4E400A67202FB051292F80801331D034403F1CE
:10F4F400050C587968F3871058710023CDF80A3049
:10F50400ADF80E30ADF806400B89ADF80830CDF8F3
:10F5140014C00DF10603049301238DF80A3002A9E7
:10F52400908BFFF733FD082826D013281BD018B979
:10F53400BDF80630A34202D07846F7F7F5FD134A2A
:10F544004FF4A67303FB052393F808311C44E4B27B
:10F55400013CE4B2012F13D90C4B4FF4A67202FB09
:10F56400053585F8084106B0BDE8F0874C46B3E799
:10F574007846F7F7D9FDB1E72846FFF759FFF2E7D8
:10F5840033445B7A26447372E6E700BFE8580020F0
:10F5940070B505460E4601B31DBB254A4FF4A6734C
:10F5A40003FB05239A8B4FF6FF739A423ED04FF428
:10F5B400A67404FB05F404F118031D4C1C44083420
:10F5C40036F80A2CA6F10A012046F9F7F6FA204685
:10F5D400F9F745FB48B9002070BD7846F7F7A4FD5C
:10F5E400DAE77846F7F7A0FDD7E74FF4A67101FBF9
:10F5F40005F1F8310E4B19440C312046F9F70EFB96
:10F6040060B90B4A4FF4A67303FB0523D3F8043106
:10F6140043B12846FFF726FF0020DDE77846F7F7D9
:10F6240083FDEEE77846F7F77FFDF2E70820D3E79E
:10F63400E858002070B584B0FFF7DCFC4FF6FF7388
:10F6440098425BD005462E4B4FF4A67202FB00F2A3
:10F6540002F118041C4404341344D3F80461002E4A
:10F664003DD0311D2046FFF7DFFC002843D0204663
:10F67400FFF752FD01238DF800308DF80150737AA5
:10F68400C3F305038DF80830736801931C4CA36918
:10F69400D4F86811684698474FF4A67303FB05F342
:10F6A40018331C4408342046F9F7D9FA30B34FF420
:10F6B400A67101FB05F1F831114B19440C312046B8
:10F6C400F9F7ACFA78B90E4A4FF4A67303FB052395
:10F6D400D3F804315BB12846FFF7C4FE0EE0784648
:10F6E400F7F722FDBDE77846F7F71EFDEBE778460E
:10F6F400F7F71AFDEFE72846FFF7B4FE04B070BD34
:10F70400E85800202DE9F04784B004460D464FF434
:10F71400A67303FB00F318332C490B441E1D013A56
:10F7240097B22B789B09022B04D0032B1ED0FFF732
:10F734007FFE18E03046FFF749FD24484FF4A673D6
:10F7440003FB04F4061996F84E311C4404F5847442
:10F7540020443A46691C04300FF0F4FC96F84E211C
:10F76400174486F84E7104B0BDE8F087DFF85C906A
:10F774004FF4A67808FB00F809EB080A9AF84E0142
:10F78400404400F5847048443A46691C04300FF044
:10F79400D9FC00238DF800308DF801409AF84D31E2
:10F7A4008DF8043008F584734B44043302939AF8BB
:10F7B4004E211744ADF80C70D9F81830D9F86811F7
:10F7C400684698473046FFF7B6FCCCE7E858002077
:10F7D400F0B585B005460C464FF4A67000FB05F065
:10F7E40018301E4B1844013A96B20B789B0906D088
:10F7F4000430012B19D02846FFF71AFE13E000232A
:10F804008DF800308DF8015014F8013BC3F3050363
:10F814008DF804300294ADF80C60104B9A69D3F85B
:10F8240068116846904705B0F0BDFFF7CFFC0B4F59
:10F834004FF4A67303FB05F505F58470384432468E
:10F84400611C04300FF07EFC2378C3F305032F44BE
:10F8540087F84D3187F84E61E5E700BFE85800208E
:10F86400F0B585B004468088FFF7C4FB4FF6FF73FC
:10F87400984209D00546E3882B4A9289934205D0E1
:10F88400294A128A934214D005B0F0BD228A022A72
:10F89400F6D1A37C13F0010FF6D005238DF80030C8
:10F8A4008DF80100204B9A69D3F868116846904797
:10F8B400EAE7278A012F0CD91B4A4FF4A67303FBEE
:10F8C400052393F84E31C3F142039F421ED900230E
:10F8D40000E000231BB34FF4A67606FB05F606F101
:10F8E4001803114E1E440436A17C01F03F0130463A
:10F8F400FFF7A3FB98B13046FFF790FB40B13A46BF
:10F9040004F112012846FFF7FDFEBDE70123E1E7FC
:10F914003A4604F112012846FFF75AFFB4E7284695
:10F92400FFF786FDB0E700BFE858002000B585B0BA
:10F934000388103B472B27D8DFE803F02429265FF0
:10F94400262626262626262626262626266B2652E2
:10F9540026262C262626262626262626262626263D
:10F964002626262626262626262626262626262633
:10F974002626262626262626262626263C264626ED
:10F98400267A263FFFF7A0FB05B05DF804FBFFF7DE
:10F9940001FCF9E7037A012BF6D102238DF800303C
:10F9A40083888DF80130244B9A69D3F8681168462E
:10F9B4009047E9E7FFF754FFE6E78088FFF73AFE50
:10F9C4001E4B01221A70DFE700231A46194680886D
:10F9D400FFF7DEFA0028D7D07846F7F7A5FBD3E780
:10F9E40000220092019269468088FFF7C9FA002834
:10F9F400CAD07846F7F798FBC6E700231A46852154
:10FA04008088FFF7B9FA0028BED07846F7F78CFB58
:10FA1400BAE700238DF800308DF8013069468088FC
:10FA2400FFF7ACFA0028AFD07846F7F77DFBABE7D9
:10FA3400FFF720FBA8E700BFE8580020545A002035
:10FA44001130704710B50446C36C63B10848201ADE
:10FA54008010084B03FB00F0E16C80B2FFF7BEFCA2
:10FA64000023E36410BD7846F7F75EFBEEE700BFC2
:10FA7400DC5A0020A737BDE910B5044620B1A4F133
:10FA84005000FFF7DFFF10BD7846F7F74DFBF6E7B0
:10FA940038B50546C36C73B10B4C2C1BA3100B4C2F
:10FAA40004FB03F4A4B2E96C2046FFF771FD30B9FE
:10FAB4000023EB6438BD7846F7F736FBECE7E96CD6
:10FAC4002046FFF78BFCF3E7DC5A0020A737BDE99B
:10FAD400F8B50D461746044678B171B1A4F1500645
:10FAE40054F8043C6BB13A46294654F8040C0FF020
:10FAF40029FB3046FFF7CCFFF8BD7846F7F714FB37
:10FB0400ECE77846F7F710FBEDE70000F8B504469C
:10FB14000D4616461F46C36C13B17846F7F704FB2F
:10FB24000848201A8010084B03FB00F03B46B2B291
:10FB3400294680B2FFF708FCE06408B10020F8BD54
:10FB44000420FCE7DC5A0020A737BDE970B50D4658
:10FB5400044638B131B1A4F1500614F80C3C2BB969
:10FB6400012070BD7846F7F7DFFAF4E7AB685988EF
:10FB7400304600F006FE08B90120F2E7EB686A6837
:10FB840000213046FFF7C2FF0028EAD00220E8E750
:10FB940010B582B00C4C0DF1070204F11C010020D9
:10FBA40005F05AFAE3690BB102B010BD0DF107027A
:10FBB40004F11C01002005F04FFAE369002BF3D196
:10FBC4007846F7F7B1FAEFE7585A002008B500F184
:10FBD400450200F14801002005F03EFA08BD00B5D9
:10FBE40087B006A9002301F8143D02684368CDF8E4
:10FBF4000520CDF80930092241F62800F7F748F925
:10FC040007B05DF804FB30B58FB005460C46002301
:10FC14000A93ADF82C3008210DF12E00FBF776F98C
:10FC2400210A41EA0421ADF8361006AA0AA9284699
:10FC3400FBF7F4FD01238DF8043008AB03CBCDF8BA
:10FC44000500CDF80910DDF82E20DDF83230CDF8AE
:10FC54000D20CDF81130112201A941F62800F7F743
:10FC640017F90FB030BD000010B582B0114BDC693C
:10FC740093F8203054B13BB908340E4B5B783BB158
:10FC8400012B0AD002B010BD3034F6E70024F4E7AB
:10FC940004F11000FFF7A3FFF4E70DF1060101A83A
:10FCA40005F0A4FABDF8041004F11800FFF7ABFF47
:10FCB400E8E700BF585A002008B5FFF769FFFFF7CF
:10FCC400D3FF08BD2DE9F04182B005460E46174624
:10FCD4009846002316220121FFF718FFA8B904460D
:10FCE400EB6C00939DF82030424639463046FEF7CF
:10FCF4004FFD30B92846FFF7CBFE204602B0BDE8E1
:10FD0400F0817846F7F710FAF4E70424F5E70000E9
:10FD14002DE9F04383B08146884617461E460024E9
:10FD240025461CB1284603B0BDE8F0830B4A5C238A
:10FD340003FB042393F844300BB90134F1E7009634
:10FD44003B464246494605484FF05C0C0CFB040018
:10FD5400FFF7B8FF0028F0D00425EEE7DC5A0020B6
:10FD64000378042B00D07047C3681B78012BFAD0AA
:10FD740010B5044601690948FCF788FC00B110BDC0
:10FD8400637E227E6169A068FFF7C2FF0028F6D176
:10FD940021690248FCF7A4FCF1E700BF7C5A00206B
:10FDA40010B5034C201DFAF793FE0023237010BDF9
:10FDB400585A002010B5044600F06DFC0023A364DB
:10FDC40010BD70B582B0044619E03035F9F74CFF28
:10FDD4000646F9F769FF94F84530003318BF01234C
:10FDE40000930346324629462046FFF76BFF70B95D
:10FDF40004F1450204F14801002005F02DF9A56C39
:10FE04002DB194F84530002BDFD10835DEE702B080
:10FE140070BD10B504460846FFF712FE00230246E3
:10FE240002212046FFF772FE18B9E06CFCF70FF9C7
:10FE340010BD0020FCE730B583B00546144601220E
:10FE440000920A462146FCF71DFA58B9EB7A2BB109
:10FE5400AB7A2BB96B8833B9012004E0002002E0AF
:10FE6400002000E0002003B030BD012A01D00920A9
:10FE7400704708B5097800F01BFC08BD70B590B058
:10FE8400402A18D812F0010617D1520833460AE066
:10FE940031F813502C0A44EA052410AD05EB430550
:10FEA40025F8404C01339342F2D3694600F013FC29
:10FEB400304610B070BD0926FAE70926F8E770B598
:10FEC40090B0402A18D812F0010617D152083346D0
:10FED4000AE031F813502C0A44EA052410AD05EB6E
:10FEE400430525F8404C01339342F2D3694600F0B0
:10FEF4001FFC304610B070BD0926FAE70926F8E762
:10FF040070B588B004460D4616460023019302934B
:10FF1400039304930593069301238DF80F30F9F7A7
:10FF2400A9FE059006950DF11E0103A805F05EF9E2
:10FF340004A8F9F731FE80B9054601A9E06CFCF785
:10FF44001CF80123E26C314601A8FCF7DCF92046D9
:10FF5400FFF79EFD284608B070BD2046FFF772FDEE
:10FF64001125F7E738B504460D460421FFF751FF84
:10FF740080B10322027094F842204270B4F8401019
:10FF84000A0A42EA01224280042229462046FFF757
:10FF9400B7FF38BD0420FCE770B59AB01446531E71
:10FFA400412B16D92A4B1B6813F0010F0FD0294B94
:10FFB4001B68012B0BDD284BD3F804350192274A2B
:10FFC40000924FF4057226490220FCF767FC1AB030
:10FFD40070BD054609AB03A8FFF72DFFA0B91C4B64
:10FFE4001B6813F0010FF2D01A4B1B68032BEEDDD4
:0CFFF400194BD3F804351B4A009240F270
:020000023000CC
:100000000F2218490420FCF74BFCE2E709A8FCF793
:1000100020F80646214603A8FCF70FF8421E337865
:10002000012B12D033B1022BD3D1711C2846FFF71C
:1000300048FF03E0711C2846FFF719FF0028C8D1CC
:1000400008992846FFF790FFC3E7711C2846FFF781
:1000500017FFF3E7383300203433002000B00040AE
:10006000F8F90300DBF90300E4F90300F0B58BB005
:1000700005460C4617461E46002304930593069337
:1000800007930893099301238DF81030FAF7EEFDDA
:1000900005901D4BEB1A9B101C4A02FB03F3ADF8B5
:1000A00018301B4B1B6813F0010F03D0194B1B6852
:1000B000032B09DC184B01221A70944218D08CB122
:1000C000022C1BD00BB0F0BD144BD3F804350296B4
:1000D0000194134A009240F2252212490420FCF7B1
:1000E000DFFBE7E704AA31463846FBF7E9FEE9E71C
:1000F00004AAF1B23846FEF783FBE3E732463946FD
:100100002846FFF74BFFDDE7DC5A0020A737BDE9A3
:100110003833002034330020485B002000B000401A
:10012000A0FA0300DBF9030038B50D460246A8B972
:100130000024134B5A701B789BB9ADB91148FAF7DC
:10014000C9FC4FF448612046F6F71AFFFFF78EFD11
:10015000F6F720FF0A4B01221A7038BD4EF66024D4
:10016000E7E7F6F727FFE8E7FFF714FDFAF77EFD6C
:10017000034B19690144181DFAF7DCFCE1E700BFE5
:10018000585A00205C5A002070B582B00446467868
:10019000864D5C2000FB06552278052A00F2EE8091
:1001A000DFE812F083009F00CB00060040006900EA
:1001B0007F4B1B6813F0010F03D07E4B1B68032B92
:1001C0001ADCFFF7EFFD794A5C2303FB06260123C7
:1001D00086F84430784A13702846FFF7EDFD28462C
:1001E000FFF7F6FC0023194693B100294FD10121F6
:1001F0000020FFF799FF4AE0704BD3F80435704AAE
:10020000009240F23F226F490420FCF749FBD8E7F7
:1002100066485C2202FB030292F8442002B10131DD
:100220000133E1E7624B1B6813F0010F03D0614B10
:100230001B68032B13DC5D4A5C2303FB06260023AB
:1002400086F844305C4A13705F4B1B78FBB15F4B00
:100250001B78E3B901210020FFF766FF17E0574B39
:10026000D3F804355A4A00924FF4147255490420C9
:10027000FCF716FBDFE74E4B1B6813F0010F03D0B2
:100280004C4B1B68032B04DC2846FFF79CFD02B097
:1002900070BD4A4BD3F804354E4A009240F25B22BF
:1002A00048490420FCF7FCFAEEE7414B1B6813F0C9
:1002B000010F03D03F4B1B68032B06DCA389A26808
:1002C00021792846FFF7D2FEE1E73C4BD3F804350D
:1002D000414A00924FF418723A490420FCF7E0FAC0
:1002E000ECE7334B1B6813F0010F03D0314B1B6855
:1002F000032B16DC237A002BC9D16568B5F1FF3FCB
:1003000014BF00250125FAF7B1FC5C2303FB06F6B8
:10031000503663680246294624483044FDF7FCFD08
:10032000B5E7264BD3F804352C4A00924FF41A72E5
:1003300024490420FCF7B4FADCE71D4B1B6813F0DA
:10034000010F03D01B4B1B68032B0BDC1F4B002240
:100350001A701D4B1B78002B99D001211046FFF716
:10036000E3FE94E7154BD3F804351D4A009240F2A2
:10037000772214490420FCF793FAE7E70C4B1B683B
:1003800013F0010F83D00B4B1B68012B7FF77FAF5E
:100390000A4BD3F804350192124A009240F28122AE
:1003A00008490220FCF77CFA71E700BFDC5A002004
:1003B0003833002034330020D85A002000B00040E9
:1003C00028FA0300DBF90300385B0020585A0020AC
:1003D00034FA030044FA030050FA030054FA03000D
:1003E00064FA030074FA030070B582B000241A4B5B
:1003F0001C701A4B93E803000090ADF804102246DD
:1004000017496846FEF7F2FE1648174B0360FAF7E5
:100410007DF8164808238360154B0360042343606E
:10042000FCF727F9134B144ADA60144A1A611C705E
:100430000CB102B070BD124D5C2606FB04F606F14D
:10044000500002220F492844FDF77EFD3544002369
:1004500085F844300134EBE7385B0020ACF9030049
:10046000890103003C5B002065FD02007C5A0020EE
:10047000985A0020585A0020BDFC0200809698002F
:10048000DC5A002094FA030030B583B00C4609B35F
:10049000002301930DF1030201A9204604F0DEFDC3
:1004A000019BDBB1019C9DF80330ECB1D3B130343A
:1004B000F9F7DCFB0546F9F7F9FB9DF80330022B51
:1004C00014BF00230123024629462046FFF722FCE1
:1004D00003B030BD7846F6F729FED9E77846F6F73F
:1004E00025FEDFE70834E3E70024E1E70B78012B82
:1004F00000D0704710B50C89104A5C2303FB04231D
:1005000093F8443073B15C2303FB042393F8423027
:100510004BB1012200F10801084B5C2000FB0430C4
:1005200000F008F910BD012200F10801034B5C2026
:1005300000FB043000F0D1F8F4E700BFDC5A0020E3
:10054000084B1B785BB910B50024074BDC61012117
:10055000044B19702046FFF7E7FD204610BD082028
:10056000704700BF385B0020585A002010B50F4B71
:10057000D86183F820100E4B01221A7000231C460C
:1005800043B18CB9B0FA80F149090120FFF7CCFDE5
:10059000204610BD07495C2202FB031292F844205A
:1005A00002B101340133EBE71124F1E7585A00207E
:1005B000385B0020DC5A00200D4B1B787BB10D4BC3
:1005C0001B7873B10B4B5B78012B01D00020704777
:1005D00048B1084BDB69834207D0002070470020F8
:1005E000704700207047012070470120704700BF0E
:1005F000385B0020585A002008B50020FFF7DCFFC8
:1006000028B101210020FFF78FFD002008BD082040
:10061000FCE70000134B1B7813B310B5114B0022FD
:100620001A70114B1B7813B900242CB110BDF6F7CA
:10063000C1FCFFF7B7FBF7E70C4A5C2303FB04237D
:1006400093F844300BB90134EFE7A0B2FEF7F2FEA5
:10065000064A5C2303FB0423002283F84420F2E7CC
:10066000704700BF385B0020585A0020DC5A002039
:10067000014B1878704700BF385B00200023B0F8AA
:1006800040209A4205D930F813208A4203D0013322
:10069000F5E7002070470120704710B5044628B1E7
:1006A000002384F84230A4F8403010BD7846F6F7B5
:1006B0003DFDF5E738B50C46054618B1012C05D9C6
:1006C0000B2038BD7846F6F731FDF7E72846FFF7EF
:1006D000E4FF85F842400020F3E72DE9F8430F4698
:1006E0009046064610B12FB1002408E07846F6F790
:1006F0001DFDF8E77846F6F719FDF5E701344445A6
:1007000016D2B6F840501F2D12D84FEA440937F8D8
:1007100014100029F2D03046FFF7B0FF0028EDD1C9
:100720006B1CA6F8403037F8093026F81530E5E79D
:10073000BDE8F883F8B50D461646044610B12DB154
:10074000002710E07846F6F7F1FCF8E77846F6F770
:10075000EDFCF5E7013A92B2A4F8402034F81220FB
:1007600024F813200137B7420CD20023B4F84020FC
:100770009A42F7D935F8170034F813108842E9D0B7
:100780000133F3E7F8BD38B50D46044650B12946AC
:100790002046FFF773FF94F8423013B180F0010058
:1007A000C0B238BD7846F6F7C1FCF0E710B5044694
:1007B000837803F00303032B21D8DFE803F0020C56
:1007C000131981788B081A4A11681944A160194BD2
:1007D0001B6800201AE083789B0803EB8303590011
:1007E0000B46F0E783789B08642101FB03F3EAE7FB
:1007F00083789B0841F2707101FB03F3E3E77846CD
:10080000F6F794FC0023DEE71846DB681BB19A6814
:100810008A1A002AF8DA18B133B1C460E36010BD57
:10082000E360044B1C60FAE7C4600023E360F6E772
:10083000645B00206C5B002010B56F4B19688B78EF
:1008400003F003036D4A1278934240F3B0808C6842
:100850006B4B1B68E41A6B4B03FB04F4032A09D8A7
:10086000DFE802F0020D0406664B09E0664B07E084
:10087000664B05E07846F6F759FC002300E0644B30
:10088000B4FBF3F35C4A1268927802F00302022A86
:1008900019D03AD8012A6AD102F1CC32A2FB031254
:1008A000D20802EB820251008B4202D00022134692
:1008B0005FE0FAF7DBF900F5742303F5107301220A
:1008C0004E490A7055E04D4A117839B9514AA2FB98
:1008D00003025209642000FB12326AB1012902D0DE
:1008E0000022134645E04C4AA2FB0312D20802EB59
:1008F000820251008B4249D1FAF7B8F9424B0344C6
:100900003E4A02211170012233E03C4A117841B97C
:10091000424AA2FB0302D20941F2707000FB12327C
:1009200082B1012904D0022915D00022134620E00B
:100930003B4AA2FB030292094FF4167000FB1232ED
:10094000002AF0D1FAF792F9304B03442B4A0321E5
:10095000117001220DE0334AA2FB03125209C2EBCF
:10096000021291008B42EDD00022134601E00022DA
:100970001346002A3DD1FAF779F904461F4B1B783C
:10098000032B0CD8DFE803F00510070900221346FB
:10099000EFE71C4B09E01C4B07E01C4B05E07846D9
:1009A000F6F7C4FB002300E0194B234421E0FAF7DB
:1009B0005DF90446104B1B689B7803F00303032B7F
:1009C00009D8DFE803F0020D04060E4B09E00E4BD8
:1009D00007E00E4B05E07846F6F7A8FB002300E0A1
:1009E0000B4B2344044A12689278C2F30102034974
:1009F0000A70184610BD00BF6C5B0020695B0020C8
:100A0000645B0020A0860100809698000046C32306
:100A100040420F001F85EB51CDCCCCCCF1197605AF
:100A2000B5814E1B8988888810B5294B1B7873B90E
:100A3000284B1B68002B42D0FFF7FEFE0146244BDB
:100A40001B78002B33D02448FAF774F83AE0224B95
:100A50005C68FAF70BF9241A204B1B78032B09D892
:100A6000DFE803F0020D04061D4809E01D4807E019
:100A70001D4805E07846F6F759FB002000E01B48CA
:100A8000001B164B1B7843B94CF25033984204D9E3
:100A9000174A136801331360CAE74009154BA3FBDB
:100AA0000030134A136803EBD0101060C0E7084B06
:100AB00001221A7008484160F9F7DAFF02E0044B9E
:100AC0001B7803B910BD0448FAF704F8FAE700BF31
:100AD000685B00206C5B00204C5B0020695B0020A1
:100AE000A0860100809698000046C32340420F0074
:100AF000645B0020C55A7C0A30B583B006E06368A9
:100B00000199284698472046FFF750FE104B1C6875
:100B1000D4B1A3680F4A1268934204D00D4A1268F8
:100B20009B1A002B10DA2588E268094B1A6002A98B
:100B3000002341F8043D284601F004FD0028DED0E2
:100B40007846F6F7F3FADAE7FFF76EFF03B030BD49
:100B50006C5B0020645B002008B5134B1B78032BF3
:100B60001ED8DFE803F0020C1116104A1368013397
:100B700013600F4B00221A70FFF7BEFF08BD0B4A2F
:100B800013680A331360F4E7084A13686433136088
:100B9000EFE7064A136803F5BB5310331360E8E729
:100BA0007846F6F7C3FAE4E7695B0020645B00204F
:100BB000685B002010B50446FFF7F8FD034B1B6887
:100BC000A34200D010BDFFF72FFFFBE76C5B0020B6
:100BD000074A002313605360D360136153610549D2
:100BE0009160054A1360054A1360054A1370704707
:100BF0004C5B0020590B0300645B00206C5B002001
:100C0000685B002070B50E461546044628B1FAF719
:100C1000CFFC144B1B68002205E07846F6F786FAF5
:100C2000F5E71A46DB680BB1A342FAD1A17866F367
:100C3000010165F38701A17013B13AB1D968D160A0
:100C400045B903B152B1FAF7D3FC70BDD868054974
:100C50000860F5E72046FFF7ADFFF4E7FFF7E4FE95
:100C6000F1E700BF6C5B002070B50E4615460446E8
:100C700040B1A378C3F301033370A378C3F38503B2
:100C80002B7070BD7846F6F751FAF2E710B44FF6C4
:100C9000FF7399420CD00C4A43001C1861000C46AB
:100CA0001144C97822444B1CD3705DF8044B704743
:100CB000054A43001C1861000C46114489782244FF
:100CC0004B1C9370F1E700BF705B002030B482B022
:100CD00001911A4943001D186C000C44A578034487
:100CE0005C002144CB78DD4201D0002303E00020EA
:100CF00020E001339BB2022B1BD81D46104C34213F
:100D000001FB034189898142F3D1342101FB034175
:100D10004C88BDF806108C42EBD1342101FB05F55F
:100D200007494C5BBDF804108C42E2D113800120CE
:100D300000E0002002B030BC704700BF705B0020B4
:100D4000AC5B002082B000230093027802F0C00365
:100D5000402B0ED00CD9802B1BD0C02B0FD1ADF85F
:100D600000204278837843EA0223ADF8023006E09F
:100D70002BB9ADF800204FF6FF73ADF80230009BA1
:100D800000209AB262F30F001B0C63F31F4002B005
:100D90007047437843EA0222ADF800204FF6FF7314
:100DA000ADF80230EBE782B00190000C4FF6FF7314
:100DB000984207D0BDF804300B70030A4B7088705E
:100DC00002B07047BDF8043013F47F4F01D10B70AF
:100DD000F6E71A0A0A704B70F2E782B001904FF6FC
:100DE000FF73B3EB104F0AD0BDF8040020F03F00B2
:100DF00080B2C02814BF0020012002B07047BDF8A7
:100E0000040010F47F4F07D120F07F039BB26BB931
:100E10007F2809D00120F0E700F44040B0F5004FF2
:100E200014BF00200120E8E70020E6E70020E4E707
:100E300070B506460D460024AC4207D256F8340081
:100E4000FFF7CBFF034610B10134F5E70123184645
:100E500070BD30B482B00191002300E00133018DF8
:100E6000994210D9416A01EBC30531F83340BDF80E
:100E700004108C42F2D16C88BDF806108C42EDD182
:100E80001360012000E0002002B030BC7047000079
:100E9000C2898AB9094B03EBC20304334A0953F8E8
:100EA000223001F01F0123FA01F111F0010F01D1ED
:100EB000002070470120704700207047485C0020E8
:100EC00008B5804708BD00004388C3F30B03C3B9CE
:100ED00030B41C460C4911F8332042F0010201F8ED
:100EE000332013B1012030BC704700EB83025168FE
:100EF000C94303EB4405044A02EB85025160013308
:100F0000EFE70020704700BF485C00204388C3F330
:100F10000B033BB9818803EB43035A00024B995200
:100F20000120704700207047705B0020F0B583B04F
:100F30000F4616464FF47043ADF80430ADF8060086
:100F400000252C46224601A90A48FCF708FA044667
:100F500010B1B04740B10135002CF3D1AF4205DAF2
:100F60007846F6F7E3F801E04FF0FF35284603B086
:100F7000F0BD00BF845B002008B57846F6F7D6F8D0
:100F800008BD0000F8B505460E4617461C4683B15D
:100F90003389B3F5BE7F10D2022D15D81F4A3423F2
:100FA00003FB052393F8303013F0010F1CD100230D
:100FB0000BE07846F6F7BAF8EAE7092323602068E1
:100FC000B0FA80F04009F8BD00237BB1134A342306
:100FD00003FB05239B894BB95FB13068FFF7FDFE2A
:100FE000C8B100232360EAE70123EEE7052323606D
:100FF000E5E70A4A342303FB05239A884FF6FF737B
:101000009A4208D0054B342202FB0535EA884FF698
:10101000FF739A42E1D107232360D0E7AC5B002045
:10102000F8B54388C3F30B03022B33D8021D018AA2
:1010300091BB1B4C342101FB0341C98951B9448A3E
:10104000A14201D0002026E0164911F8341011F019
:10105000010F23D0418A31B9124D15F8314044F0C7
:10106000040405F831400E4D342101FB03F3E91867
:101070001468D2F804C09768D668EC50C1F804C070
:101080008F60CE6014690C618188008AFFF7FEFDD5
:10109000012000E00020F8BD0020FCE70020FAE776
:1010A000AC5B0020485C002008B5064B01221A709A
:1010B0000548FCF703F900B908BD0448FCF74CFBF0
:1010C000FAE700BFA85B0020845B002060330020AB
:1010D0002DE9F041FAF76CFA5A4B1B78002B47D1F7
:1010E000594B1B780BB1002543E0062201215748DC
:1010F000FCF7DBF950B10124C48003220281848013
:10110000FCF70CFA504B1C70002532E0112530E042
:1011100003EB44004E4A02EB80025268D24301EBDB
:1011200083004260013316E011250134A4B2002C83
:1011300048D11DBB464B13F8343003F00303032B97
:10114000F3D1042244F440514048FCF7AEF9014683
:101150000028E9D02B46002BDAD00846FCF7DEF950
:101160003B4A12F8343023F0020302F83430DCE753
:1011700008250024DBE711250134A4B2002C56D148
:101180002DBB04EB44035A00324B13445B7913F03C
:10119000020FF1D0022244F480512C48FCF785F96B
:1011A0000028E8D02B4F4FEA440808EB04014B001D
:1011B000FE18FB5A8380FCF7B1F9737923F0020320
:1011C0007371D9E70024D9E711250134A4B2022CA8
:1011D0002FD875BB204A342303FB042393F8303007
:1011E00003F00303032BF0D1142244F400511748F9
:1011F000FCF75BF902460028E6D01749342606FBC7
:1012000004163168D6F804C0B768F0685160C2F8B7
:1012100008C0D7601061316951611046FCF77EF952
:1012200096F8303023F0020386F83030CDE7002402
:10123000CDE71DB9FAF7DCF9BDE8F0810748FCF706
:101240008BFAF7E7A85B0020A95B0020845B0020F5
:10125000485C0020705B0020AC5B002070330020F5
:101260000378012B08D0438804339BB2032B12D898
:1012700000230B800120704730B583B00D46044633
:1012800001A802F049FE6388BDF804209B1A2B8058
:10129000012003B030BD00207047000008B59C223B
:1012A00000210D480DF079FF0C4A00231360938054
:1012B0000B4A136053600CE00749342202FB03120F
:1012C0004FF6FF71D18091800120D081918103443C
:1012D0009BB2022BF0D908BDAC5B0020705B0020F4
:1012E000485C002000B587B00F4B03930F4B04936D
:1012F0000F4B05930423029302F00CFDA0F58050E0
:101300000090012301930B4A137069460A48FCF7C9
:10131000DDF928B9074B00221A7007B05DF804FB0D
:101320000648FCF719FAF8E7CD130300790F03001C
:1013300041130300A85B0020845B00205033002091
:1013400010B500231BB100237BB1002321E01C4A10
:1013500012F8332012F0010F04D042F002021849B3
:1013600001F8332001339BB2ECE703EB43014A0061
:1013700014498A5A42B108465A00D41861000144FF
:101380004A7942F002024A7101339BB2DCE7013331
:101390009BB2022B11D80C49342202FB031292F8A3
:1013A000302012F0010FF2D00846342101FB030176
:1013B00042F0020281F83020E9E7FFF793FF10BD09
:1013C000485C0020705B0020AC5B002070B58CB0E6
:1013D00005460E461446012A05D0022C07D0032CE0
:1013E00009D00CB070BD7846F5F7A0FEF5E7784659
:1013F000F5F79CFEF3E72C22002101A80DF0CDFEAD
:1014000010238DF8043002238DF808300396EB6822
:1014100005932B69069301A8F7F744FAE1E700006A
:101420002DE9F04F95B004AF82460C46154607F102
:101430003C03FFF7A7FD20B9F86B4437BD46BDE874
:10144000F08F07F1380002F067FD9C4A342303FB5C
:101450000A239E897B8F9E4280F029813B8F1E4408
:10146000B6B2002D00F0A180B5F81E80B5F824902A
:1014700007F130030C3595E8030083E803008F4B38
:10148000342202FB0A3A9AF81050FF2D00F0A08097
:1014900007F1300001F0F8FA8246002840F09B8006
:1014A000BAF1000F04D097F83030012B00F0FD8026
:1014B000EB462422002107F10C000DF06EFE23897B
:1014C00022683A604FF6FF71B1EB124F00F0A08036
:1014D00003221344073323F00703ADEB030D0DF193
:1014E000100A07F124024146484603F03BFCF8632A
:1014F000002840F0948007F10C0307F1300292E8D5
:10150000030083E80300BE82BD75A37AFB75E37A0E
:101510003B76C7F81CA023892268BA604FF6FF719A
:10152000B1EB124F7DD0032213443B84E368FB628E
:1015300051462068FFF737FC23687B604FF6FF7247
:10154000B2EB134F74D003202289616850440DF030
:10155000FBFD002107F10C00F8F7AAFFF863002853
:1015600040F0A280564B1B6813F4005F03D0554B2C
:101570001B68042B63DC524B1B6813F4005F00F004
:101580009380504B1B68042B40F38E80E846B4F8E0
:1015900008C04FEA4C030833DB08A8EBC3039D46A1
:1015A0000DF1100E7646002369E0444A342303FB14
:1015B0000A23B3F8048007F13001D88802F0A2FDB5
:1015C000002876D17B8E002B75D04FF6FF7956E739
:1015D0003D4B1D785CE7E368FB6023683B61636813
:1015E0007B6123893B837E8307F11C0307F1300273
:1015F00092E8030083E8030087F82450A7F82680C8
:10160000A7F8289007F10C0001F04EFAF86347E7BD
:101610003A88FF2A01D902225BE7012259E7DD4619
:101620000BE73A89FF2A01D902227DE701227BE7F5
:10163000BB88FF2B01D9022086E7012084E7234BDA
:10164000D3F8043522880192214A00924FF4CC72DB
:1016500020490520FBF724F98DE76268D25C4FEA48
:10166000121959001C4D286810F8090006F81300DB
:1016700002F00F0201312868825C72540133634525
:10168000EBD300230EF81C30104BD3F80435CDF803
:1016900008E0124A0192124A009240F299120D4952
:1016A0000520FBF7FDF8C546DD46F86BC5E61020C2
:1016B000C3E60520C1E61020BFE600BFAC5B0020FA
:1016C00038330020343300208033002000B0004045
:1016D00028FB03001DFB03003C3300203CFB030000
:1016E00038F40300F8B5FCF74FF828B9FAF72AF8F0
:1016F0000028F8D020BFF6E75F4B00221A700121C6
:101700005E48FBF705FE002800F0B380C288012A7E
:1017100040F0A7800289032A01D00024A2E0838838
:10172000012B01D000249DE00121534B1970544A34
:101730004FF44050FFF7FAFB002820DA00231C4644
:10174000002B00F08F8092E04E4C5A001A4451005A
:10175000621800209070D0706052517921F002011F
:1017600051710133002BEFDD474A01214FF48050C6
:10177000FFF7DCFBC743FF0F1FB90023DFE70023A0
:10178000F0E7424A03214FF40050FFF7CFFB002857
:1017900061DD002538E002F0D3FB002848D0784610
:1017A000F5F7C4FC44E010240FE07846F5F7BEFCE2
:1017B00012E051420A40364901FB02F2D20E35498D
:1017C0008C5C04EB431400E01024102C1AD0A0B25F
:1017D00002F050FC0028E8D101340F2CF4D8630942
:1017E00056F8232004F01F04012101FA04F4614299
:1017F0000A40002ADDD1013302D156F82320F8E750
:101800001024E2E70135ADB2022D25D8224A342357
:1018100003FB05239A894FF6FF739A42F2D01E4BC1
:10182000342404FB0534E0884FF6FF739842B2D1AC
:10183000E289012AE6D0194B03EBC2031E1D5B6847
:10184000002BB0D05A421A40114B03FB02F3DB0EBF
:10185000104AD45CB9E700270FB101236FE70023DA
:101860006DE70024044B00221A70FFF71DFC204690
:10187000F8BD0024FBE700BFA95B0020845B0020CB
:10188000C90E0300705B00200D0F03002110030040
:1018900031B57C07D4FA0300AC5B0020485C002023
:1018A000F0B583B0064600F11404204603F076FC40
:1018B00008B903B0F0BD4FF6FF73ADF802306946CA
:1018C0002046FFF7CDFC074608B100241EE00DF1CD
:1018D0000201204602F0C2FC0028F6D07846F5F757
:1018E00025FCF2E7BDF802102846FFF7D1FA1CE00C
:1018F000254A342303FB04235A6A019902EBC102EF
:101900005568DA6A3146A0B2A8470134022CD0DC0F
:101910001D4B342505FB0435002FE3D0AB89BDF802
:101920000000984214BF00200120174A342303FB13
:10193000042393F8303013F0010FE6D00028E4D0F0
:10194000342303FB04F308331344F28B510953F897
:10195000213002F01F0223FA02F212F0010FD4D05C
:1019600001AA31682846FFF774FA0028CDD0337DEC
:10197000012BBDD1044A342303FB0423DA6A314628
:10198000A0B200F0B5FFB3E7AC5B002070B590B03B
:10199000044600284BD02068FFF7D4F90F9085B299
:1019A0007F2D42D0304B1B6813F4005F03D02F4BC8
:1019B0001B68042B3FDCE06902F0CBFC0646A06903
:1019C00002F0B0FC0F9A059223684FF6FF71B1EB5D
:1019D000124F3CD0032213440693A388BDF83E1057
:1019E0004FF6FF72914238D003229B1AADF81C309B
:1019F000237A8DF820306389ADF82230E3680993AB
:101A0000237C8DF82830638AADF82A3063690B9304
:101A100094F820308DF83030ADF83260636A0D9361
:101A2000ADF8380005A8FFF73BFF10B070BD784651
:101A3000F5F77CFBAFE70E4BD3F8043501950D4A63
:101A40000092F1220C490520FAF72AFFB3E7FF2D97
:101A500001D90222BFE70122BDE7FF2D01D80122F3
:101A6000C3E70222C1E700BF38330020343300202F
:101A700000B00040C0FA03001DFB030008B5037866
:101A800003B108BD0430FFF781FFFAE708B5FFF79F
:101A900005FC00F075FFFFF707FB08BD08B5FFF771
:101AA000FDFB0748074B0360F8F730FD00F05AFFD5
:101AB000FFF78EF800F0ECFFFFF714FC08BD00BF45
:101AC000785B00207D1A0300002800F09580F8B5AF
:101AD00004468268002A00F09180002900F090807E
:101AE0004FF6FF720A80C268002A00F08B8080885F
:101AF000002840F089800D460A462168FFF7E6F885
:101B000048B12B88444A342101FB032393F8303039
:101B100013F0010F7AD1E168A068FFF789F9002876
:101B200076D02A884FF6FF739A4257D029882069C9
:101B3000394B342202FB0131C8622988A06802FBBC
:101B400001314862E068298802FB01310885298853
:101B5000606902FB01318861298802FB01308182C2
:101B6000298802FB013393F8302042F0010283F808
:101B70003020002049E09AB22A804FF6FF739A4243
:101B800048D0254E342707FB02621946D3802B88A4
:101B900007FB036399802B88A28807FB03639A8164
:101BA0002B88628807FB03635A802B88228807FBF7
:101BB00003F3F2522B8807FB0363184A12781A7456
:101BC0002188A088FFF762F82B8807FB036696F848
:101BD000303043F0020386F83030A7E70023022BB1
:101BE000CAD80D48342101FB030191F8301011F0DF
:101BF000010FC0D00133F2E70E2070470E2004E041
:101C00000E2002E0092000E00520F8BD0F20FCE7CF
:101C10000720FAE70420F8E7AC5B002080330020BF
:101C200021B108B50022FFF7FBFB08BD0E2070476D
:101C300039B108B50B4632B111461A46FFF7F0FB31
:101C400008BD0E2070470E20FAE7000002280AD8CF
:101C5000154A342303FB002393F8303013F0010FAF
:101C600019D1002300E00023BBB10F2917D80E4A79
:101C7000342303FB0023DB888B4212D0134634222B
:101C800002FB0030C18090F8303043F0020380F84E
:101C90003030002070470123E6E705207047072019
:101CA00070470020704700BFAC5B00200A46C1B1FE
:101CB00002280AD80D49342303FB001393F830306F
:101CC00013F0010F0BD1002300E000235BB1074BA1
:101CD000342101FB0030C3881380002070470123AA
:101CE000F4E70E2070470520704700BFAC5B002072
:101CF00002282BD8174A342303FB002393F83030F3
:101D000013F0010F24D0342303FB00239B7C03F04A
:101D1000070301F0070293420CD00E4B342202FB62
:101D20000030817490F8303043F0020380F8303096
:101D300000207047074A342303FB00239A7CC1F339
:101D4000C403B3EBD20FE8D10020704705207047E1
:101D500005207047AC5B00200A4691B1022812D8DA
:101D60000B49342303FB001393F8303013F0010FB9
:101D70000BD00B46342101FB0030837C1370002014
:101D800070470E207047052070470520704700BF40
:101D9000AC5B0020022839D870B5224C342303FBF9
:101DA000004393F8303013F0010F31D0342303FB9C
:101DB00000439B6973B33F2A2ED803292ED83423BE
:101DC00003FB00435B7CB2EB930F07D1342303FB8F
:101DD00000435B7C03F003038B4221D0114C34237E
:101DE00003FB00F025186B7C62F3870361F30103AA
:101DF0006B74103020440430FEF704FF95F8303047
:101E000043F0020385F83030002002E005207047DF
:101E1000052070BD0620FCE70720FAE70720F8E759
:101E20000020F6E7AC5B002021B30B4622B310B5CF
:101E300002280AD8134C342101FB004191F83010DC
:101E400011F0010F14D1002100E00021B1B10D4CBF
:101E5000342101FB0041896991B11946342303FB08
:101E600000F0103020440430FEF7FEFE002010BDCC
:101E70000121EBE70E2070470E2070470520F6E7A2
:101E80000620F4E7AC5B002002280AD8184A342365
:101E900003FB002393F8303013F0010F0DD1002322
:101EA00000E0002313B3124A342303FB0023DB8931
:101EB000012B04D00023184670470123F2E70023CA
:101EC0000BB10423F7E70B4A12F8332012F0010F8D
:101ED00001D00133F4E742F00102064901F8332052
:101EE000034A342101FB0020C381E4E70523E2E734
:101EF000AC5B0020485C002002280AD8214A342329
:101F000003FB002393F8303013F0010F30D100238E
:101F100000E0002373B31B4A342303FB0023DA8958
:101F2000012A29D00F2929D830B4174B03EBC2035B
:101F300004334C0953F8242001F01F0122FA01F563
:101F400015F0010F1CD1012505FA01F10A4343F8F0
:101F500024200C4B342202FB0030C1890A4A12F8BB
:101F6000313043F0020302F83130002030BC7047BA
:101F70000123CFE7052070470620704707207047F0
:101F80000020F3E7AC5B0020485C002002280AD860
:101F9000224A342303FB002393F8303013F0010F5F
:101FA00031D1002300E000237BB31C4A342303FB20
:101FB0000023DA89012A2AD00F292AD830B4184BF5
:101FC00003EBC20304334C0953F8242001F01F0132
:101FD00022FA01F515F0010F1DD0012505FA01F1D6
:101FE00022EA010243F824200C4B342202FB003089
:101FF000C1890B4A12F8313043F0020302F8313044
:10200000002030BC70470123CEE705207047062032
:102010007047072070470020F3E700BFAC5B00204B
:10202000485C002000293CD02DE9F8438846002A6E
:1020300039D002280AD82049342303FB001393F82F
:10204000303013F0010F11D1002300E0002363B3FF
:102050000746194B342101FB0030C389012B26D0E0
:102060001646B2F800900024148002E00123EEE747
:1020700001340F2C12D8A5B229460F4B342000FB97
:102080000730FEF705FF0028F2D03388994510D9B4
:1020900028F81350338801333380E9E70020BDE886
:1020A000F8830E2070470E20F9E70520F7E7062099
:1020B000F5E70920F3E700BFAC5B002002280AD84F
:1020C0001D4A342303FB002393F8303013F0010F33
:1020D00029D1002300E000233BB3082927D830B4DE
:1020E000342303FB00F30833134A13444C0953F819
:1020F000242001F01F0122FA01F515F0010F18D17B
:10210000012505FA01F10A4343F824200A4B342241
:1021100002FB003090F8303043F0020380F830309A
:10212000002030BC70470123D6E705207047072008
:1021300070470020F5E700BFAC5B002002280AD8FA
:102140001D4A342303FB002393F8303013F0010FB2
:102150002AD1002300E0002343B3082928D830B453
:10216000342303FB00F30833134A13444C0953F898
:10217000242001F01F0122FA01F515F0010F19D0FA
:10218000012505FA01F122EA010243F824200A4B55
:10219000342202FB003090F8303043F0020380F824
:1021A0003030002030BC70470123D5E70520704750
:1021B000072070470020F5E7AC5B0020A9B370B49E
:1021C0000D46A2B302280AD81C49342303FB00138E
:1021D00093F8303013F0010F07D1002300E0002303
:1021E0003BB316880023138002E00123F8E7013394
:1021F000072B17D8342101FB00F108310F4C214483
:102200005C0951F8241003F01F04E14011F0010FA4
:10221000EDD011888E420ED925F811301188013188
:102220001180E4E7002070BC70470E2070470E203C
:10223000F9E70520F7E70920F5E700BFAC5B0020D0
:1022400002280AD8154A342303FB002393F83030C0
:1022500013F0010F19D1002300E00023BBB10829BE
:1022600017D80E4A342303FB00239B888B4212D0DD
:102270001346342202FB0030818090F8303043F066
:10228000020380F83030002070470123E6E7052084
:102290007047072070470020704700BFAC5B0020EC
:1022A0000A46C1B102280AD80D49342303FB0013A2
:1022B00093F8303013F0010F0BD1002300E000231E
:1022C0005BB1074B342101FB003083881380002071
:1022D00070470123F4E70E2070470520704700BFC8
:1022E000AC5B002010F0800F05D1012805D0044B15
:1022F000187000207047072070470720704700BF04
:1023000080330020014B1878704700BF80330020D5
:1023100002280AD8164A342303FB002393F83030EE
:1023200013F0010F1BD1002300E00023CBB181F09B
:1023300080037E2B17D90E4A342303FB00231B7C1A
:102340008B4212D01346342202FB0030017490F805
:10235000303043F0020380F8303000207047012312
:10236000E4E705207047072070470020704700BF52
:10237000AC5B00200A46C1B102280AD80D493423BB
:1023800003FB001393F8303013F0010F0BD100233F
:1023900000E000235BB1074B342101FB0030037CDC
:1023A0001370002070470123F4E70E2070470520CA
:1023B000704700BFAC5B00200A4641B148B900EB52
:1023C000400043000449CB5A1380002070470E2080
:1023D00070470520704700BF705B002061B110B4EA
:1023E00060B900EB40004200054B13449B780B7032
:1023F00000205DF8044B70470E2070470520F8E779
:10240000705B002061B110B460B900EB4000420085
:10241000054B1344DB780B7000205DF8044B7047CC
:102420000E2070470520F8E7705B00200A46D9B1FE
:1024300002280AD80E49342303FB001393F83030E6
:1024400013F0010F0ED1002300E0002373B10849FF
:10245000342303FB00F00B185B8853800B5A138066
:10246000002070470123F1E70E20704705207047D8
:10247000AC5B002030B482B0019152B3154650BB22
:102480004FF6FF731380002301E001339BB2022B50
:102490001BD81C461149342202FB03129289824246
:1024A000F3D1342202FB03125188BDF80620914279
:1024B000EBD1342202FB04F4084A115BBDF804207E
:1024C0009142E2D12B80002000E0052002B030BC18
:1024D00070470E20FAE70520F8E700BFAC5B00204C
:1024E00029B3F0B40F4622B328BB1688002313800B
:1024F00000E00133022B17D81488B4421DD2104DCE
:10250000342101FB035191F8301011F0010FF0D08C
:10251000342101FB035189898142EAD127F8143023
:10252000118801311180E4E70020F0BC70470E20D3
:1025300070470E20F9E70520F7E70920F5E700BF0F
:10254000AC5B00200A46C1B102280AD80D493423E9
:1025500003FB001393F8303013F0010F0BD100236D
:1025600000E000235BB1074B342101FB0030C36A5C
:102570001360002070470123F4E70E207047052008
:10258000704700BFAC5B002002280AD8204A3423E1
:1025900003FB002393F8303013F0010F34D10023F4
:1025A00000E0002393B370B50546194C342303FBB8
:1025B00000F606F110002044002211460430FEF718
:1025C00021FB284600F018FAA3194FF6FF72DA80B3
:1025D0009A80997C01F0F8016FF3C701997400208B
:1025E0001874597C01F0030160F301015974997D5D
:1025F00001F0030160F30101997593F8302042F076
:10260000020283F8302070BD0123CBE7052070471C
:10261000AC5B002008281AD830B583B005460024EA
:1026200001E00134A4B2022C0ED80DF106012046BF
:10263000FFF736FE0028F4D1BDF80630AB42F0D1EA
:102640002046FFF7A1FFECE7002003B030BD0720D4
:10265000704700004FF6FF730B800023022B18D841
:1026600010B402E00133022B0DD80C4C2C2202FBDB
:10267000034292F84020002AF4D02C2202FB0342AD
:10268000128B8242EED106230B8001205DF8044BB1
:10269000704706230B800120704700BF505C00206C
:1026A00010B4124A2C2303FB0020836B104C1C44F3
:1026B00000234FF6FF7001E001339BB2022B11D8CB
:1026C0000A492C2202FB031292F84020002AF3D080
:1026D0002C2202FB0312926B111B0029ECDA184624
:1026E0001446E9E75DF8044B704700BF505C0020DA
:1026F0000087930310B50446204A2C2303FB0023D4
:1027000093F84030B3B11D4BB3F89C30B3B11B4AC2
:102710002C2303FB0423002183F84010B2F89C30E3
:10272000013B9BB2A2F89C3023B3B2F89E30A34287
:1027300008D010BD7846F4F7F9FCE4E77846F4F7E2
:10274000F5FCE4E72046FFF7ABFF0C4BA3F89E0037
:102750004FF6FF73984209D00848B0F89E302C22FB
:1027600002FB0303996BF8F7E5F9E2E77846F4F723
:10277000DDFCF1E70148F8F7ADF9DAE7505C00203D
:10278000F0B583B00546594BB3F89C3043B105F51D
:102790007A76564B4FF6FF72A3F89E20002471E024
:1027A0007846F4F7C3FCF2E72C2303FB0423002153
:1027B00083F84010B2F89C100139A2F89C1001A9CE
:1027C000188BFFF7BFFE48B9484A2C2303FB0423AC
:1027D0005F6B01220199188BB84752E07846F4F7F5
:1027E000A5FCF1E7414F2C2101FB04F17B181831C6
:1027F00039440431188BFFF713FAA7F89E40B8B993
:102800002C2303FB0473DA6B996B11449963520018
:10281000DA63364A2C2303FB04231A6B9B6BD31A0F
:10282000002B2EDA31492C2303FB04139A6328E092
:10283000042803D07846F4F779FCEAE72B4B2C22E6
:1028400002FB0434A36B03F51C434033A363274B03
:10285000B3F89C30002B44D0244BB3F89E30022BAD
:1028600039D8224AB2F89E302C2101FB03239B6BFE
:102870005A1B34D41D4BDA6003B0F0BD1B4BA3F8D8
:102880009E400134022CE2D8184A2C2303FB042377
:1028900093F84030002BF4D02C2303FB04231B6B54
:1028A0009B1B002B80DB114A2C2303FB04239B6B17
:1028B0009A1B002A96DB0D4AB2F89E204FF6FF7154
:1028C0008A42DBD009492C2000FB0212926B9B1A32
:1028D000002BD6DAD2E77846F4F728FCC1E7EA1AEB
:1028E000C8E7024B0022DA60C6E700BF505C002058
:1028F00070B582B004460D461646022815D8F8F782
:1029000057FE0DF106012046FFF7A4FE48B1BDF8C1
:102910000600134A2C2303FB00239A8D2B889A422E
:1029200007D0F8F765FE02B070BD7846F4F7FEFBFD
:10293000E5E70B4A2C2303FB0023DA8D6B889A42D0
:10294000EFD1FFF7D7FEBDF80630054A2C2101FB79
:1029500003235B6B0022314620469847E1E700BF26
:10296000505C002010B5044CA022002120460CF041
:1029700014FC024BA36010BD505C002081270300B3
:1029800070B582B0F8F714FE1A4BB3F89C300BB94F
:1029900000240BE017480023A0F89C30F8F79AF8C1
:1029A000F6E7022201992846B0470134022C1DD8CF
:1029B000104A2C2303FB042393F84030002BF4D05F
:1029C00010462C2202FB04F3C1180D8B4E6B1833FA
:1029D000002118440CF0E1FB01A92846FFF7B2FDE5
:1029E0000028DED07846F4F7A1FBDAE7F8F700FE1E
:1029F00002B070BD505C002010B582B0022828D80B
:102A00000446F8F7D5FD0DF102012046FFF722FE3E
:102A100028B90524F8F7ECFD204602B010BDBDF83A
:102A20000200FFF767FE01A92046FFF78BFD60B9A2
:102A3000BDF80230084A2C2101FB03235B6B022204
:102A40000199204698470024E4E77846F4F76EFBA6
:102A5000EEE70524E0E700BF505C002010B50AE077
:102A600004F11C00FEF71CFF06480168F9F781FE1F
:102A700020460CF0CFFA034B1C68002CF0D101204B
:102A800010BD00BFF45C002008B502F087FB08BD54
:102A900008B50348F8F7CEFD024B186008BD00BF2B
:102AA0005D2A0300F05C002070B505468089443043
:102AB0000CF066FA00282FD00446052303712B681A
:102AC00083606B68C36100F144030362AA89828456
:102AD000012180F82810E989418500F1300605F1CF
:102AE000100103C986E80300297E84F83810698B39
:102AF0006187211DE163A98BA4F84010A9681846DD
:102B00000CF022FB21460548F9F708FE044B186833
:102B1000F8F7B0FD002070BD0420FCE7F45C002055
:102B2000F05C002002460E4B1B6813F0010F0AD028
:102B30000C4B1B8898420FD30A48408803449A42A2
:102B40000CDB002300E00023184623B14A80012358
:102B50000B7000234B6070470023F5E70123F3E778
:102B6000005D0020E05E00204FF6FF730B80002325
:102B7000072B26D810B40DE05A09134C54F8222024
:102B800003F01F04E24012F0010F08D10B80013363
:102B9000072B12D80C884FF6FF729442ECD00B4AE8
:102BA00032F823208242F2D1084A02EB8302D27823
:102BB000002AECD00B80012000E000205DF8044BDF
:102BC00070470020704700BFF85C0020105D0020B7
:102BD0000B88072B01D8013300E000234FF6FF726A
:102BE0000A80072B1ED810B409E003EB8304A2006F
:102BF0000D4CA25A82420ED00133072B0ED85A092F
:102C00000A4C54F8222003F01F04E24012F0010F96
:102C1000EBD10B80F0E70B80012000E000205DF895
:102C2000044B70470020704788600020085D00203A
:102C30004FF6FF730B800023072B21D810B407E059
:102C40000C884FF6FF72944214D00133072B13D82F
:102C50005A090C4C54F8222003F01F04E24012F0F1
:102C6000010FEDD0084A32F823208242EDD10B80CB
:102C7000012002E00B80E8E700205DF8044B70477C
:102C800000207047F85C0020105D00204FF6FF73B5
:102C90000B80002373B10020704708330B800120A4
:102CA0001EE00C884FF6FF72944215D103F1080222
:102CB0000A8011E010B45A090B4C54F8222003F09A
:102CC0001F04E24012F0010FEBD0162202FB03F2C8
:102CD000064CA25A8242E0D00133002BEBD00020F8
:102CE0005DF8044B704700BF885E0020905E0020B6
:102CF0004FF6FF730B800023072B23D810B407E097
:102D00000C884FF6FF72944216D00133072B15D86A
:102D10005A090D4C54F8222003F01F04E24012F02F
:102D2000010FEDD02A2202FB03F2084CA25A824284
:102D3000EBD10B80012002E00B80E6E700205DF87C
:102D4000044B704700207047305D0020385D002044
:102D5000F0B416680023136000E00133072B1ED87F
:102D60005C09114D55F8244003F01F05EC4014F0A8
:102D7000010FF2D00D4D2A2404FB035464888442D1
:102D8000EBD11568B5420DD02A2404FB03F4074F9C
:102D90003C5B21F81540146801341460DDE7012024
:102DA000F0BC70470020FBE7305D0020385D00205C
:102DB00070B40D6800230B6000E00133012B17D8BD
:102DC0005A090E4C54F8222003F01F04E24012F07E
:102DD000010FF2D00C68AC420DD0C82202FB03F206
:102DE000074EB25A20F814200A6801320A60E4E75C
:102DF000012070BC70470020FBE700BFF05E0020A0
:102E0000F85E0020014688B100230BB10020704716
:102E1000162202FB03F20648825A8A4201D001338D
:102E2000F3E7162202FB0303181D704700207047CA
:102E3000905E00200D4B23F8210003EB810300225C
:102E4000DA709A704B090A4801F01F01012202FA58
:102E500001F150F823200A4340F82320054850F898
:102E60002320114340F82310704700BF105D00205D
:102E7000F85C0020FC5C00200A68014B1A60704777
:102E8000E05E002008B50B8881B21846FFF7D2FF3C
:102E900008BD0000014B1B680B607047E05E00201E
:102EA000024B33F820300B80704700BF105D0020CC
:102EB0002DE9F041083B164F162505FB03F57C195B
:102EC000D2F80080D2F804E0D2F808C0D268C4F882
:102ED0000680C4F80AE0C4F80EC0C4F8122000222C
:102EE000627101222271618078535909094803F007
:102EF0001F039A4050F82130134340F82130064810
:102F000050F821301A4340F82120BDE8F08100BF7D
:102F1000905E0020885E00208C5E002010B50C467C
:102F200000F108039BB20A1D49882088FFF7C0FF03
:102F300010BD0000F0B40B4D162303FB00F02C185D
:102F4000234653F806CF5F689E68DB68C1F804C06B
:102F50008F60CE600B612B5A0B8063884B80F0BC76
:102F6000704700BF905E002010B400EB800082002C
:102F7000064B134453F8044F58689A68DB680C609A
:102F800048608A60CB605DF8044B70478860002021
:102F900010B5044608B1A04710BD7846F4F7C6F84E
:102FA000F9E700002DE9F84307460C46904699469C
:102FB00005281AD80F4EFD00EA1B930033449B6985
:102FC0004A46414620469847ED1BAB001E447268B6
:102FD000610904F01F04012303FA04F452F82130BC
:102FE000234342F82130BDE8F8837846F4F79EF891
:102FF000E0E700BF44FB030010B5044670B10C4B82
:103000009C420FD3C8339C420FD8A3F1C800201AAA
:10301000084CA4FB0030C0F38F1010BD7846F4F7C5
:1030200085F8ECE74FF6FF70F7E74FF6FF70F4E72F
:10303000685F00201F85EB5138B5044608B10020B9
:103040000FE07846F4F772F8F9E7C82303FB00F3C2
:1030500003F12002144B13440233A34222D0013067
:1030600080B201281CD81049C82303FB001393F831
:1030700064100029E9D0C82303FB00F303F1200208
:10308000094B13440233A3420CD0C82303FB00F3C3
:1030900003F14002044B13440333A342DFD101E0A8
:1030A0004FF6FF7038BD00BFF85E002010B5044633
:1030B00090B1134B9C4203D303F593739C420FD9F9
:1030C000104B9C4216D318D8E01A0F4CA4FB0030CA
:1030D0000009083080B210BD7846F4F727F8E8E719
:1030E000A3F59370201A4008084CA4FB0030C0F3ED
:1030F0008F00F0E74FF6FF70EDE74FF6FF70EAE75D
:103100003C5D0020945E0020A38B2EBA310CC330AE
:1031100070B504460E461546106828B3FFF7C6FF83
:10312000013000E00130072820D84309114A52F845
:10313000233000F01F02D34013F0010FF2D00E4AEB
:103140002A2303FB00235B88A342EBD12A2303FB42
:1031500000235B79734013F03F0FE3D12A2303FB75
:10316000002304332B6003E00020DCE700232B6006
:1031700070BD00BF305D0020385D00202DE9F843B0
:1031800006460D461C4623482A2303FB04F3C118B8
:10319000D2F80090D2F80480D2F808E0D2F80CC03F
:1031A000C1F80690C1F80A80C1F80EE0C1F812C05B
:1031B000103303440020C3F80900C3F80D00C3F81E
:1031C0001100C3F8150005311046F9F7A5F9E8B963
:1031D00010492A2303FB04F3CA18002010719075CC
:1031E000CE52558063090C4904F01F04012202FAF3
:1031F00004F451F82320224341F82320074951F8D1
:103200002320144341F82340BDE8F8837846F3F7C0
:103210008DFFDDE7385D0020305D0020345D00204B
:10322000F8B505460C46164683B20A1D4988208823
:10323000FFF7A4FF242E05D0142E02D07846F3F712
:1032400075FFF8BD12492A2303FB05F3CA180120B4
:10325000907510331944204650F8147F46688468EE
:10326000C268C1F80970C1F80D60C1F81140C1F819
:1032700015200831F9F750F930B9054B2A2202FB25
:1032800005352B79EB75DCE77846F3F74FFFF4E76C
:10329000385D00202DE9F04106460C4615462422F3
:1032A000002120460BF079FF174F2A2202FB06F27D
:1032B000B9180B4653F8068FD3F804E0D3F808C0CA
:1032C000DB68C4F80480C4F808E0C4F80CC02361CB
:1032D000BB5A23804B8863808B7D23B92B88043BAA
:1032E0002B80BDE8F0812A2303FB06F606F11003CC
:1032F0003E461E4456F8095F7068B168F368656120
:10330000A061E1612362ECE7385D0020F8B5064674
:103310000C4615462422002120460BF03EFF1A4998
:10332000C82303FB06F3CA18CB5A238092F86430F3
:10333000A370134653F802CF5F689868DB68C4F83F
:1033400003C0C4F80770C4F80B00C4F80F3092F83B
:1033500064301BB92B88043B2B80F8BDC82303FBCA
:1033600006F606F11003084E1E4456F8025F706818
:10337000B168F368C4F81350C4F81700C4F81B1000
:10338000C4F81F30E9E700BFF85E00202DE9F041E6
:103390000D461446394BC82202FB04F202F16801C3
:1033A000194413445967064610B9354B01221A7067
:1033B000C82101FB04F12031304B19440231284669
:1033C000F9F7B5F800284CD1C82303FB04F3783390
:1033D0002A4919442846F9F7BDF8002845D1C823E1
:1033E00003FB04F39033254919442846F9F7DCF828
:1033F00000283ED1214FC82202FB04F2B818D5F8AC
:103400000080D5F804E0D5F808C0E968C0F802806B
:10341000C0F806E0C0F80AC0C0F80E1002F11001B2
:1034200039440023C1F80230C1F80630C1F80A302F
:10343000C1F80E30BE5280F864306309114904F0BF
:103440001F04012202FA04F451F82320224341F818
:1034500023200D4951F82320144341F82340BDE8AF
:10346000F0817846F3F762FEAEE77846F3F75EFE4A
:10347000B5E77846F3F75AFEBCE700BFF85E0020D8
:10348000DC5E0020F05E0020F45E0020F8B505460A
:103490000C46164682B203312088FFF777FFA278E8
:1034A0001949C82303FB051383F864202AB3242E8B
:1034B0001BD11549C82303FB05F303F110020A448D
:1034C000204650F813CF47688668C468C2F802C027
:1034D000C2F80670C2F80A60C2F80E4040331944C0
:1034E0000331F9F724F820B9F8BD7846F3F71EFE4A
:1034F000DFE77846F3F71AFEF6E7142EF4D07846A5
:10350000F3F714FEF0E700BFF85E0020F8B5A1F174
:103510000804A2002244950011492944076846681E
:103520008568C3684F608E60CD600B61F9F764F801
:1035300090B963090B4904F01F04012202FA04F454
:1035400051F82320224341F82320074951F8232032
:10355000144341F82340F8BD7846F3F7E7FDE8E768
:1035600088600020085D00200C5D002008B50B4637
:1035700000F1080189B21846FFF7C8FF08BD000036
:1035800008B5064B00221A700548F9F797FE00B9F6
:1035900008BD0448FAF7E0F8FAE700BFA65E00208D
:1035A000A85E002084330020F8B504460D46F7F7E6
:1035B000FFFF052C1ED81E4B1E78FEB1E200121B29
:1035C00091001C4B0B44998929441A6989B21A4805
:1035D000F9F76BFF074688B1C4EBC404A200154B92
:1035E00013445B690246011D284698473846F9F79F
:1035F00095FF18E07846F3F799FDDCE7C4EBC404C7
:10360000A2000C4B13449A68690905F01F050123B9
:1036100003FA05F552F821302B4342F821300748D0
:10362000FAF79AF80026F7F7E3FF3046F8BD00BF37
:10363000A65E002044FB0300A85E0020CC5E0020B4
:1036400010B50A2201210A48F9F72FFF002814BFFC
:103650000124002409D0082343818381022282802F
:10366000C38001230381F9F759FF204610BD00BF35
:10367000A85E002070B504460E46F7F799FF052CAA
:1036800029D8174B1D7875B1C4EBC4039A00154BAC
:1036900013449989314489B21348F9F767FFB0FAA6
:1036A00080F56D099DB9C4EBC404A2000D4B134411
:1036B0009A68710906F01F06012303FA06F652F80C
:1036C0002130334342F821300848FAF745F8F7F73C
:1036D0008FFF284670BD7846F3F728FDD1E700BF7D
:1036E000A65E002044FB0300A85E0020CC5E002004
:1036F0002DE9F84F00264FF0010818E0A4EB421125
:1037000001238B40013B55F8221019421ED1013292
:1037100004F11F035B099A4205D2013B9A42EDD0A6
:103720004FF0FF33EFE7434693B10136F6B2052E73
:1037300042D8B8F1000F3FD037462049F3009B1B19
:103740009A008B189D688C580022E1E70023EBE774
:103750004FF000090FE049463046FFF78BFF48B3B2
:10376000012303FA0BFB55F82A3023EA0B0345F833
:103770002A3009F101094C45D7D94FEA591A55F8B1
:103780002A3009F01F0B23FA0BF313F0010FF0D0CE
:10379000C7EBC7039A00094B13445B6853F82A3000
:1037A00023FA0BF313F0010FD5D049463046FFF74B
:1037B000FBFED4E78046B8E7BDE8F88F44FB030082
:1037C00038B5072828D84409334951F8243000F087
:1037D0001F0223FA02F515F0010F1DD02F4D05EB46
:1037E0008005AD78002D4ED12C4D05EB8005ED7890
:1037F0000DB100204AE0012505FA02F223EA020396
:1038000041F824300024254B23F820400146284667
:10381000FFF730FF204639E0A0F108039BB2072BE9
:1038200033D859091E4A52F8212003F01F0322FA07
:1038300003F313F0010F2AD0A0F1080101EB81037B
:103840009A00184B13449B781BBB164B1344DB7830
:103850000BB100201AE04C09114801F01F020123AE
:1038600003FA02F250F8243023EA020340F824302D
:1038700001EB8102930000240A4AD4520220FFF790
:10388000F9FE204602E0002000E0052038BD0520BA
:10389000FCE70020FAE700BFF85C0020105D002084
:1038A000085D00208860002030B58DB005460C46CC
:1038B000012905D0022C07D0032C09D00DB030BD52
:1038C0007846F3F733FCF5E77846F3F72FFCF3E798
:1038D0002C22002101A80BF060FC10238DF804308D
:1038E00002238DF808300395044BDA6805921B69B2
:1038F000069301A8F4F7D6FFE0E700BFA85E00201A
:1039000008B511460020FFF7CFFF08BD08B50846EF
:103910001146FFF7C9FF08BD70B505460C461646AF
:103920004FF6FF730B80F6F737FC3070022823D078
:10393000032841D0012841D0002070BD03EB830152
:103940008A0020498A5AAA4213D00133072B15D87E
:1039500021884FF6FF729142F0D15A091A4951F865
:10396000222003F01F01CA4012F0010FE6D123808C
:10397000EBE723800120E0E70023E7E70020DCE716
:10398000124A32F82320AA4213D00133072B17D84A
:1039900021884FF6FF729142F2D15A090C4951F831
:1039A000222003F01F01CA4012F0010FE8D123804A
:1039B000EBE723800120C0E70023E7E70023E5E7EA
:1039C0000020BAE788600020085D0020105D00201C
:1039D000F85C002000293CD070B582B00E46144639
:1039E00005460DF1070201A9FFF796FF1CB99DF8E6
:1039F0000730032B2FD1012C1BD068B9BDF8041060
:103A00004FF6FF73994228D02846FFF713FABDF806
:103A100004100120FFF7C8FDBDF80430338084B1E5
:103A20000F4A02EB83039A7801329A70002002B0A9
:103A300070BD9DF80730032BDFD0012BDDD01020A7
:103A4000F5E7074A02EB8303DA780132DA700020E7
:103A5000EDE70E2070471020E9E70420E7E700BFFC
:103A6000105D002070B506460D464FF6FF730B80C3
:103A700000240BE004EB8402930010481844102249
:103A8000314604300BF02AFB98B10134072C13D8CF
:103A900063090B4A52F8233004F01F02D34013F09D
:103AA000010FE7D12A884FF6FF739A42EDD12C809F
:103AB000EBE72C80012000E0002070BD8860002032
:103AC000085D0020F0B583B04FF6FF73ADF8063007
:103AD00000283AD00746002939D015460C460DF18A
:103AE0000601FFF7BFFFBDF8063003F10806B6B2C6
:103AF00060B94FF6FF7293422BD031463846FFF73C
:103B000005FDBDF806100220FFF74EFD268075B1B9
:103B1000BDF80600104A83001C18A1000C46114491
:103B2000897822444B1C9370002003B0F0BDBDF88F
:103B30000600094A83001C18A1000C461144C978EC
:103B400022444B1CD3700020EFE70E20EDE70E203F
:103B5000EBE70420E9E700BF8860002030B583B0C0
:103B600005460C46486820B10DF10601FFF77AFFC3
:103B700018B94FF6FF73ADF806300DF1060128466F
:103B8000FFF726F80246A8B1BDF8063003EB830321
:103B900099000B4B0B44DB787BB1658002232370CB
:103BA000BDF8061001EB810101FA03F0044B034458
:103BB00004336360104603B030BD0022FAE700BF53
:103BC0008860002000B583B0488003230B70002379
:103BD0004B60A0F57F43FC3B032B17D8DFE803F0D5
:103BE0000402071A002016E0FCF742FD13E06946C4
:103BF0004FF4C870F7F7E7F920B90198003018BF03
:103C0000012008E07846F3F791FAF6E76946FEF7F7
:103C1000ABFF00E0012003B05DF804FB70B5F9F7DD
:103C2000B3FD28B9F7F78EFD0028F8D020BFF6E7DE
:103C3000344B187800B970BD01213348F9F768FB9F
:103C4000044600285BD04389082B02D18389082BC6
:103C500003D0FFF795FC0020EDE7C388082BF8D1CF
:103C60000389012BF5D18388022BF2D1002519E0BD
:103C7000002B36D0B3F5805F2ED1012000E0032069
:103C80006988C0EBC0039A00204B13449E892B889F
:103C900003F57F533F339B009BB22A1D891BFFF71F
:103CA00081F93DB32A4600211748F9F758FB05462C
:103CB0000028F6D08442F4D0428802F47043B3F571
:103CC000005F13D0D4D9B3F5804F11D0B3F5A04F16
:103CD0000AD0B3F5405FD2D07846F3F727FA002038
:103CE000CEE7023AD0B2CBE70520C9E70220C7E70A
:103CF0000420C5E7064B186800F001009BE7002090
:103D000099E700BFA65E0020A85E002044FB0300E8
:103D1000005D002008B5F5F7BFFDA0F5805008BD97
:103D200010B586B0164B0393164B0493164B0593B0
:103D300000230293FFF7EEFF009001230193F7F7B2
:103D400037FC69461148F9F7C1FC50B90F4B1B7895
:103D5000012B0CD0F7F74CFC0D4B01221A7006B06A
:103D600010BDF7F745FC0B48F9F7F6FCF7E7FFF74E
:103D700067FC0446F7F73CFC002CF4D0ECE700BFEE
:103D80000D39030001390300993D0300A85E0020AE
:103D9000A65E00209433002008B5FFF7C1FF08BDE0
:103DA00070B5002513E02149EB005B1B9A008E18CB
:103DB0008C581F346409A4002246002170680BF05F
:103DC000ECF922460021B0680BF0E7F90135052D2A
:103DD000E9D9002206E0164B03EB82030021D970DB
:103DE00099700132072AF6D9002308E09900194496
:103DF0008800104A02440021D17091700133072BD2
:103E0000F4D900230C4A13600C4A13600C4A136067
:103E10000C4A13600C4A13600C4A13600C4A13805E
:103E200053800C4A1370FFF7ABFB70BD44FB0300DB
:103E3000105D002088600020005D0020F85C0020FC
:103E4000085D0020F05E0020305D0020885E0020CC
:103E5000E05E0020DC5E002008B50848084B0360E7
:103E6000F6F754FB074B084A9A60084ADA60084B99
:103E700000221A70FFF754FF08BD00BFE45E002067
:103E800061490300CC5E0020912F0300F13603004E
:103E9000A65E002010B5044680B11C4B1B6813F0D1
:103EA000010F2ED1208863880344013B98422ADC0D
:103EB000F6F772F9012805D00B2025E07846F3F7D4
:103EC00035F9EAE720886388184480B2013880B267
:103ED000F6F762F9012801D00B2015E022680C4B9F
:103EE0001A600A4A136843F0010313600021084670
:103EF000FFF75AFB074A136843F0010313600020E1
:103F000002E00F2000E00B2010BD00BF005D00208C
:103F1000E05E0020045D002010B5044618B1044B9B
:103F20001B68236010BD7846F3F700F9F7E700BF80
:103F3000E05E002008B50122FFF74CFD08BD00003F
:103F4000072809D843091E4A52F8233000F01F02FF
:103F5000D34013F0010F13D1A0F108039BB2072B3C
:103F600010D85909174A52F8212003F01F0322FAEA
:103F700003F313F0010F01D0012304E0002302E05A
:103F8000012300E00023CBB1072807D80E4B03EB39
:103F900080008378013383700020704710B40838A4
:103FA0000A4A83001C18A1000C4611448978224457
:103FB0004B1C937000205DF8044B70470520704740
:103FC000F85C0020085D0020105D00208860002063
:103FD00008B50122FFF776FD08BD000038B50728B7
:103FE00009D843091A4A52F8233000F01F02D3407F
:103FF00013F0010F1ED1A0F108039BB2072B22D8AA
:104000005909144A52F8212003F01F0322FA03F33E
:1040100013F0010F19D0A0F108040F4AA3001D19D5
:10402000A9000D46114489782A444B1E9370FFF76E
:10403000C7FB38BD094B03EB80039A78013A9A70AD
:10404000FFF7BEFBF5E70520F3E70520F1E700BF2A
:10405000F85C0020085D002088600020105D0020D2
:1040600008B50022FFF7B6FC08BD08B50022FFF72F
:1040700029FD08BD072809D843091E4A52F82330F4
:1040800000F01F02D34013F0010F13D1A0F1080379
:104090009BB2072B10D85909174A52F8212003F078
:1040A0001F0322FA03F313F0010F01D0012304E0F0
:1040B000002302E0012300E00023CBB1072807D84A
:1040C0000E4B03EB8000C3780133C37000207047B0
:1040D00010B408380A4A83001C18A1000C46114489
:1040E000C97822444B1CD37000205DF8044B704704
:1040F00005207047F85C0020085D0020105D00205E
:1041000088600020002937D038B50A46072809D82A
:1041100043091C4951F8233000F01F01CB4013F034
:10412000010F1ED1A0F108039BB2072B26D85C0912
:10413000154951F8241003F01F0321FA03F313F07B
:10414000010F1DD00838114B81000D18AC00254619
:104150001C5B54802B4404335360022313700020F3
:1041600038BD14460A4B33F820005080F6F714F897
:10417000207000206060F3E70E2070470520EFE715
:104180000520EDE7F85C0020085D00208860002035
:10419000105D0020072809D843092C4A52F8233023
:1041A00000F01F02D34013F0010F13D1A0F1080358
:1041B0009BB2072B10D85909254A52F8212003F049
:1041C0001F0322FA03F313F0010F01D0012304E0CF
:1041D000002302E0012300E00023A3B310B582B066
:1041E00004466946FFF78EFF50BB9DF80030032B55
:1041F00003D0022B11D00F2023E0164B03EB8403D6
:10420000DB780BB905201CE0124A02EB8402013B6B
:10421000D3702046FFF7D4FA13E0A4F1080303EBB0
:10422000830291000C4A0A44D2780AB9052008E0BA
:10423000094B0B44013ADA702046FFF7C1FA00E05F
:10424000002002B010BD0520704700BFF85C0020C0
:10425000085D0020105D00208860002068B330B544
:1042600083B0054659B30C464088F5F795FF022800
:104270000ED0032803D0012801D0102020E02146D1
:104280006888FEF7D5FC08B1002019E0052017E08A
:104290004FF6FF73ADF80630686850B10DF10601B6
:1042A000FFF7E0FB38B1BDF806300833238000206B
:1042B00006E00E2004E0052002E00E2070470E20EC
:1042C00003B030BD10B404464FF6FF70002304E085
:1042D0004FF6FF72904216D00133012B15D85A09C0
:1042E0000E4951F8222003F01F01CA4012F0010FBD
:1042F000EED0C82202FB03F209498A5A9442EBD15C
:1043000098B2012302E098B2E6E7002313B15DF80A
:10431000044B70474FF6FF70F9E700BFF05E0020D6
:10432000F85E002018B108B5FEF786FE08BD4FF60E
:10433000FF70704700B583B00DF10601FEF7D8FCA1
:1043400020B1BDF8060003B05DF804FB4FF6FF7026
:10435000F9E718B108B5FEF7A9FE08BD4FF6FF70E2
:10436000704700000A4699B1072813D843090B4942
:1043700051F8233000F01F01CB4013F0010F0BD098
:104380002A2303FB00F0064B1B5A138000207047C2
:104390000E2070470520704705207047305D0020D3
:1043A000385D002008286AD800296AD038B50D4643
:1043B0000446072830D84309354A52F8233000F024
:1043C0001F02D34013F0010F5DD0324A2A2303FBB2
:1043D00000235B88012B17D82E4A2A2303FB0423D2
:1043E0005B8859092C4A52F8212003F01F0322FA56
:1043F00003F313F0010F0BD0264B2A2000FB0434EB
:1044000063882B80002038BD7846F2F78FFEE3E703
:104410007846F2F78BFEEFE7A0F1080462091F4B24
:1044200053F8223004F01F02D34013F0010F2CD0B8
:104430001B4A162303FB04235B88012B17D8184A59
:10444000162303FB04235B885909134A52F82120E1
:1044500003F01F0322FA03F313F0010F0BD0104BEC
:10446000162202FB043463882B800020CBE77846B9
:10447000F2F75CFEE3E77846F2F758FEEFE7052037
:1044800070470E2070470520BDE70520BBE700BF41
:10449000305D0020385D0020F05E0020885E002046
:1044A000905E0020002951D038B50D46002A4FD02B
:1044B000B0F5805F4ED24FF6FF731380002305E006
:1044C00014884FF6FF718C4216D00133012B15D89A
:1044D0005C09234951F8244003F01F01CC4014F03B
:1044E000010FEDD0C82101FB03F11E4C615A884237
:1044F000EBD11380012302E01380E6E70023294675
:10450000144605465BB11088164BC82202FB0030EA
:10451000102202300AF0E2FDF0B903201BE01288FD
:104520004FF6FF739A4219D0FEF730FF218803201F
:10453000FFF73AF82188C82303FB01F388330949C0
:1045400019442846F5F7EBFF002004E00E207047E1
:104550000E2000E0072038BD0F20FCE70420FAE71A
:10456000F05E0020F85E0020012812D843090B4AB3
:1045700052F8233000F01F02D34013F0010F0AD08D
:10458000074BC82202FB003090F864300B7000200B
:104590007047052070470520704700BFF05E00207F
:1045A000F85E0020002900F083802DE9F8430D46D5
:1045B00001287FD84609434B53F8263000F01F07E7
:1045C000FB4013F0010F78D004463F4AC82303FB99
:1045D000002393F864307BB1012B70D1C82000FB1D
:1045E00004F010301044102202300AF077FD08B9B0
:1045F000002060E008205EE03349C82303FB00F39D
:1046000003F110020A4402F10208D5F80090D5F82F
:1046100004E0D5F808C0E868C2F80290C8F804E0E1
:10462000C8F808C0C8F80C004033194403312846C4
:10463000F7F77DFF80BBC82303FB04F3A0332249B7
:1046400019444046F7F786FF50BBC82303FB04F329
:10465000B8331D4919442846F7F7A6FF20BB1A486E
:10466000C82303FB04F3C218012582F8645003F148
:10467000B0012A460144C05AF5F7E8FA134B05FA8F
:1046800007F753F826502F4343F82670214603209E
:10469000FEF78AFF00200EE07846F2F747FDCAE7F2
:1046A0007846F2F743FDD0E77846F2F73FFDD6E7CC
:1046B0000E2070470520BDE8F8830520FBE70820A1
:1046C000F9E700BFF05E0020F85E0020F45E0020F5
:1046D000012832D870B545091A4B53F8253000F03F
:1046E0001F06F34013F0010F29D0174AC82303FB1C
:1046F000002393F86430012B01D0082070BD0446DC
:104700001046C82303FB04F3D118022281F8642069
:1047100003F1B0010144C05AF5F798FA0B4A01239E
:1047200003FA06F652F82530334342F82530214685
:104730000320FEF739FF0020E0E705207047052041
:10474000DCE700BFF05E0020F85E0020F45E002091
:10475000012800F2CB802DE9F0474609664B53F85B
:10476000263000F01F07FB4013F0010F00F0C0805F
:10477000624AC82303FB002393F86430002B00F047
:10478000B980C82101FB00F1551801F11003134451
:1047900053F8028FD3F804E0D3F808C0DB68C5F8FB
:1047A0000280C5F806E0C5F80AC0C5F80E3001F170
:1047B0002003134440310A44D11C02332332D1F880
:1047C00000E0D1F804C08D68CC68C3F800E0C3F8FD
:1047D00004C09D60DC60103110339142EFD10A7843
:1047E0001A70464AC82303FB00F303F17801A03393
:1047F00013440A4403F12001D3F800E0D3F804C0C5
:104800009D68DC68C2F800E0C2F804C09560D4601E
:10481000103310328B42EFD1054619685B68116086
:1048200053603648C82303FB05F3C218002482F8FE
:10483000644003F1880122460144C05AF5F706FAA4
:1048400000E00134072C41D862092D4B53F8223087
:1048500004F01F01CB4013F0010FF2D029482A23A6
:1048600003FB04035B88AB42EBD12A2303FB040365
:104870009B7D002BE5D003462A2000FB04F003EBD0
:10488000000E1030034453F807AFD3F80490D3F868
:104890000880D868CEF804A0CEF80890CEF80C8036
:1048A000CEF810001B8AAEF8143000238EF81630B4
:1048B0001548012303FA01F150F822300B4340F868
:1048C000223021460420FEF76FFEBAE70F4A01238B
:1048D00003FA07F752F826303B4342F826302946C0
:1048E0000320FEF761FE0020BDE8F0870520704739
:1048F0000520F9E70820F7E7F05E0020F85E0020C9
:10490000305D0020385D0020345D0020F45E002022
:1049100070B504460D469DF81060FEF76DFB4FF62E
:10492000FF73984202D03034AC4200D070BD56B113
:104930000A4AC82303FB002393F86430012BF5D106
:10494000FFF7C6FEF2E7054AC82303FB002393F8EE
:104950006430002BEAD0FFF7FBFEE7E7F85E0020AB
:104960000378042B00D0704710B582B00446037E54
:10497000426981684068647E0094003318BF012357
:10498000FFF7C6FF02B010BD40B108B541B1FEF758
:104990000FFA08B1002008BD0920FCE70E2070477F
:1049A0000E20F8E792B3F0B583B0144683B31F46E8
:1049B0000E460546F5F7F0FB01282BD1012E2CD829
:1049C00073091A4A52F8233006F01F02D34013F03D
:1049D000010F24D00DF106012846FEF757F900BB60
:1049E000BDF806304FF6FF7293421CD02246314686
:1049F0002846FEF75DFABDF8061008390520FEF7D7
:104A0000D3FDBDF806303B80002004E00E20704747
:104A10000E2000E0102003B0F0BD0520FBE70520CC
:104A2000F9E70F20F7E70420F5E700BFF05E00206C
:104A3000AAB3F8B51746A3B3012934D84C091F4AC5
:104A400052F8244001F01F02D44014F0010F2CD082
:104A5000B0F5805F2BD21D460C4606461946FEF780
:104A600047F960B12888164B2A2202FB0030102239
:104A7000394606300AF032FBD8B9032014E02B88FF
:104A80004FF6FF72934216D03A4621463046FEF763
:104A900075FB29880420FEF787FD002004E00E2026
:104AA00070470E2000E00520F8BD0520FCE7072038
:104AB000FAE70F20F8E70420F6E700BFF05E0020D9
:104AC000385D0020002965D0F8B50F46072863D867
:104AD0004409344B53F8243000F01F05EB4013F029
:104AE000010F5BD030492A2303FB00135B882F4959
:104AF000C82606FB031393F86430012B50D10646F9
:104B0000294A2A2303FB00239B7D73B12A2303FB3D
:104B100000F31033104618441022394609300AF0C9
:104B2000DDFA002839D0082037E01F492A2303FB8B
:104B300000F3CA180120907510331944D7F800E02B
:104B4000D7F804C0B868FA68C1F809E0C1F80DC028
:104B5000C1F81100C1F8152008313846F7F7DCFC20
:104B6000A0B9114A2A2303FB06231A79DA75104AE1
:104B7000012303FA05F552F824302B4342F8243080
:104B800031460420FEF710FD002006E07846F2F7DB
:104B9000CDFAE6E70E2070470520F8BD0520FCE7BA
:104BA0000820FAE7305D0020385D0020F85E002024
:104BB000345D0020072818D838B544090D4A52F84A
:104BC000243000F01F0523FA05F111F0010F0ED07B
:104BD0000146012000FA05F523EA050342F82430D6
:104BE0000420FEF747FD002038BD05207047052052
:104BF000FAE700BF305D002001287BD82DE9F041A5
:104C00004509404C54F8253000F01F06F34013F0DE
:104C1000010F71D0236813B90223002114E05A4216
:104C20001340394A02FB03F3DB0E384AD35CF4E746
:104C300057423A40344F07FB02F2D20E334FBA5C70
:104C400002EB431300E00223022B19D001315F1C59
:104C5000012FF8D87B092B4A52F8232007F01F07B1
:104C60004FF0010C0CFA07F77F423A40002ADFD1DF
:104C7000013303D1234A52F82320F7E70223E3E765
:104C800001293CD08046002700E00137072F19D8C2
:104C90007B091F4A52F8233007F01F02D34013F05C
:104CA000010FF2D01B4A2A2303FB07235B884345ED
:104CB000EBD1B8B2FFF77EFF0028E6D07846F2F7D6
:104CC00035FAE2E7C82303FB08F3134AD35A13B9B2
:104CD000124B00221A70012303FA06F654F825300D
:104CE00023EA060344F8253041460320FEF7C2FCC0
:104CF000002002E0052070470520BDE8F0810F206C
:104D0000FBE700BFF05E002031B57C07ECFB030041
:104D1000305D0020385D0020F85E0020DC5E002061
:104D2000B1B10B46B2B1012816D810B541090C4CEF
:104D300054F8211000F01F04E14011F0010F0DD0D4
:104D40001946FEF705F808B1002008E0092006E042
:104D50000E2070470E20704705207047052010BDBB
:104D6000F05E0020082979D8002A79D030B40729CC
:104D70002ED8404C07292DD80B465D0954F8254004
:104D800003F01F0324FA03F313F0010F6AD04FF668
:104D9000FF73984221D0012867D84309364C54F854
:104DA000233000F01F04E34013F0010F5FD0072908
:104DB00033D8324CC82303FB004393F86430022BF2
:104DC0001BD02F4C2A2303FB0141043151602BE0FF
:104DD0002C4CCFE7A1F10803CFE7072905D82848D5
:104DE0002A2303FB01035888D5E7A1F108032648CD
:104DF000162404FB03035888CDE7214C2A2303FB28
:104E000001439B7D002BDCD02A2303FB01F11031F1
:104E100023460B440733536006E008391A4B162427
:104E200004FB0131043151601449C82303FB001312
:104E300093F86430022B09D0C82303FB00F0203024
:104E40000E4B03440233136000200CE0C82303FB25
:104E500000F040300B4603440333F4E7052070476D
:104E60000E207047052030BC70470820FBE7082063
:104E7000F9E700BF305D0020F05E0020F85E002002
:104E8000385D0020885E0020905E00200A46A1B1B7
:104E9000012814D843090C4951F8233000F01F01B0
:104EA000CB4013F0010F0CD0C82303FB00F070308F
:104EB000064B18441060002070470E2070470520F4
:104EC00070470520704700BFF05E0020F85E0020AC
:104ED00010B50C46FFF7F6F9B4B1012816D843090E
:104EE0000C4A52F8233000F01F02D34013F0010F98
:104EF0000ED0C82303FB00F000F12003064818443D
:104F000002302060002002E00E2000E0052010BDED
:104F10000520FCE7F05E0020F85E002070B5064634
:104F200015460C4659B175B1206880B1FEF784F87A
:104F30000130002323602B6006F07F011BE07846E0
:104F4000F2F7F4F8EFE77846F2F7F0F8ECE7002034
:104F5000EFE73BB12A4AC82303FB002393F8433011
:104F60008B4239D0264AC82303FB002393F8223012
:104F70008B423BD00130012840D84309214A52F8E6
:104F8000233000F01F02D34013F0010FF2D01C4A6F
:104F9000C82303FB002393F86430002BD9D01646B6
:104FA000C82202FB006292F822208A42D1D1C82294
:104FB00002FB006292F843208A42CAD13346C822DB
:104FC00002FB00F000F12002324402322260403045
:104FD000034403332B6011E0C82303FB00F303F108
:104FE0004002074B13440333236007E0C82303FB4D
:104FF00000F02030134603440233236070BD00BF2D
:10500000F85E0020F05E002070B504460E4615469E
:1050100062B17CB12046FEF70FF84FF6FF7398425D
:105020000CD02A463146FEF773F870BD7846F2F789
:105030007DF8EEE77846F2F779F8EBE700232B608E
:10504000F3E738B505460C4621B12846FDF7DAFEF0
:10505000206038BD7846F2F769F8F6E7F8B50546FE
:1050600017460E4639B157B1306800286FD0FDF7AA
:10507000C3FF441C0DE07846F2F758F8F3E7784692
:10508000F2F754F8F0E7012300E00023002B42D1AF
:105090000134012C5DD863092F4A52F8233004F003
:1050A0001F02D34013F0010FF2D02C4AC82303FB98
:1050B000042393F864307BB9002DE4D0C82303FBAC
:1050C00004F3883308222549194428460AF006F8D3
:1050D0000028DAD10123D9E7BDB1C82303FB04F3CB
:1050E000883308221D491944284609F0F7FF70B19A
:1050F000C82303FB04F3B033082218491944284697
:1051000009F0ECFF28B90123C0E70123BEE7012322
:10511000BCE70023BAE7124B1B784BB1C82303FB53
:1051200004F30E4AD35A0BB1002102E0012100E042
:1051300001210A4AC82303FB04F4131983F87010F1
:1051400070341444346093F864303B7003E00024FE
:105150009FE700233360F8BDF05E0020F85E00207A
:10516000DC5E002038B504460D46F5F715F8022838
:105170000FD0032808D0012801D0002003E02946E1
:105180002046FDF7CFFC38BD29462046FEF71AFD24
:10519000F9E729462046FEF7E1FCF4E700B583B0C5
:1051A0000378022B0ED0032B03D0012B01D0002358
:1051B00004E069464088FFF7D5FF0346184603B070
:1051C0005DF804FB69464068FEF74CFC0346002886
:1051D000F4D0BDF8003003EB83039A00034B134473
:1051E000DB78003318BF0123E8E700BF88600020A8
:1051F00038B50C46054630B129B1054B1A882A80CE
:105200005B88238038BD7846F1F790FFF5E700BF53
:10521000E05E0020034643B1A3F1080013F8082C18
:105220008A4203D012B11B68F5E70020704750B1E5
:10523000426852B14378073BDBB2F72B01D900201B
:105240007047072070470E2070470E20704710B53A
:10525000007848B9002404E0E0B200F099F8013485
:10526000A4B2FF2CF8D910BD00F092F8FBE70000C3
:10527000F8B50546FFF7DBFF044608B12046F8BD48
:10528000094E37682846FFF7E2FF05F1080130466E
:10529000F7F744FA002FF1D1002000F089F801203F
:1052A00000F066F8EAE700BF286100202DE9F84326
:1052B0000646884691461F460C4616E05B682178F4
:1052C0003A460139A01C984765B161782846FFF736
:1052D000A1FF034630B185684278B242EED0FF2A82
:1052E000ECD0F1E7237801331C4408EB0903A34217
:1052F00002D9024B1D68E7E7BDE8F883286100206A
:10530000F0B41A4B1E7BB6FA86F56D090021437D79
:10531000063BDBB28B421ADD4218577F4A1C02441F
:10532000527F4FEA521C114C04EB8C04246902F0AA
:105330001F0224FA02F212F0010F02D101373944A0
:10534000E5E75B1A9F420ADA351C18BF01251DB13B
:10535000064A536B013353632846F0BC7047034A37
:10536000136B013313630125F6E700BF2C610020A6
:1053700008B518B9044800F021FE08BD0248034BE7
:10538000036000F005FEF8E72C61002001530300E4
:105390004109064A00F01F00012303FA00F052F809
:1053A0002130034342F82130704700BF3C610020A8
:1053B00010B50446012802D97846F1F7B7FE014B33
:1053C0001C7310BD2C61002010B5044648B1E36F7A
:1053D0005BB1E36FD4F89820D4F894102046984736
:1053E00010BD7846F1F7A2FEF1E77846F1F79EFE90
:1053F000EFE710B50446037813F0FE0301D0022B4B
:1054000005D1237803F0FE03022B04D010BD7846AB
:10541000F1F78CFEF5E7A37963F03F03A371F5E79D
:1054200010B582B0044628E0002002B010BD7846D6
:10543000F1F77CFE26E004F15C00F3F722FC08B1F2
:10544000012324E0002322E0012300E0012333B301
:10545000616831B1043904F15C00F3F729FC0023E1
:10546000636001A904F15C00F3F7DAFB0028DBD1EB
:10547000019B1A1D62600C3363626368002BE7D0E6
:10548000002BD4D063681B79FF2BD4D00023626833
:105490001279002BDAD1002AD6D00023D7E70120D9
:1054A000C3E7000070B5064643682BB106F17405EA
:1054B0002B79DBB1002405E07846F1F737FEF5E7FC
:1054C0000134E4B2EB789C4210D21348F5F70CFD9E
:1054D000EA78B0FBF2F302FB1300C3B2A342EFD0B1
:1054E0002B5DC0B22A5C2A552B54E9E774682379F6
:1054F00053B12379FF2B01D0013B237106F1080042
:1055000000F00AFD20B970BD7846F1F70FFEF0E714
:105510007846F1F70BFEF6E7646100200B78002B6C
:1055200036D070B50C4691F8403053B9CB6F33B1DB
:1055300001F18000F6F7FCF8E0B1012300E0002360
:10554000D3B104F14405266F94F84430DBB2062B46
:1055500002D07846F1F7EAFD0F48F5F7C5FC0F4B8E
:10556000A3FB00235B0B42F2107202FB13033344D4
:10557000EB6070BD0023E3E72046FFF751FF0546CF
:1055800010B9002DF5D0DCE72046FFF78BFFF8E7D8
:1055900000230B65704700BF646100205917B7D125
:1055A00010B5044650F8202C1379013BDBB2FD2BDB
:1055B00008D9836D33B11368036741675C30F6F730
:1055C00095F820B954F8201C0B7923B110BD78460A
:1055D000F1F7ACFDF6E744F8203C043904F138005B
:1055E000F3F766FBF2E7000008B50248F5F7B6FCF2
:1055F00008BD00BF646100200378E3B970B50446BC
:1056000001230370436883B104F14406256F0A48FF
:10561000F5F76AFCB0FBF5F405FB1404F5F726FB7F
:1056200021183046F5F786FA70BD5C30F3F719FBA8
:105630000028E9D1F8E770476461002030B583B0F5
:105640000C46054678B11F2C11D804F1110292B214
:1056500001A905F15C00F3F783FA60B1042826D1B3
:10566000002003B030BD7846F1F760FDEBE77846E7
:10567000F1F75CFDE9E7019B181DE4B206345C73A9
:105680001A7B022161F303021A7395F86820C2F3B2
:105690004002197B62F38611197355F8692FC3F81C
:1056A0000F20AA88A3F8132000225A60D9E7784671
:1056B000F1F73CFD0020D4E770B505460C4611B368
:1056C00008B323791BB3237A03F0CF036FF3C71317
:1056D00023720023A37234F8042C211F05F15C000F
:1056E000F3F76DFA2B78D3B195F84430ABB195F858
:1056F0004430DBB2042B13D095F84430DBB2052BD9
:1057000009D001230AE07846F1F710FDD9E7784681
:10571000F1F70CFDD7E7002300E0002313B170BDC3
:105720000023FBE705F144062D6F0748F5F7DCFB86
:10573000B0FBF5F405FB1404F5F798FA2118304690
:10574000F5F7F8F9EBE700BF6461002038B50446CF
:105750000D4631B128B1291F04F15C00F3F7A8FA16
:1057600038BD7846F1F7E2FCF5E7000038B50D46A4
:105770000446C0B1132D1AD9B5F5205F1BD84FF4DC
:105780007A7000FB05F5256794F84430CBB194F8A6
:105790004430DBB2042B19D094F84430DBB2052B33
:1057A0000DD001230EE07846F1F7C0FCE2E7784621
:1057B000F1F7BCFCE0E77846F1F7B8FCDFE700233F
:1057C00000E000230BB1237813B938BD0023F9E7BB
:1057D00044340748F5F788FBB0FBF5F305FB1305E8
:1057E000F5F744FA29182046F5F7A4F9EDE700BFCC
:1057F0006461002038B50D46044610B184F8285085
:1058000038BD7846F1F792FCF8E710B504465C30F5
:10581000F3F77DF9EFF3108272B663680BB10021E4
:10582000197102B962B610BD10B504464FF080532D
:10583000D3F8A03013F0010304D093B97846F1F700
:1058400075FC03E003786FF347030370084B186897
:10585000C4F801009B88A4F805302046FFF7C9FD75
:1058600010BD0378012262F347030370EEE700BF27
:10587000A4000010F8B50D4617461E46044688B130
:1058800082B10A2E12D9B2B2394604F15C00F3F7A4
:10589000E7F804F16800FFF7C7FF44F620632367C9
:1058A00000230EE07846F1F741FCEAE77846F1F78D
:1058B0003DFCE8E7154AD15CE21882F87410013328
:1058C000DBB2022BF6D984F87730002284F87820F6
:1058D0000F49216325216185032184F82C1084F868
:1058E000282004F17401A16384F83C30094B636300
:1058F0006262E567084BE364646522702DB122465D
:10590000064904F18000F5F7D7FEF8BD0CFC030052
:10591000D6BE898EA15503001D550300C95303004F
:10592000084B01225A60DA604FF0FF32C3F80823B7
:105930000022C3F80022044B4FF48062C3F8802198
:10594000704700BF00A0004000E100E0044B4FF0B2
:10595000FF32C3F80823034B0222C3F880217047AB
:105960000010004000E100E008B5054B1B7803B9CA
:1059700008BD00F029FE024B00221A70F8E700BFB4
:105980008561002010B5FFF7CBFF1A4B0022C3F84A
:1059900040210121C3F840150420C3F81005C3F8C5
:1059A0000425C3F80825144A1448C2F86005A0F578
:1059B00003503838C2F864054FF48060C2F804051B
:1059C00019600C4BD3F84031002BFAD0094C00235E
:1059D000C4F84031084B4FF48062C3F80825F5F74E
:1059E00007FD074BD3F848351844D4F84035C01AA2
:1059F00010BD00BF00A0004000F0014040A10040E9
:105A00000080004008B5074B1B7803B108BDFFF7C5
:105A10009DFF044B01221A70FFF7B4FF00F0BEFD9A
:105A2000F4E700BF8561002038B5F5F7CBFC00B185
:105A300038BD1248F4F7C4FD054668B10468F5F7AF
:105A4000DDFC1CB1E3686433834207D3B0F5FA7F11
:105A5000EED9FFF7D7FFEBE70024F0E7FFF784FF6D
:105A60000648F4F798FD854202D07846F1F75EFBD0
:105A700000236361204600F025F8D9E77861002013
:105A800008B5F5F7F3F80C4B1B68C01A00280BDAC1
:105A90000020F5F703FD094B00221A60084B1B7824
:105AA00033B9FFF7C1FF08BD7846F1F73FFBEFE7D9
:105AB000F5F7E0FCF7E700BF806100208861002077
:105AC0008661002070B505460120F5F7E7FC0D4C16
:105AD0002560FFF73BFFFFF755FF2368DA680244B4
:105AE00009490A60094C00262670094D01222A70D6
:105AF0001A68196990472E70237803B970BDFFF7B3
:105B0000BFFFFBE7886100208061002074610020F6
:105B10008461002010B5124B1B68B3B19B686BB158
:105B2000104C012323700E4B1B689A68186990472C
:105B3000002323700C4B1B7823B910BD7846F1F776
:105B4000F5FAEDE7FFF79CFFF7E7084B1B7813B179
:105B500000F058FDF1E77846F1F7E8FAF8E700BF02
:105B6000886100208461002074610020856100202C
:105B700008B50948F4F7E8FC0023084A1360084A0E
:105B80001370084A01211170074A1370074A1370F5
:105B9000074A82F80A3308BD786100208861002036
:105BA00085610020866100208461002074610020EE
:105BB00000E100E0064B1B783BB110B50024044B1C
:105BC0001C70F5F745FC204610BD0820704700BF4B
:105BD0008661002008B5064B1B7833B9044B0122BF
:105BE0001A70F5F735FC002008BD0820FCE700BF5F
:105BF0008661002010B50446C0B12368D3B1E368C4
:105C0000E3B1E268154B9A421CD86369A34221D0E4
:105C1000646104F114011248F4F7A1FC114B1B78E4
:105C2000D3B9114B1B688BB1002016E07846F1F711
:105C30007DFAE2E77846F1F779FAE0E77846F1F79E
:105C400075FADEE77846F1F771FADEE7F5F700FC62
:105C5000002002E0082000E0002010BDA086010026
:105C600078610020866100208861002008B50F4B14
:105C70001B6863B1F5F7E6FB68B10D4B1B7873B990
:105C80000C4B1B787BB10A4B01221A7008BD784679
:105C9000F1F74CFAEEE77846F1F748FAEDE7784687
:105CA000F1F744FAECE7FFF7EBFEEFE7886100203D
:105CB000746100208461002010B5F5F7C3FB90B13A
:105CC000134B1B68D3B15B688BB1124C012323705B
:105CD0000F4B1B685A6818699047002323700E4BBE
:105CE0001B7843B910BD7846F1F720FAE8E778460B
:105CF000F1F71CFAE9E7FFF7C3FEF3E7074B1B7860
:105D000013B100F06BFCEDE77846F1F70FFAF8E716
:105D1000886100208461002074610020856100207A
:105D200008B5F5F78FFB18B1054B1B6823B108BD0B
:105D30007846F1F7FBF9F7E7FFF776FEF7E700BFE4
:105D40008861002008B5F5F77DFB70B1094B1B6831
:105D500013B17846F1F7EAF9074B4FF480621A6005
:105D600002221A60FFF760FE08BD7846F1F7DEF9FF
:105D7000ECE700BF8861002000E100E008B5F5F71E
:105D800061FB88B10A4B1B6813B17846F1F7CEF975
:105D9000FFF7EAFDFFF7C4FDFFF7D8FD054B4FF411
:105DA0008062C3F8802008BD7846F1F7BFF9E9E7C3
:105DB0008861002000E100E0064B074AC3F8602537
:105DC00002F50F423C32C3F864254FF48062C3F8F9
:105DD0000425704700F001400411004070B50546ED
:105DE000254BD3F81031CBB1234B0022C3F810213F
:105DF000224C23780133237000F0F2FD95F8342013
:105E000023789A420ED39A422AD92A6BD05C00F0AA
:105E10001FF9194BD3F810314BBB70BD7846F1F721
:105E200085F9E1E7164BD3F84065164B1B681E4415
:105E3000F4F71CFF0446EB6A314605F11C00984755
:105E4000F4F714FF001B502802D47846F1F76EF9DE
:105E500000F000FEFFF70AFF002385F83830DCE78A
:105E6000054B0322C3F8002200F0CAFDD1E77846B3
:105E7000F1F75CF9D1E700BF00100040906100200D
:105E800000A000408C61002038B505460C46FFF7A5
:105E900093FF00F0BDF804F1200000F0EDF80021C0
:105EA000A06A00F039F9236B187800F0D1F80121CD
:105EB000154B1970154B1D60E269154BC3F804258D
:105EC0000022C3F810211022C3F80423114A5164A0
:105ED0001960D2F84405084400F038FD94F83430D5
:105EE000012B0AD90A4B0722C3F80022226B064B6A
:105EF0001B78D05C00F0ACF838BD054B0322C3F82A
:105F0000002200F07DFDF7E7906100208C61002009
:105F10000010004000A0004010B50446C36A1BB347
:105F200094F838305BBB174B2360174B6360E36911
:105F300094F8341094F824205B780C33042A17D09A
:105F40001248825C03FB02F32E3303FB01F3983308
:105F5000E3602461012384F838302046FFF74AFECD
:105F6000034638B9184610BD7846F1F7DFF8D7E791
:105F70000133E5E77846F1F7D9F80023F2E711237A
:105F8000F0E700BF895E0300DD5D030010FC030045
:105F900010B5044638B123684BB104F10801064836
:105FA000F6F7BCFB10BD7846F1F7C0F8F3E778468A
:105FB000F1F7BCF8F1E700BF9861002010B5044686
:105FC00028B104F108010448F6F7D3FB10BD784668
:105FD000F1F7ACF8F5E700BF9861002038B5054649
:105FE000094B1C684CB154F8083C54F8041C284672
:105FF0009847034630B92468F4E7044A136801332C
:1060000013600023184638BD986100209461002079
:106010000D4B0022C3F8FC2F0122C3F8FC2F40F2E5
:106020005B62C3F8382540F20312C3F83425074AEF
:10603000C3F83C259622C3F84425D3F8502642F0F5
:106040000102C3F850267047001000405555550016
:1060500010B50446272807D8054B1A5D054BC3F831
:106060000825C3F8544510BD7846F1F75FF8F3E70B
:1060700018FC03000010004010B5044688B32379D3
:10608000052B32D86388002B33D063880233B3F5F5
:10609000817F32D823781F4AC2F80C352379C2F8A1
:1060A0001035A37843F0007343F44033C2F8183539
:1060B0006388252B25D90823C3F10802120402F4B2
:1060C0007022134343F48073124AC2F81435D2F895
:1060D000143543F48013C2F814352379042B12D0FD
:1060E00010BD7846F1F722F8C9E77846F1F71EF8B7
:1060F000C8E77846F1F71AF8C7E77846F1F716F8D7
:10610000C8E70623D8E7D2F8143543F08073C2F805
:106110001435E5E70010004038B504460D46124B33
:10612000D3F81835C3F30243032B06D14DB1012D2B
:106130000FD07846F0F7FAFF0AE07846F0F7F6FF5E
:10614000F4E7220E084BC3F824252402C3F81C45AB
:1061500038BD230C03F47F43034AC2F824352402DC
:10616000C2F82045F4E700BF00100040074B0022B2
:106170001A71EFF3108272B65B781BB1044B0221E7
:10618000C3F8001102B962B6704700BF9C610020DD
:1061900000E100E00D4A53790133DBB2537192F80C
:1061A0002F20934202D3094B00225A71074B02223F
:1061B0001A71EFF3108272B65B781BB1044B0221A7
:1061C000C3F8001102B962B6704700BF9C6100209D
:1061D00000E100E030B482B0114B1B68ADF8043030
:1061E0001B0C8DF80630002203E000239BB1013226
:1061F000D2B28A420ED20023022BF6D8855C02ACC2
:106200001C4414F8044CA54202D00133DBB2F3E77E
:106210000123EBE70123184602B030BC704700BFF2
:1062200040FC030010B5FFF7F3FE1C48FFF724FF06
:1062300000241B4BC3F8304500E00134072C13D871
:1062400004F10A03174A02EB830398680028F4D08C
:106250002146FFF761FF1249D1F830350122A240F3
:106260001343C1F83035E8E70D4B0822C3F8042387
:106270001122C3F800220022C3F8042103F5F033F1
:10628000094AC3F8602502F5DE424432C3F86425AA
:106290004FF48062C3F8042510BD00BFB861002030
:1062A000001000409C6100200411004008B5114B13
:1062B0009B6813B17846F0F739FF0E483C2200F195
:1062C00008018430F2F74CFC031E0CBF01200020B3
:1062D00009D008498A6901328A61003318BF012355
:1062E000044A937008BD034A926818320249C1F803
:1062F0000425F2E79C6100200010004010B51B4B04
:10630000D3F850357BB91A4C6379234493F82C00A9
:10631000FFF79EFEE37853B9FFF7C8FF60B9144B4F
:1063200001221A7110BD7846F0F700FFEBE7FFF786
:1063300079FF0022E270EFE70E4C012161640B4B04
:106340005960D4F84405084400F024FB00F058FBE1
:106350000023C4F84431084B4FF48062C3F8802115
:106360004FF40033C4F80433D9E700BF00100040F5
:106370009C61002000A0004000E100E008B5064B51
:106380001B791BB1022B02D8FFF7B8FF08BD784676
:10639000F0F7CCFEFAE700BF9C61002010B50C4B73
:1063A00001221A610022C3F80C210A4B996831B10D
:1063B0001C4603F18400F2F77BFC0023A360044B2E
:1063C000D3F85035002BFAD100F044FB10BD00BFCC
:1063D000001000409C61002008B50D4B1B79012B7B
:1063E00007D073B1022B0FD1FFF7D8FFFFF786FF5D
:1063F00008BDFFF75BFF0028FAD0064B01229A6028
:10640000F6E7FFF7CBFFF3E77846F0F78FFEEFE70D
:106410009C6100200010004008B5094B1B79012B3E
:1064200006D033B1022B07D1FFF7B8FFFFF766FFA5
:1064300008BDFFF7B3FFFBE77846F0F777FEF7E715
:106440009C61002008B5114B1B78012B05D0022B55
:1064500006D07846F0F76AFE01E0FFF79FFF08BD1F
:106460000B4BD3F85035032B0CD8DFE803F00208B0
:106470000508FFF783FFF2E7FFF7AEFFEFE7FFF74F
:10648000CBFFECE77846F0F751FEE8E79C6100208F
:106490000010004070B52F4B9C682F4BD3F8003490
:1064A00063B92C4A1369013313612A488168843027
:1064B000F2F7FEFB274B00229A6070BD251D627E1D
:1064C000244BDB8B9A4204D9224A5369013353612E
:1064D000EBE7214AD2F848355B426373D2F80834BF
:1064E0001C4E0A3306EB83039B68A360D2F8543535
:1064F00003F03F032373F4F77BFF184BD3F84835C1
:1065000018446060234653F81B2FC4F80F209B8863
:10651000A4F81330237EC3F38011A27B61F34702FA
:10652000A273C3F303036375F3680133F360D6F812
:1065300090320BB128469847627E064C1732A1680C
:1065400004F18400F2F73BFBD4F88000F5F792F8F1
:10655000B0E700BF9C6100200010004000800040B8
:1065600010B5F4F783FB0446094B9A6A596A8A42CC
:1065700008D001440748F4F7DDFA21460648F4F74D
:10658000D9FA10BD03F16800F4F7A4FAF5E700BFEB
:106590009C61002004620020EC61002010B5094CD1
:1065A000012363700023E370C4F89402FFF73AFEFE
:1065B0002378022B00D010BD2379002BFBD0FFF7EE
:1065C0009DFEF8E79C61002008B5034B00225A703D
:1065D000FFF7E4FE08BD00BF9C61002008B5084B32
:1065E000D3F80C3113B9FFF72DFF08BD044B00227F
:1065F000C3F80C21D3F80C31FFF74CFFF3E700BFD1
:106600000010004008B50A4BD3F8443163B1084B81
:106610004FF40032C3F808230022C3F84421D3F812
:10662000443100F0DDF908BD7846F0F77FFDEEE774
:1066300000A0004008B5094B1B7823B1074B1B781D
:10664000012B04D008BD7846F0F770FDF6E7FFF7A0
:1066500087FF024B02221A70F4E700BF9C61002002
:1066600010B5124B1B7823B1104B1B78022B04D0B2
:1066700010BD7846F0F75AFDF6E70C4C04F16800BF
:10668000F4F728FA04F15000F4F724FA01232370F8
:10669000EFF3108372B662781AB1054A0221C2F88C
:1066A0000011002BE4D162B6E2E700BF9C6100203C
:1066B00000E100E038B5054698B10C4C291F04F103
:1066C0008400F2F7F5FAA37853B1EFF3108372B6B2
:1066D00062781AB1064A0221C2F8001103B962B603
:1066E00038BD7846F0F722FDE7E700BF9C61002047
:1066F00000E100E000B583B001A90A48F2F790FA82
:1067000060B901980430FFF769FC20B101980430AA
:10671000FFF7D0FFF0E70198043000E0002003B05D
:106720005DF804FB2062002008B50248F2F799FAF0
:1067300008BD00BF20620020024B83F82000012228
:10674000DA7070479C61002038B504460D468842D7
:106750000FD30F4B9C4210D840F6B7339D4210D94F
:106760000C4B9C625D625C67DC651B78022B0CD075
:1067700038BD7846F0F7DAFCEBE77846F0F7D6FC60
:10678000EAE77846F0F7D2FCEAE7FFF7E9FEEFE741
:10679000000071029C61002070B506460C464B1E3D
:1067A000DBB2022B10D821463046FFF713FD78B13B
:1067B000094D2246314605F12C0008F0C5FC0023A6
:1067C0006B7185F82F4070BD7846F0F7AFFCEAE7B3
:1067D0007846F0F7ABFCEBE79C610020F8B5074684
:1067E0000E464B1EDBB2072B0FD80A4C04F13005C6
:1067F00020220021284608F0D0FCB2003946284665
:1068000008F0A2FC0123E370F8BD7846F0F78EFC97
:10681000EBE700BF9C61002000B583B00D4B1B6807
:10682000ADF804301B0C8DF80630032101A8FFF7EA
:10683000B3FF02A8084B40F8083D0121FFF7CEFF47
:106840000320FFF779FF05480146FFF77DFF03B0FE
:106850005DF804FB40FC0300D6BE898E80841E00D8
:1068600038B50546104C4FF426720021204608F03A
:1068700094FC4FF4007204F1900104F18400F2F7EB
:10688000EFF8FFF7C9FF002323772523E383074BA6
:106890002367074BA3650123237023712846F4F770
:1068A000C9FEC4F8800038BD9C6100206D61030002
:1068B00095610300037813F0020F0BD04FF0031320
:1068C0000278920843EA022301F5A271024A42F8D3
:1068D00021307047014BF3E70060004003001300D4
:1068E00010B400230B600B4B9C780B4804F1A20200
:1068F00040F832101B799B0003F1804303F5C0433D
:1069000000EBC20253600123A340C0F804355DF8D8
:10691000044B70473464002000F00140037813F00A
:10692000010F0AD013F0020F08D103789A0801234F
:1069300093404FF0A042C2F8083570479A080123EF
:1069400093404FF0A042C2F80C3570470E4B5B7974
:1069500023B10D4B1B7813F0010F00D1704770B5B8
:106960000C460546084EB1783046FFF7A3FF0749AD
:1069700001EB84013046FFF7B3FF163504F5A8712B
:10698000034B43F8215070BD3464002040A1004007
:1069900000A000400F4B5B7923B10E4B5B7813F0E6
:1069A000010F00D1704770B50C460546094B5E1CBF
:1069B00099783046FFF77EFF074901EB84013046A6
:1069C000FFF78EFF163504F5A871044B43F82150EC
:1069D00070BD00BF3464002040A1004000A0004012
:1069E000054B5B7933B1044B9A7801239340034AFA
:1069F000C2F80835704700BF3464002000F0014041
:106A0000104B5B79E3B110B40F4B0022C3F8102197
:106A10000C4BD8780D4900F1A2020D4C41F83240E0
:106A20001B799B0003F1804303F5C04301EBC202D5
:106A3000536001238340C1F804355DF8044B70476F
:106A4000704700BF346400200010004000F0014097
:106A5000101100400F4B5B7903B9704710B50D4C16
:106A6000A378012202FA03F3E1788A4013430A4A29
:106A7000C2F80835237903F5A273A2F5C8320021C4
:106A800042F823102046FFF749FF601CFFF746FF3E
:106A900010BD00BF3464002000F001400369C268EB
:106AA000934202D99B1A581E70478068801A03448B
:106AB000581E70472DE9F041054688461646C768BE
:106AC0008468E41B94420ED840682246384408F09B
:106AD0003BFB361B324608EB0401686808F034FBC8
:106AE000EE60BDE8F0814068384408F02DFB3E447C
:106AF000EE60F6E72DE9F843064688461746C56876
:106B00004FF000091AE0B268641B1444621EB368B7
:106B10005C1B944228BF1446BC4228BF3C467068A8
:106B200022464146284408F00FFBA144A0443F1BE5
:106B30002544B368AB4207D0F5603FB13469A54244
:106B4000E1D2641B621EE2E70025F5E74846BDE896
:106B5000F8830000114B02221A615A6110499961B1
:106B6000104ADA614FF480621A6200229A625A6215
:106B7000DA6299640C49D964802119659A655A656D
:106B8000DA650A4A1068C3F80700094A92E8030068
:106B90001860998020229A71704700BF3C640020E1
:106BA00044FC030034650020B464002050FC030062
:106BB00054FC03002DE9F047054688469146234BD7
:106BC0001B78C3B16A002A44D100204B0B449F6D4F
:106BD0005C6DA74212D80026E41B4C4528BF4C46EA
:106BE00034BB2EB105EB4500C200184B13449F6522
:106BF0003046BDE8F087FFF7ADFFE3E7134B03EB4B
:106C0000010ADAF85060F61B4E4528BF4E46DAF806
:106C10004C1032463944404608F096FAB044A9EB8D
:106C200006093744DAF85030BB42D5D10027D3E704
:106C300005EB4503DA00054B1344D96C2246394471
:106C4000404608F081FA26442744CAE73C64002005
:106C500010B50B46EFF311844FF0800181F31188DA
:106C60001946FFF7A7FF84F3118810BDF8B50F464A
:106C70001646194A431C03EB4303DD00154400EBA1
:106C80004000C3001A44D46A012C10D01CB1022C5D
:106C90001BD0002417E02846FFF700FF864212D8D9
:106CA000324639462846FFF705FF34460BE02846B2
:106CB000FFF7F4FE3446864228BF04462246394692
:106CC0002846FFF7F7FE2046F8BD32462846FFF774
:106CD00011FF0446F7E700BF3C640020F8B5054605
:106CE0000E461746094B1B786BB1EFF311844FF03A
:106CF000800181F311883A4631462846FFF7B6FFF6
:106D000084F31188F8BDFFF725FFEEE73C6400200F
:106D100000B583B001220DF107010020FFF798FFB5
:106D2000012804D19DF8070003B05DF804FB4FF083
:106D3000FF30F9E710B58268531C4468A34205D8B8
:106D40000468A1548360C3680133C36082684368E8
:106D50009A4200D010BD044601680069FFF7BEFFEB
:106D6000A368984203D04FF0FF33E360F2E70023BB
:106D7000A360EFE72DE9F84F80460F4615461E4603
:106D8000DDF828A00B9A0B464FF0010903E0B3FB96
:106D9000F5F309F10109AB42F9D2B14500D2B14690
:106DA00012F0010B18D1BAF1000F15D012F0020F3A
:106DB00002D0BEB1202400E02024BAF1000F0BD095
:106DC000CA4509D90AF1FF3A21464046FFF7B2FF0A
:106DD000D8F80C30002BF0DAD8F80C30002B33DB6D
:106DE000012407E03024E8E7B7FBF4F39D4205D81F
:106DF00005FB04F4012EF7D9013EF9E7B7FBF4F3E4
:106E000004FB1377114AD15C4046FFF793FFD8F893
:106E10000C30002B03DBB4FBF5F4002CEED1BBF1FE
:106E2000000F11D0BAF1000F0ED0BAF1000F0BD045
:106E3000CA4509D90AF1FF3A20214046FFF77AFFF7
:106E4000D8F80C30002BF0DABDE8F88F5CFC0300BA
:106E50002DE9F04782B00746894615469A460A9EB4
:106E6000DDF82C8081EAE173A3EBE173012402E0F9
:106E700093FBF5F301349D42FADD544500D25446AC
:106E800036B1B9F1000F02DB18F0040F00D0013E5B
:106E900018F0020F02D0BAF1000F03D018F0010F62
:106EA00000D1F6B9FB68002B18DBB9F1000F25DB28
:106EB00018F0040F29D1FB68002B0FDB08F0030347
:106EC000022B27D0FB68002B08DBCDF8048000964E
:106ED00053462A4649463846FFF74CFF02B0BDE804
:106EE000F087002EDED0A642DCD9013E20213846B4
:106EF000FFF720FFFB68002BF3DAD3E7C9F10009A5
:106F00002D213846FFF716FFD5E72B213846FFF72E
:106F100011FFD0E7BAF1000FD4D1002ED2D0002E4D
:106F2000D0D0A642CED9013E30213846FFF702FF2D
:106F3000FB68002BF3DAC5E7F0B599B006460C46BE
:106F4000154603AB13934023149300231593179016
:106F50001693A5E00027012203E047F00107013462
:106F600082B32378233B0D2B2AD801A151F823F0BB
:106F7000B96F0300C16F0300C16F0300C16F03004D
:106F8000C16F0300C16F0300C16F0300C16F030035
:106F9000B16F0300C16F03005B6F0300C16F03009B
:106FA000C16F0300A96F030047F002070134D7E760
:106FB00047F004070134D3E747F008070134CFE76F
:106FC0000022CDE72078A0F13001C9B2092906D806
:106FD000013402EB820253001A18303AF2E72E28ED
:106FE00002D00023217812E00134002394F800C07D
:106FF000ACF13000C0B20928F4D8013403EB8303AC
:10700000590001EB0C03303BF0E714F8011B6C292D
:10701000FBD06829F9D064294CD00FD9732954D0FA
:1070200017D9752924D12968081D28600968019796
:1070300000920A2213A8FFF79DFE2DE0582919D0CF
:10704000632922D0252927D1252113A8FFF772FE15
:1070500022E0702920D12B681A1D2A6019680023AC
:10706000019308230093102213A8FFF783FE13E077
:10707000782911D12968081D2860096801970092B4
:10708000102213A8FFF776FE06E02B681A1D2A606F
:10709000197813A8FFF74EFE0134169B002B23DB53
:1070A00014F8011B01B325293FF454AF13A8FFF7CF
:1070B00041FEF2E72968081D2860096801970092DF
:1070C0000A2213A8FFF7C4FEE6E72B681A1D2A6000
:1070D0001F6817F8011B0029DED013A8FFF72AFE4E
:1070E000169B002BF5DAD7E7169B002B05DD159ACA
:1070F00032B9159A169B13441693169819B0F0BD21
:1071000003A93046FFF7EAFDF3E700BF0EB400B570
:1071100082B003AB53F8041B02AA42F8043DFFF708
:107120000BFF02B05DF804EB03B0704730B40346C8
:10713000002010C920CA641910C310C920CA6C41AC
:1071400010C310C920CA6C4110C310C920CA6C41B9
:1071500010C310C920CA6C4110C310C920CA6C41A9
:1071600010C310C920CA6C4110C310C920CA6C4199
:1071700010C3404130BC704730B4002310C920CA4E
:10718000641B10C010C920CAAC4110C010C920CA6D
:10719000AC4110C010C920CAAC4110C010C920CAEF
:1071A000AC4110C010C920CAAC4110C010C920CADF
:1071B000AC4110C010C920CAAC4110C05B41B3FA49
:1071C00083F0400930BC70472DE9F041013B9B0042
:1071D000002425462646A4465FF0000E03E05FEA41
:1071E0000C0EBEEB030EBCEB0E0752F8078051F8F5
:1071F0000E70A7FB0878E41955EB080556F1000658
:107200001EF1040E9E4501DCE645ECDD40F80C4025
:107210002C46354600261CF1040C9C45DCDDBCEBFD
:10722000430FDCDD40F80C40BDE8F081002304E0B2
:10723000002240F8232001335BB28B42F8DB704719
:1072400000231A468B420DDA10B450F82340224333
:1072500001335BB28B42F8DBB2FA82F040095DF891
:10726000044B7047B3FA83F0400970474B1150F854
:10727000230001F01F01012303FA01F108407047C8
:10728000013949B201E0013949B2002903DB50F864
:107290002130002BF7D0013148B2704710B50446B9
:1072A000FFF7EEFF90B1024600F18043013B54F836
:1072B0002330002101E05B080131002BFBD1501E7F
:1072C00080B2400180B2084400B210BD0020FCE74B
:1072D000002393420BDA10B451F8234040F82340C6
:1072E00001335BB29342F7DB5DF8044B70477047A4
:1072F000013A52B2002A14DB10B450F8224051F87F
:1073000022309C4208D809D3013A52B2002AF4DA5A
:1073100000205DF8044B70470120FAE74FF0FF3082
:10732000F7E70020704730B4013A52B2002407E07A
:1073300050F8223051F822506B401C43013A52B2AF
:10734000002AF5DAB4FA84F0400930BC704730B551
:1073500089B0154613460A4601466846FFF70CFFFA
:10736000041C18BF012429466846FFF769FF640022
:10737000002814BF6042C4F1010009B030BD10B450
:1073800000EB8101002307E051F8042C43EA52038B
:1073900041F8043CD30721460C1F8142F4D85DF824
:1073A000044B704770B505461E469DF910402346B4
:1073B000FFF7BCFE30B9224629463046FFF798FF5A
:1073C000012805D02346324629462846FFF7D4FE39
:1073D00070BD70B505461E469DF910402346FFF767
:1073E000CBFE00B970BD2346324629462846FFF73A
:1073F0009DFEF7E730B591B005461C4693F9003085
:107400006846FFF7E1FED4F8AC3069462846984755
:1074100011B030BD08B513460A46FFF7EBFF08BDB3
:1074200070B506461446006810F001050ED12146DD
:107430003046FFF7A4FF45B104F18044013C56F803
:10744000243043F0004346F8243070BD13460A460A
:1074500031463046FFF76AFE0546E8E7F0B5A1B0D1
:1074600007460E4615461C4619463046FFF7E8FE0D
:10747000A0B92246314618A8FFF72AFF224629461E
:1074800010A8FFF725FF214608A8FFF7CFFE01232C
:10749000089321466846FFF7C9FE0DE021463846AD
:1074A000FFF7C4FE71E0214618A8FFF768FF2246E7
:1074B000294608A8FFF7B4FF224610A918A8FFF72D
:1074C00017FF024600285BD0189B13F0010FEAD08B
:1074D000109B13F0010F1ED0002A2DDD234610AAA9
:1074E00018A90846FFF748FE214618A8FFF747FFEE
:1074F0002246694608A8FFF7FBFE002815DB234655
:107500006A4608A90846FFF737FE2246294608A81A
:10751000FFF786FFD0E7214610A8FFF730FF22468D
:1075200029466846FFF77CFFC6E723462A4608A996
:107530000846FFF7FBFDE2E7234618AA10A9084614
:10754000FFF71AFE214610A8FFF719FF224608A9E7
:107550006846FFF7CDFE00280BDB234608AA6946E4
:107560006846FFF709FE224629466846FFF758FF9E
:10757000A2E723462A4669466846FFF7D7FDECE7AF
:10758000224608A93846FFF7A3FE21B0F0BD2DE939
:10759000F04792B00546894614461F4693F90060AD
:1075A00031461046FFF74CFE10B112B0BDE8F0872F
:1075B0003A4649460AA8FFF72DFF3B460AAA294644
:1075C00002A8FFF717FF3A460AA90846FFF722FF6D
:1075D0003B46224649464846FFF70CFF3A462146BD
:1075E0002046FFF717FF07F104080096434622469E
:1075F00029462846FFF7D6FE0096434622462146F6
:107600002046FFF7CFFE00964346224629462046F5
:10761000FFF7DFFE3B46224629462846FFF7EAFEF3
:10762000009643462A4629462046FFF7BBFE0096B1
:107630004346224629462846FFF7B4FE0021284645
:10764000FFF714FE00284AD0334642462946284612
:10765000FFF76CFD824631462846FFF790FE06F1A3
:107660008043013B55F8232042EACA7245F82320A3
:107670003A4629462046FFF7CDFE0096434602AA29
:1076800021462046FFF7A5FE0096434602AA214662
:107690002046FFF79EFE00964346224602A9084672
:1076A000FFF797FE3B4602AA29462846FFF7A2FEAF
:1076B000009643460AAA29461046FFF78AFE32463C
:1076C00021462846FFF704FE324649462046FFF78A
:1076D000FFFD32460AA94846FFF7FAFD65E7314645
:1076E0002846FFF74CFEC3E72DE9F0438BB0044674
:1076F0008946164600230393049305930693079344
:10770000089309930AAF032347F8203D154615F95E
:10771000048BFFF77FFECDF800802B463A462146CA
:107720002046FFF756FE33464A4621462046FFF7DD
:1077300061FECDF800802B4606F1840221462046EA
:10774000FFF730FE0BB0BDE8F0830000F0B589B064
:1077500006460C460822FFF7BBFD0027029701975B
:107760000097E36A0393236B0493636B0593A36B06
:107770000693E36B079308236A4669466846FFF75A
:10778000D5FC054608236A4631463046FFF7CEFC55
:107790000544236B0393636B0493A36B0593E36B23
:1077A0000693079708236A4669466846FFF7BEFCBA
:1077B000054408236A4631463046FFF7B7FC0544C6
:1077C000236A0093636A0193A36A0293059704975F
:1077D0000397A36B0693E36B079308236A4631462E
:1077E0003046FFF7A3FC0544636A0093A36A019344
:1077F000E36A0293636B0393A26B0492E26B0592BC
:107800000693236A079308236A4631463046FFF7FA
:107810008DFC0544E36A0093236B0193636B029331
:10782000059704970397236A0693A36A079308238F
:107830006A4631463046FFF79FFC2D1A236B0093B2
:10784000636B0193A36B0293E36B03930597049718
:10785000636A0693E36A079308236A463146304613
:10786000FFF78AFC2D1A636B0093A36B0193E36B04
:107870000293236A0393636A0493A36A05930697AA
:10788000236B079308236A4631463046FFF774FCA2
:107890002D1AA36B0093E36B01930297636A039322
:1078A000A36A0493E36A05930697636B079308231F
:1078B0006A4631463046FFF75FFC2D1A0FD5082384
:1078C0000C4A31463046FFF731FC2D18F7D40FE053
:1078D0000823084A31463046FFF74EFC2D1A002D8A
:1078E000F6D1082231460348FFF702FD0128EFD107
:1078F00009B0F0BD70FC0300F0B589B007460D4635
:1079000016461C461A4631466846FFF783FD234655
:107910006A4639463846FFF76DFD234632466946CA
:107920006846FFF767FD23466A4629462846FFF763
:1079300061FD09B0F0BD2DE9F04389B005460E4662
:10794000904699461099119C94F9007019B33A46E3
:107950006846FFF7BDFC3A4629464046FFF7B8FCAB
:107960003A4631464846FFF7B3FC23466A4631465D
:107970002846FFF7C1FFD4F8A47023466A46314673
:107980002846B84723466A4649464046FFF7B4FFB3
:1079900009B0BDE8F08339466846FFF747FC01238C
:1079A0000093D8E72DE9F0438BB080468946144612
:1079B0001F46129D15F9046B00962B460246214680
:1079C00002A8FFF706FD129A02A90846FFF722FD5A
:1079D000129B02AA41464046FFF70CFD129B02AAE9
:1079E00021462046FFF706FD00962B464A463946BB
:1079F0003846FFF7EEFC129A394602A8FFF70AFD57
:107A000000962B46424602A90846FFF7E2FC009684
:107A10002B46224602A90846FFF7DBFC00962B46C0
:107A2000424621462046FFF7D4FC129B2246494697
:107A30004846FFF7DFFC00962B4602AA4146204647
:107A4000FFF7C7FC129B224639463846FFF7D2FCA7
:107A500000962B464A4639463846FFF7BAFC32466E
:107A600002A92046FFF734FC0BB0BDE8F0832DE9F6
:107A7000F0439BB00746894616469846229C14F967
:107A8000045B009523460246314612A8FFF7A1FC8D
:107A9000229A12A90846FFF7BDFC229B12AA39467A
:107AA0003846FFF7A7FC229B12AA31463046FFF763
:107AB000A1FC009523464A46414612A8FFF772FCF6
:107AC000009523464A4641464046FFF782FC009512
:107AD00023463A4631460AA8FFF77BFC229B0AAAB6
:107AE00049464846FFF786FC00952346324639460C
:107AF0000AA8FFF757FC229A41463046FFF78AFC56
:107B0000009523460AAA31463046FFF762FC0095ED
:107B100023463246394602A8FFF75BFC229B02AAA5
:107B200041464046FFF766FC009523464A464146DB
:107B30004046FFF74EFC229A12A902A8FFF76AFC02
:107B4000009523460AAA02A90846FFF742FC0095C1
:107B500023463A4602A90AA8FFF73BFC229B12AA39
:107B60000AA90846FFF746FC009523464A460AA99B
:107B70004846FFF72EFC2A4602A93846FFF7A8FB25
:107B80001BB0BDE8F0832DE9F04FAFB004900D4677
:107B9000059102921C46DDF8E48098F900A0524657
:107BA00026A8FFF795FB4FEA8A0B2B465B4403930D
:107BB0005246194616A8FFF78BFBCDF804800094B7
:107BC0000EAB1EAA16A926A8FFF7B5FEBDF9E06008
:107BD000023E36B2474624E031460298FFF746FBA4
:107BE000B0FA80F04009C0F1010464011EAB1D1918
:107BF0000EAB1C4440011EAB03EB00080EAB03EBC5
